:100000000C9499320C94CA320C94CA320C94CA32B1
:100010000C94CA320C9446690C94CA320C94CA32BD
:100020000C94CB680C94CA320C94CA320C94FFCB5B
:100030000C94CA320D94A0BD0C94CA320C94CA32EE
:100040000C94CA320D94621C0C94CA320C94CA32BD
:100050000C94CA320C94CA320D9400330D94C7B577
:100060000C94CA320C943C3F0C94CA320C94CA32A1
:100070000C94CA320C94CA320C94CA320C94CA3210
:100080000C94CA320C94CA320C94CA320C94CA3200
:100090000C94803F0C94CA320C94CA320C94CA322D
:1000A0000C94CA320C94CA320C94CA320C94CA32E0
:1000B0000C94CA320C94CA320C94CA320C94CA32D0
:1000C0000C94CA320C94CA320C94CA320C94CA32C0
:1000D0000C94CA320C94CA320C94CA320C94CA32B0
:1000E0000C94CA322B3E2F3E343E3C3E513E6A3E7B
:1000F0008F3EB93E6C014801EE01C201C001800192
:10010000E6018A01C601A60160014001580184018F
:10011000D601CC01F40164014A01E001EC013E0189
:100120003601D201DA012C012C012C01AE01AE0105
:10013000AE01C401F601AE019A01700186016601AB
:10014000BC019801D40134017201880144015E01AF
:1001500050016E017A01D40154015A01E201AA0151
:100160005201D8012A0132015601BA014E0146015D
:100170008C018201B6017601AC015601B2013C014D
:10018000EA01084AD73B3BCE016E84BCBFFDC12FBC
:100190003D6C74319ABD56833DDA3D00C77F11BE78
:1001A000D9E4BB4C3E916BAAAABE000000803F057B
:1001B000A84CCDB2D44EB93836A9020C50B99186AC
:1001C00088083CA6AAAA2ABE000000803F07634216
:1001D00036B79BD8A71A39685618AEBAAB558C1DDE
:1001E0003CB7CC5763BD6DEDFD753EF6177231BF60
:1001F000000000803F08000000BE922449123EAB80
:10020000AAAA2ABECDCCCC4C3E00000080BEABAA30
:10021000AAAA3E00000000BF000000803F000000CE
:100220000000084178D3BB4387D1133D190E3CC36E
:10023000BD4282AD2B3E68EC8276BED98FE1A93EED
:100240004C80EFFFBE01C4FF7F3F000000000000B4
:100250000D940E9A0D94B7B70D949F720D942E4C79
:100260000D9492B80D94BDB70D9430B70D9465728E
:100270000D94AD420D94EFAB0D94F2B70D94427214
:100280000D9485700D945B960D944AB70D94D2B77A
:100290000D9454600D94F1710D946A880D94CCB74F
:1002A0000D945EB70D94C4B70D9481B70D94FBB750
:1002B0000D949D700D948BB70D9407860D9454B7D3
:1002C0000D9418610D9445A10D9429710D9412B7E8
:1002D0000D942D4B0D94E43F0D943F600D946DB73C
:1002E0000D9408B70D9438B70D94CC5F0D94E4B716
:1002F0000D947C8F0D9477B70D947B3D0D948F6793
:100300000D949D600D94DAB70D94B4700D940DB7F3
:100310000D9440B70D94C1600D94D6B70D94B3649D
:100320000D9454410D940C880D946D5D0D94B15C49
:100330000D9426B70D94B1720D94DD3E0D94237F7C
:100340000D9454510D94A85C0D9429540D94F060B3
:100350000D94C35C0D94C1B70D94E8B70D94C572AC
:100360000D947A4C0D94EEB70D949B4B0D94E0B721
:100370000D943C5B0D94C8B70D941CB70D94984236
:100380000D9498600D9473600D94A7720D94D660CF
:100390000D94B5910D9461410D94DE700D94BA5C8D
:1003A0000D9423870D948F720D949FB70D94CA708E
:1003B0000D94B3B70D9497720D94A7420D94BC445D
:1003C0000D9414720D9495B70D94995E0D94A760D9
:1003D0000D94A1590D94F6B70D9425720D945960A2
:1003E0000D94004C0D943BA70D940C710D94D57297
:1003F00048617264636F6465642044656661756C0E
:10040000742053657474696E6773204C6F61646502
:10041000640053746F7265642073657474696E67E9
:1004200073207265747269657665640046696C61F3
:100430006D656E742073657474696E67733A2044D9
:10044000697361626C6564002020204D3230302079
:10045000440046696C616D656E74207365747469DF
:100460006E67733A002020204D323039205300410E
:1004700075746F2D526574726163743A20533D3008
:1004800020746F2064697361626C652C2031207464
:100490006F20696E7465727072657420657874720D
:1004A0007564652D6F6E6C79206D6F766573206154
:1004B00073207265747261637473206F7220726549
:1004C000636F766572696573002046002020204DB9
:1004D0003230382053005265636F7665723A20538C
:1004E0003D4578747261206C656E67746820286D74
:1004F0006D2920463A537065656420286D6D2F6D17
:100500002900205A002046002020204D323037207C
:100510005300526574726163743A20533D4C656EAA
:1005200067746820286D6D2920463A5370656564AC
:1005300020286D6D2F6D29205A3A205A4C69667417
:1005400020286D6D29002044002049002020204DE6
:10055000333034205000504944206865617462652E
:10056000642073657474696E67733A0020440020D8
:1005700049002020204D3330312050005049442084
:1005800073657474696E67733A00205A00205900CD
:1005900020204D323036205800486F6D65206F6640
:1005A0006673657420286D6D293A00204500205A35
:1005B0000020590020580020420020540020204DE7
:1005C000323035205300416476616E636564207675
:1005D00061726961626C65733A20533D4D696E20AA
:1005E000666565647261746520286D6D2F73292CB2
:1005F00020543D4D696E2074726176656C2066658D
:1006000065647261746520286D6D2F73292C2042FA
:100610003D6D696E696D756D207365676D656E748E
:100620002074696D6520286D73292C20583D6D61FB
:1006300078696D756D205859206A65726B20286D38
:100640006D2F73292C20205A3D6D6178696D756D71
:10065000205A206A65726B20286D6D2F73292C201B
:1006600020453D6D6178696D756D2045206A657224
:100670006B20286D6D2F73290020540020204D32EF
:100680003034205300416363656C65726174696F37
:100690006E3A20533D616363656C65726174696F86
:1006A0006E2C20543D7265747261637420616363C3
:1006B000656C65726174696F6E00204500205A0098
:1006C00020590020204D3230312058004D6178698A
:1006D0006D756D20416363656C65726174696F6EE1
:1006E00020286D6D2F7332293A00204500205A00D2
:1006F00020590020204D3230332058004D61786958
:100700006D756D2066656564726174657320286D12
:100710006D2F73293A00204500205A0020590020EF
:10072000204D393220580053746570732070657203
:1007300020756E69743A0053657474696E6773202E
:1007400053746F72656400454550524F4D20457299
:10075000726F720029002C20002C200070687973C1
:100760006963616C20636F6F7264696E6174657335
:100770003A20280029002C20002C2000776F726C72
:100780006420636F6F7264696E617465733A2028C8
:10079000006F6B0A002046002045004731205A00B8
:1007A0004D3234004D32362053256C75004D3130BA
:1007B000362053004D38320047312046256400472B
:1007C000312045322A312046343830004731205A12
:1007D0000020463230303000205900473120580088
:1007E0004D383300506F736974696F6E20726561A4
:1007F000642066726F6D20656570726F6D3A004D92
:100800003233202573002E67636F0046656564727E
:100810006174653A007265636F7665725F6D6163DE
:1008200068696E655F73746174655F616674657233
:100830005F706F7765725F70616E69632C20696E9F
:10084000697469616C20007265636F7665725F6DB3
:10085000616368696E655F73746174655F61667416
:1008600065725F706F7765725F70616E69632C206F
:10087000696E697469616C200047393220450063F4
:10088000757272656E745F706F736974696F6E5B99
:10089000455F415849535D3A0063757272656E74E5
:1008A0005F706F736974696F6E5B5A5F415849532B
:1008B0005D3A0043757272656E7420706F7369746F
:1008C000696F6E20595F415849533A0043757272FF
:1008D000656E7420706F736974696F6E20585F4124
:1008E0005849533A004166746572207761697469AA
:1008F0006E6720666F722074656D703A0047312014
:10090000452D3120463438300047312045352046CA
:10091000313230004D3833004D31393020532564A9
:10092000004D31303920532564004732382058209B
:1009300059004731205A32352046383030004D3189
:10094000343020532564004D313034205325640069
:10095000494E54340055564C4F202D20656E64008E
:10096000737470730020423A0020453A00543A00F4
:100970005A206C6976652061646A757374206F759E
:1009800074206F662072616E67652E2053657474E3
:10099000696E6720746F20302E20436C69636B2072
:1009A000746F20636F6E74696E75652E005A206CCB
:1009B0006976652061646A757374206F7574206F41
:1009C000662072616E67652E2053657474696E6768
:1009D00020746F20300020573A0020453A00543AE6
:1009E000004B494C4C3A20004D3730310022283220
:1009F00029005400496E76616C6964205420636F4D
:100A000064652E00556E6B6E6F776E204D20636FA0
:100A100064653A202573200A004D32323020532578
:100A20006900203A2000004C414E472053454C209D
:100A3000464F5243454400222831290020453A00C0
:100A4000205A3A0020593A0020453A00205A3A00EC
:100A500020593A00583A004D3131332053002000DC
:100A60002E0020423A0020453A00543A0020413AF4
:100A70000020503A002042403A0020403A00202F07
:100A8000003A00205400202F0020423A00202F007E
:100A90006F6B20543A002569206D696E2C20256902
:100AA0002073656300496E76616C6964204D206334
:100AB0006F64653A202573200A00556E6B6E6F7760
:100AC0006E204720636F64653A202573200A004D2D
:100AD00065736820626564206C6576656C696E6715
:100AE000206E6F74206163746976652E000A0020A1
:100AF00020000A4D6561737572656420706F696EC0
:100B000074733A000A5A20736561726368206865DD
:100B1000696768743A20002C004E756D20582C5976
:100B20003A2000206D6963726F6E730045786365CB
:100B3000737369766520626564206C6576656C699F
:100B40006E6720636F7272656374696F6E3A20001E
:100B5000473238205730003A200054656D70657276
:100B600061747572652063616C6962726174696F2A
:100B70006E20646F6E652E20436F6E74696E7565AE
:100B80002077697468207072657373696E6720746A
:100B90006865206B6E6F622E0000205A20736869B2
:100BA000667420286D6D293A0050494E44412074E6
:100BB000656D70657261747572653A2000002F363C
:100BC00000537465703A200000205A2073686966EB
:100BD0007420286D6D293A0050494E4441207465B7
:100BE0006D70657261747572653A20002F36202829
:100BF000736B69707065642900537465703A2000E6
:100C0000005A45524F3A2000007374617274207488
:100C1000656D70657261747572653A200050494E59
:100C200044412070726F62652063616C6962726119
:100C300074696F6E20737461727400473238205784
:100C400030000A00205A3A200020593A200020584B
:100C50003A200043616C6962726174696F6E20664C
:100C600061696C65642120436865636B2074686505
:100C7000206178657320616E642072756E206167F3
:100C800061696E2E0043524153485F4445544543C9
:100C900054454458590043524153485F44455445D4
:100CA00043544544590043524153485F44455445D9
:100CB0004354454458004D323900627573793A20E7
:100CC00070617573656420666F7220696E707574EB
:100CD00000627573793A2070617573656420666F80
:100CE00072207573657200627573793A2070726F45
:100CF00063657373696E67002055706C6F61642063
:100D0000696E2070726F6772657373004449534156
:100D1000424C45440A00454E41424C45440A004677
:100D200053656E736F722000504154393132355F14
:100D3000696E69743A25640A004665622020312094
:100D40003230313800436F6D70696C65643A200051
:100D5000286E6F6E652C2064656661756C74206307
:100D60006F6E666967290046656220203120323047
:100D700031382032303A30313A34360020332E3197
:100D80002E312D5243352D3135310A007374617285
:100D90007400466163746F72792052455345540064
:100DA0001B5B324A1B5B313B31484F726967696E8E
:100DB000616C2050727573612069331B5B323B3369
:100DC0004850727573612052657365617263680083
:100DD000250020202020202000202020202020006E
:100DE00045524153494E4720616C6C2064617461E7
:100DF00000466163746F7279205245534554004335
:100E0000524153485F5245434F564552004732388E
:100E10002058205900FFFFFF0000A0400000A04024
:100E20000000004000007F43000056439AD9514320
:100E300000000000000080C09A99193E00007F4326
:100E4000000052430000524300000000000080C038
:100E50009A99193E6563686F3A004572726F723AEB
:100E60000000002110422063308440A550C660E796
:100E700070088129914AA16BB18CC1ADD1CEE1EF4F
:100E8000F13112100273325222B5529442F772D6E7
:100E900062399318837BB35AA3BDD39CC3FFF3DE9F
:100EA000E36224433420040114E664C774A4448537
:100EB000546AA54BB528850995EEE5CFF5ACC58DEF
:100EC000D55336722611163006D776F6669556B487
:100ED000465BB77AA719973887DFF7FEE79DD7BC3F
:100EE000C7C448E5588668A77840086118022823D7
:100EF00038CCC9EDD98EE9AFF9488969990AA92B8F
:100F0000B9F55AD44AB77A966A711A500A333A1226
:100F10002AFDDBDCCBBFFB9EEB799B588B3BBB1ADE
:100F2000ABA66C877CE44CC55C222C033C600C4176
:100F30001CAEED8FFDECCDCDDD2AAD0BBD688D492E
:100F40009D977EB66ED55EF44E133E322E511E70C6
:100F50000E9FFFBEEFDDDFFCCF1BBF3AAF599F787E
:100F60008F8891A981CAB1EBA10CD12DC14EF16F2F
:100F7000E18010A100C230E3200450254046706794
:100F800060B9839893FBA3DAB33DC31CD37FE35EC0
:100F9000F3B1029012F322D23235421452776256E4
:100FA00072EAB5CBA5A89589856EF54FE52CD50DD0
:100FB000C5E234C324A01481046674476424540534
:100FC00044DBA7FAB79987B8975FE77EF71DC73C60
:100FD000D7D326F2369106B0165766767615463484
:100FE000564CD96DC90EF92FE9C899E9898AB9AB70
:100FF000A94458654806782768C018E1088238A3D4
:10100000287DCB5CDB3FEB1EFBF98BD89BBBAB9AFF
:10101000BB754A545A376A167AF10AD01AB32A9223
:101020003A2EFD0FED6CDD4DCDAABD8BADE89DC90F
:101030008D267C076C645C454CA23C832CE01CC173
:101040000C1FEF3EFF5DCF7CDF9BAFBABFD98FF89F
:101050009F176E367E554E745E932EB23ED10EF0C3
:101060001E7C3C3E5E2B3D3F2F5B5D3B2C2A225C71
:10107000004D3234004D3233202573006175746F9A
:1010800025692E67000A002F000A002E0044656CB7
:101090006574696F6E206661696C65642C204669B1
:1010A0006C653A200046696C652064656C65746502
:1010B000643A002E002E002E002E004E6F77206620
:1010C000726573682066696C653A20004E6F772000
:1010D000646F696E672066696C653A200022207033
:1010E0006F73002220706172656E743A220053554E
:1010F00042524F5554494E452043414C4C20746157
:10110000726765743A2200747279696E6720746F31
:101110002063616C6C207375622D67636F6465205A
:1011200066696C6573207769746820746F6F206DD1
:10113000616E79206C6576656C732E204D41582068
:101140006C6576656C2069733A00256920686F7557
:101150007273202569206D696E757465730054493A
:101160004D454F55543A004D3131300046756C6C49
:1011700020525820427566666572002220666169B9
:101180006C65643A204275666665722066756C6CA3
:101190002100456E717565696E6720746F207468F3
:1011A000652066726F6E743A2022002200456E71CF
:1011B0007565696E6720746F207468652066726F4C
:1011C0006E743A20220022206661696C65643A20C0
:1011D0004275666665722066756C6C210022004D52
:1011E000363030004731204533204632303000471A
:1011F0003120452D332046323030005072757361F6
:10120000206933204D4B33206F6B00507275736132
:10121000206933204D4B332072656164792E007A4A
:101220005F6D696E3A20007A5F6D61783A20005AEE
:10123000204F666673657400795F6D696E3A2000B1
:10124000795F6D61783A20005920767A64616C6527
:101250006E6F7374206F64206D696E3A005920645C
:10126000697374616E63652066726F6D206D696E5F
:101270003A00416E6F0059657300785F6D696E3A90
:101280002000785F6D61783A200044657461696C74
:10129000792058595A206B616C2E0058595A206396
:1012A000616C2E2064657461696C73004E796E699F
:1012B0002070726F76656475207A206B616C69624C
:1012C000726163692E00492077696C6C2072756EBB
:1012D000207A2063616C6962726174696F6E206E3E
:1012E0006F772E004E796E692070726F7665647527
:1012F0002078797A206B616C6962726163692E2053
:101300005A616265726520746F20707269626C69DF
:101310007A6E65203132206D696E2E004920776922
:101320006C6C2072756E2078797A2063616C6962CA
:10133000726174696F6E206E6F772E20497420770A
:10134000696C6C2074616B6520617070726F782EAF
:10135000203132206D696E732E004E796E692070D7
:10136000726564656872656A6920747279736B75F9
:101370002070726F20504C412E004E6F7720492014
:1013800077696C6C2070726568656174206E6F7A25
:101390007A6C6520666F7220504C412E00446F625B
:1013A00072792064656E2C206A73656D2076617396
:1013B00065207469736B61726E61204F7269676931
:1013C0006E616C2050727573612069332E20436802
:1013D000636574652061627963682056617320706B
:1013E000726F7665646C61206B616C6962726163B7
:1013F0006E696D2070726F636573656D3F0048693B
:101400002C204920616D20796F7572204F726967B9
:10141000696E616C2050727573612069332070723F
:10142000696E7465722E20576F756C6420796F75C4
:10143000206C696B65206D6520746F206775696429
:101440006520796F75207468726F7567682074689D
:10145000652073657475702070726F636573733F78
:10146000005A61636E75207469736B6E6F757420BA
:101470006C696E6B752061205679206275646574A5
:101480006520706F737475706E6520736E697A6F06
:1014900076617420747279736B75206F7461636503
:1014A0006E696D20746C616369746B6120646F6B2D
:1014B0007564206E65646F7361686E657465206F16
:1014C0007074696D616C6E69207679736B792E200A
:1014D00050726F686C65646E657465207369206F07
:1014E0006272617A6B792076206E61736920707206
:1014F0006972756363652076206B617069746F6CC7
:1015000065204B616C69627261636500492077698F
:101510006C6C20737461727420746F207072696EC9
:1015200074206C696E6520616E6420796F75207718
:10153000696C6C206772616475616C6C79206C6F8A
:1015400077657220746865206E6F7A7A6C652062A8
:101550007920726F746174696E6720746865206B9E
:101560006E6F622C20756E74696C20796F752072B5
:1015700065616368206F7074696D616C206865696E
:101580006768742E20436865636B207468652070FB
:101590006963747572657320696E206F7572206857
:1015A000616E64626F6F6B20696E20636861707436
:1015B00065722043616C6962726174696F6E2E009E
:1015C0004E796E69207A6B616C696272756A692006
:1015D000767A64616C656E6F7374206D657A6920CC
:1015E0006B6F6E63656D20747279736B7920612007
:1015F000706F76726368656D20686561746265649A
:10160000752E004E6F7720492077696C6C206361DE
:101610006C6962726174652064697374616E63657C
:10162000206265747765656E20746970206F66202E
:10163000746865206E6F7A7A6C6520616E642068CC
:1016400065617462656420737572666163652E00FE
:101650004E656A6472697620706F6D6F636920737E
:10166000656C667465737475207A6B6F6E746F6CDD
:10167000756A69206E656A63617374656A7369204F
:10168000636879627920767A6E696B616A696369E9
:101690002070726920736573746176656E69207459
:1016A00069736B61726E792E0046697273742C20B7
:1016B000492077696C6C2072756E207468652073A0
:1016C000656C667465737420746F20636865636B02
:1016D000206D6F737420636F6D6D6F6E2061737317
:1016E000656D626C792070726F626C656D732E002F
:1016F0005370757374656E692057697A617264619D
:101700002076796D617A6520756C6F7A656E6520DB
:101710007679736C65646B79207673656368206B8A
:10172000616C6962726163692061207370757374A2
:1017300069206B616C69627261636E692070726F9F
:10174000636573206F64207A616361746B752E200A
:10175000506F6B7261636F7661743F0052756E6E8D
:10176000696E672057697A6172642077696C6C20B2
:1017700064656C6574652063757272656E74206350
:10178000616C6962726174696F6E20726573756CE9
:10179000747320616E642073746172742066726F5A
:1017A0006D2074686520626567696E6E696E672E6C
:1017B00020436F6E74696E75653F0043686365749E
:1017C00065206F70616B6F76617420706F736C65EC
:1017D000646E69206B726F6B206120706F7A6D652B
:1017E0006E697420767A64616C656E6F7374206DB7
:1017F000657A6920747279736B6F752061206865F2
:1018000061746265643F00446F20796F7520776171
:101810006E7420746F20726570656174206C6173E2
:1018200074207374657020746F20726561646A75CA
:1018300073742064697374616E6365206265747784
:1018400065656E206E6F7A7A6C6520616E642068C3
:101850006561746265643F0057697A6172646120F2
:101860006D757A657465206B64796B6F6C69762031
:101870007A6E6F76752073707573746974207A2030
:101880006D656E752043616C6962726174696F6E1B
:10189000202D3E2057697A61726400596F7520636C
:1018A000616E20616C7761797320726573756D6507
:1018B000207468652057697A6172642066726F6D62
:1018C0002043616C6962726174696F6E202D3E20E5
:1018D00057697A6172642E004A6520746F20504CFB
:1018E000412066696C616D656E743F0049732069C3
:1018F0007420504C412066696C616D656E743F00C8
:1019000050726F73696D20766C6F7A746520504CDD
:10191000412066696C616D656E7420646F20657826
:10192000747275646572752C20706F2074652073F5
:101930007469736B6E65746520746C616369746B34
:101940006F2070726F207A61766564656E692066BB
:10195000696C616D656E74752E00506C65617365A0
:1019600020696E7365727420504C412066696C6109
:101970006D656E7420746F2074686520657874726C
:10198000756465722C207468656E2070726573735F
:10199000206B6E6F6220746F206C6F6164206974BD
:1019A0002E0050726F73696D207A6176656474657C
:1019B00020504C412066696C616D656E7420612019
:1019C000706F207465206F626E6F76746520576942
:1019D0007A6172646120737469736B6E7574696D7A
:1019E00020726573657420746C616369746B612E19
:1019F00000506C65617365206C6F616420504C41D0
:101A00002066696C616D656E7420616E6420746817
:101A1000656E20726573756D652057697A617264B1
:101A2000206279207265626F6F74696E67207468D6
:101A300065207072696E7465722E005072656465FF
:101A400068726976616D20747279736B752E20509F
:101A5000726F73696D2063656B656A74652E0050E3
:101A6000726568656174696E67206E6F7A7A6C65FD
:101A70002E20506C6561736520776169742E004A71
:101A8000652066696C616D656E74207A6176656447
:101A9000656E3F0049732066696C616D656E7420E8
:101AA0006C6F616465643F00567365206A652068E9
:101AB0006F746F766F2E00416C6C20697320646FB9
:101AC0006E652E204861707079207072696E74693D
:101AD0006E67210050726F73696D206F6369737454
:101AE0006574652068656174626564206120737443
:101AF00069736B6E65746520746C616369746B6F78
:101B00002E00506C6561736520636C65616E2068A2
:101B100065617462656420616E64207468656E201E
:101B2000707265737320746865206B6E6F622E002F
:101B300050726F73696D206E61686C65646E657458
:101B40006520646F206D616E75616C752061206F1A
:101B50007072617674652070726F626C656D2E2094
:101B6000506F207465206F626E6F767465205769C0
:101B70007A61726461207265626F6F746F76616EF4
:101B8000696D207469736B61726E792E00506C659B
:101B900061736520636865636B206F75722068618F
:101BA0006E64626F6F6B20616E642066697820746A
:101BB00068652070726F626C656D2E205468656E6A
:101BC00020726573756D65207468652057697A6148
:101BD0007264206279207265626F6F74696E67202B
:101BE000746865207072696E7465722E0057697A28
:101BF00061726400205761746368646F6720526586
:101C000073657400496E666F726D61636500496E3D
:101C1000666F2073637265656E0043656B616E6904
:101C2000206E61207A63686C61646E7574692074DB
:101C30007279736B79206120706F646C6F7A6B7945
:101C40002E0057616974696E6720666F72206E6F2F
:101C50007A7A6C6520616E642062656420636F6FC0
:101C60006C696E67004B616C2E207072766E692015
:101C7000767273747679004669727374206C617938
:101C800065722063616C2E005761697420666F7203
:101C900020757365722E2E2E00506F757A697465EB
:101CA00020626568656D207469736B750055736596
:101CB0006420647572696E67207072696E74004288
:101CC000796C6F20767973756E7574692066696CAE
:101CD000616D656E74752075737065736E653F0018
:101CE0005761732066696C616D656E7420756E6CEA
:101CF0006F6164207375636365737366756C3F0011
:101D000056796A6D6F75742066696C616D656E7465
:101D100000556E6C6F61642066696C616D656E74F0
:101D2000005679736F7576616D2066696C616D65BB
:101D30006E7400556E6C6F6164696E672066696CC5
:101D4000616D656E7400556E6B6E6F776E20636F9C
:101D50006D6D616E643A2022004C616469740054B8
:101D6000756E650053442063617264205B466C733A
:101D7000684169725D005344206361726420205B96
:101D80006E6F726D616C5D00537461626C65206191
:101D90006D6269656E742074656D706572617475CD
:101DA00072652032312D323643206973206E6565AD
:101DB0006465642061207269676964207374616E70
:101DC000642069732072657175697265642E0054B0
:101DD00065706C2E206B616C2E20205B7A61705DCB
:101DE0000054656D702E2063616C2E2020205B6F87
:101DF0006E5D005465706C2E206B616C2E20205B34
:101E00007679705D0054656D702E2063616C2E20B4
:101E1000205B6F66665D005465706C6F746E692040
:101E20006B616C69627261636520646F6B6F6E6376
:101E3000656E612E20506F6B726163756A746520E8
:101E4000737469736B656D20746C616369746B6125
:101E50002E0054656D7065726174757265206361E2
:101E60006C6962726174696F6E2069732066696E55
:101E700069736865642E20436C69636B20746F20FE
:101E8000636F6E74696E75652E005465706C2E20DC
:101E90006B616C2E20202020202020202020005448
:101EA000656D702E2063616C2E2020202020202064
:101EB000202020005465706C6F74610054656D7053
:101EC0006572617475726500506F64706F72610045
:101ED000537570706F7274005A61737461766974AF
:101EE000207469736B0053746F70207072696E7424
:101EF0000053544F505045442E2000537465707267
:101F000061746520746F6F20686967683A20004AC1
:101F100065207469736B6F767920706C6174206EC4
:101F20006120686561746265643F00497320737461
:101F300065656C207368656574206F6E20686561E7
:101F4000746265643F0043656C6B6F7679206361F2
:101F500073203A00546F74616C207072696E742043
:101F600074696D65203A0046696C616D656E742018
:101F700063656C6B656D203A00546F74616C20660C
:101F8000696C616D656E74203A00436173207469F9
:101F9000736B75203A2020005072696E742074694A
:101FA0006D653A20200046696C616D656E74203A5B
:101FB00020200046696C616D656E742075736564E0
:101FC0003A20200053746174697374696B61202036
:101FD00000537461746973746963732020004368EB
:101FE000796261202D20446F736C6F206B207072BA
:101FF0006570697375207374617469636B652070B3
:10200000616D65746921004572726F72202D2073B5
:102010007461746963206D656D6F72792068617396
:10202000206265656E206F7665727772697474657B
:102030006E00527963686C6F7374005370656564E9
:102040000054726964656E6920202020205B436122
:10205000735D00536F72743A2020202020205B545F
:10206000696D655D0054726964656E692020205B4E
:102070005A61646E655D00536F72743A20202020AF
:1020800020205B4E6F6E655D0054726964656E69F9
:10209000205B416265636564615D00536F72743AF1
:1020A00020205B416C7068616265745D00547269E8
:1020B00064656E6920736F75626F727500536F721D
:1020C00074696E672066696C65730020536F66746F
:1020D00077617265205265736574004C65686B6545
:1020E000207A6B6F73656E693A00536C6967687428
:1020F00020736B65773A004D6F6420202020205BB1
:10210000537465616C74685D004D6F6465202020B8
:10211000205B537465616C74685D004D6F642020B2
:10212000202020205B4E6F726D616C5D004D6F64EE
:102130006520202020205B4E6F726D616C5D005326
:10214000746176206B6F6E632E207370696E2E0043
:1021500053686F7720656E642073746F70730054DA
:10216000657A6B65207A6B6F73656E693A005365AB
:102170007665726520736B65773A004E61737461A2
:10218000767465207465706C6F74753A005365746D
:102190002074656D70657261747572653A004E6188
:1021A00073746176656E690053657474696E6773E4
:1021B000004368796261207A61706F6A656E6900B8
:1021C000576972696E67206572726F720050726F24
:1021D000686F7A656E65005377617070656400534F
:1021E000656C66207465737420737461727420204A
:1021F000005469736B6F76792076656E742E3A00A1
:102200005072696E742066616E3A005A6B6F6E741C
:10221000726F6C756A7465203A00506C6561736505
:1022200020636865636B203A0053656C66207465B3
:102230007374204F4B004E657A61706F6A656E6FE4
:1022400020202020004E6F7420636F6E6E656374D3
:102250006564004D6F746F72004865617465722F1C
:10226000546865726D6973746F720053656E7A6F2E
:10227000722066696C616D656E74753A0046696CB2
:10228000616D656E742073656E736F723A00546F82
:102290006369207365005370696E6E696E67004EE6
:1022A00065746F6369207365004E6F742073706985
:1022B0006E6E696E6700507265646E692F6C65762C
:1022C000792076656E742E0046726F6E742F6C6581
:1022D00066742066616E7300546573742076656E53
:1022E00074696C61746F72750046616E20746573F9
:1022F000740053656C66746573742073656C6861F3
:102300006C20200053656C66746573742066616987
:102310006C65642020004C6576792076656E742E9D
:102320003A0045787472756465722066616E3A0091
:102330004C6576792076656E74206E6120747279B2
:102340007363653F004C65667420686F74656E64E6
:102350002066616E3F0053656C667465737420651A
:1023600072726F72202100456E6473746F70206EFC
:102370006F742068697400456E6473746F707300C5
:10238000456E6473746F7000507265646E6920747A
:1023900069736B6F76792076656E743F0046726F55
:1023A0006E74207072696E742066616E3F004B6FB0
:1023B0006E74726F6C61205A2061786973202000FE
:1023C000436865636B696E67205A20617869732082
:1023D00020004B6F6E74726F6C61205920617869B8
:1023E00073202000436865636B696E672059206124
:1023F0007869732020004B6F6E74726F6C61205887
:102400002061786973202000436865636B696E679B
:10241000205820617869732020004B6F6E74726FB2
:102420006C6120686F74656E64202000436865638A
:102430006B696E6720686F74656E642020004B6F57
:102440006E74726F6C612073656E7A6F7275004383
:102450006865636B696E672073656E736F72732056
:10246000004B6F6E74726F6C6120656E6473746F75
:10247000707300436865636B696E6720656E647393
:10248000746F7073004B6F6E74726F6C6120626555
:1024900064202020202000436865636B696E6720FC
:1024A000626564202020202000567365204F4B2059
:1024B0002020202020202020202000416C6C206340
:1024C0006F727265637420202020202000426564B2
:1024D000202F204865617465720044656C6B612033
:1024E0006F73790041786973206C656E677468005A
:1024F0004F736100417869730053656C667465734E
:10250000742020202020202020200052506920709C
:102510006F7274202020205B7A61705D00525069D8
:1025200020706F727420202020205B6F6E5D00523F
:10253000506920706F7274202020205B7679705D66
:102540000052506920706F7274202020205B6F66EB
:10255000665D0057726974696E6720746F206669E2
:102560006C653A2000766F6C756D652E696E6974C6
:10257000206661696C6564002053697A653A2000C1
:102580004B617274612076796A6D75746100436184
:1025900072642072656D6F766564005344207072BA
:1025A000696E74696E67206279746520006F70656A
:1025B0006E206661696C65642C2046696C653A2002
:1025C000006F70656E526F6F74206661696C656430
:1025D000004B6172746120766C6F7A656E610043A6
:1025E00061726420696E736572746564005344207F
:1025F000696E6974206661696C0046696C65207358
:10260000656C65637465640046696C65206F706510
:102610006E65643A20006572726F72207772697419
:10262000696E6720746F2066696C6500534420638F
:10263000617264206F6B0043616E6E6F7420656E13
:10264000746572207375626469723A200050726119
:1026500076793A0052696768743A004F626E6F7615
:102660006F76616E69207469736B7500526573755E
:102670006D696E67207072696E74004F626E6F765E
:10268000656E69207469736B7500526573756D6949
:102690006E67207072696E7400506F6B7261636F49
:1026A00076617400526573756D65207072696E7421
:1026B00000526573656E643A20004F6473747261F2
:1026C0006E7465207469736B6F767920706C6174B9
:1026D000207A20686561746265642070726F736926
:1026E0006D2E00506C656173652072656D6F766547
:1026F00020737465656C2073686565742066726FFD
:102700006D20686561746265642E00446574656B54
:102710006F76616E207679706164656B2070726F80
:102720007564752E4F626E6F766974207469736B71
:102730003F00426C61636B6F7574206F63637572E9
:102740007265642E205265636F76657220707269BF
:102750006E743F004F626E6F766F76616E692074A3
:1027600069736B7520202020005265636F76657257
:10277000696E67207072696E74202020200050728C
:102780006F73696D2076796A6D65746520757279ED
:1027900063686C656E652066696C616D656E74005A
:1027A000506C656173652070756C6C206F7574205A
:1027B00066696C616D656E7420696D6D65646961D3
:1027C00074656C7900686F77746F2E7072757361C1
:1027D00033642E637A00686F77746F2E707275732E
:1027E0006133642E636F6D00666F72756D2E70724B
:1027F00075736133642E637A00666F72756D2E7027
:102800007275736133642E636F6D007072757361DE
:1028100033642E637A00707275736133642E636F54
:102820006D005469736B20706F7A617374617665A3
:102830006E005072696E7420706175736564005427
:1028400069736B20707265727573656E0050726982
:102850006E742061626F72746564005072696E7488
:10286000657220646973636F6E6E6563746564007E
:1028700050726F20767973756E7574692066696C15
:10288000616D656E747520737469736B6E657465C4
:102890002070726F73696D20746C616369746B6F03
:1028A00000506C6561736520707265737320746885
:1028B00065206B6E6F6220746F20756E6C6F616443
:1028C0002066696C616D656E740050726F206E6178
:1028D000687261746920747279736B7920612070F9
:1028E0006F6B7261636F76616E6920737469736B6D
:1028F0006E65746520746C616369746B6F2E005033
:1029000072657373206B6E6F6220746F20707265D6
:1029100068656174206E6F7A7A6C6520616E6420E0
:10292000636F6E74696E75652E00612073746973D0
:102930006B6E65746520746C616369746B6F0061A4
:102940006E6420707265737320746865206B6E6F9F
:10295000620050726564656872656A74652074729D
:1029600079736B75210050726568656174207468B5
:1029700065206E6F7A7A6C652100507265646568B7
:10298000726576005072656865617400506F776596
:102990007255700050726F73696D2063656B656A64
:1029A000746500506C656173652077616974004ED1
:1029B000656A6472697665207A61766564746520FB
:1029C000504C412066696C616D656E742070726F49
:1029D00073696D2E00506C65617365206C6F616466
:1029E00020504C412066696C616D656E742066698B
:1029F0007273742E004A6520504C412066696C61E8
:102A00006D656E74207A61766564656E3F0049730A
:102A100020504C412066696C616D656E74206C6F4E
:102A2000616465643F002020506C616E6E65724287
:102A3000756666657242797465733A2000556D69F2
:102A400073746574652070726F73696D2074697337
:102A50006B6F767920706C6174206E61206865619F
:102A60007462656400506C6561736520706C6163AD
:102A70006520737465656C207368656574206F6E7E
:102A800020686561746265642E004E6168726976C3
:102A9000616E692050494E44410050494E444120E6
:102AA00048656174696E6700504944206B616C2E03
:102AB00020202020202020202020200050494420B9
:102AC00063616C2E20202020202020202020200048
:102AD000504944206B616C2E20756B6F6E63656E80
:102AE00061005049442063616C2E2066696E6973F1
:102AF00068656400504944206B616C69627261636F
:102B000065005049442063616C6962726174696F49
:102B10006E00506F7A6173746176697420746973A2
:102B20006B005061757365207072696E7400556D2D
:102B3000697374657465206C697374207061706961
:102B40007275206E6120706F646C6F7A6B75206196
:102B5000207564727A756A7465206A656A20706F80
:102B60006420747279736B6F7520626568656D207F
:102B70006D6572656E69207072766E696368203467
:102B800020626F64752E20506F6B756420747279AB
:102B9000736B61207A616368797469207061706910
:102BA000722C207679706E657465207469736B6120
:102BB000726E752E00506C616365206120736865CC
:102BC0006574206F6620706170657220756E646533
:102BD0007220746865206E6F7A7A6C6520647572F5
:102BE000696E67207468652063616C6962726174E4
:102BF000696F6E206F66206669727374203420706E
:102C00006F696E74732E20496620746865206E6F3C
:102C10007A7A6C6520636174636865732074686593
:102C20002070617065722C20706F776572206F66FE
:102C30006620746865207072696E74657220696DB3
:102C40006D6564696174656C792E006F6B004F6609
:102C500066004E6F206D6F76652E005A61646E615E
:102C6000205344206B61727461004E6F20534420E6
:102C70006361726400547279736B61004E6F7A7A8B
:102C80006C650046696C616D656E74206E657A6175
:102C9000766564656E0046696C616D656E74206E64
:102CA0006F74206C6F6164656400426172766120AC
:102CB0006E656E6920636973746100436F6C6F7237
:102CC000206E6F7420636F7272656374004E6500CE
:102CD0004E6F0050726F73696D20616B7475616C1B
:102CE000697A756A74652E00506C6561736520752C
:102CF0007067726164652E005679736C61206E6F27
:102D00007661207665727A65206669726D77617288
:102D1000653A004E6577206669726D77617265204D
:102D200076657273696F6E20617661696C61626C41
:102D3000653A00506F73756E6F7574205A004D6F51
:102D40007665205A00506F73756E6F757420590048
:102D50004D6F7665205900506F73756E6F757420D6
:102D600058004D6F7665205800457874727564651B
:102D70007200506F73756E6F7574206F7375004DB0
:102D80006F76652061786973004D657368204265D0
:102D900064204C6576656C696E67004E6170657481
:102DA0006900566F6C7461676573005465706C6F71
:102DB00074790054656D7065726174757265730025
:102DC0004B616C6962726163650043616C69627238
:102DD0006174696F6E00537461762072656D656E03
:102DE000750042656C742073746174757300207A89
:102DF000203900206F662039004D6572696D2072A0
:102E000065666572656E636E69207679736B752091
:102E10006B616C69627261636E69686F20626F6476
:102E200075004D6561737572696E672072656665C0
:102E300072656E636520686569676874206F6620D7
:102E400063616C6962726174696F6E20706F696E24
:102E500074004D6572656E65207A6B6F73656E697F
:102E60003A004D6561737572656420736B65773ADE
:102E700000486C61766E69206E616269646B610006
:102E80004D61696E004D32323120496E76616C6958
:102E90006420657874727564657220004D32313833
:102EA00020496E76616C696420657874727564651A
:102EB0007220004D32303020496E76616C6964209A
:102EC000657874727564657220005265706F7274F3
:102ED000696E6720656E6473746F702073746174BB
:102EE0007573004D313137204B616C2E2070727636
:102EF0006E6920767273747679004D3131372046D1
:102F000069727374206C617965722063616C2E0044
:102F10004649524D574152455F4E414D453A4D61EC
:102F2000726C696E2056312E302E323B20537072F7
:102F3000696E7465722F6772626C206D617368755B
:102F40007020666F722067656E36204649524D5775
:102F50004152455F55524C3A68747470733A2F2F42
:102F60006769746875622E636F6D2F707275736117
:102F700033642F50727573612D69332D506C7573E6
:102F80002F2050524F544F434F4C5F564552534998
:102F90004F4E3A312E30204D414348494E455F5403
:102FA0005950453A5072757361206933204D4B3347
:102FB0002045585452554445525F434F554E543A5C
:102FC0003120555549443A30303030303030302D92
:102FD000303030302D303030302D303030302D30FA
:102FE00030303030303030303030300A004D313019
:102FF0003920496E76616C696420657874727564F5
:10300000657220004D31303520496E76616C6964FF
:1030100020657874727564657220004D31303420FB
:10302000496E76616C696420657874727564657246
:10303000200055766F6C6E656E612072656D656EF1
:1030400069636B61004C6F6F73652070756C6C65A4
:1030500079005A61766573742066696C616D656E7E
:1030600074004C6F61642066696C616D656E7400FC
:103070005A61766164656E692066696C616D656E22
:103080007475004C6F6164696E672066696C616D70
:10309000656E740043697374656E6920626172764F
:1030A00079004C6F6164696E6720636F6C6F7200AA
:1030B0004C6576793A004C6566743A0056796265DB
:1030C00072206A617A796B610053656C6563742064
:1030D0006C616E67756167650043657374696E61E5
:1030E00000456E676C697368004B494C4C45442E33
:1030F0002000496E76616C6964206578747275642D
:10310000657200566C6F7A74652066696C616D65D6
:103110006E7400496E736572742066696C616D65CA
:103120006E74005469736B2E2076656E743A00508D
:1031300072696E742046414E3A2000547279736B66
:103140002E2076656E743A004E6F7A7A6C65204652
:10315000414E3A00457874727564657220696E66F6
:103160006F00207A203400206F662034005A6C658E
:103170007073756A6920707265736E6F7374206BFB
:10318000616C69627261636E69686F20626F6475F9
:1031900000496D70726F76696E67206265642063A6
:1031A000616C6962726174696F6E20706F696E74B0
:1031B000004B616C696272756A69205A0043616CE8
:1031C0006962726174696E67205A004B616C696252
:1031D00072616365204F4B0043616C696272617478
:1031E000696F6E20646F6E65004B616C6962726F0F
:1031F000766174205A0043616C6962726174652063
:103200005A005A6168726976616E69204F4B2E00D0
:1032100048656174696E6720646F6E652E005A613F
:1032200068726976616E690048656174696E6700ED
:103230005641524F56414E493A204E657A6E616D65
:10324000612C206E65706F64706F726F76616E6155
:10325000207665727A65206669726D776172652E77
:1032600020506F757A697469206E6120766C617385
:10327000746E69206E6562657A70656369210057B6
:1032800041524E494E473A20546869732069732071
:10329000616E20756E6F6666696369616C2C20755E
:1032A0006E737570706F72746564206275696C649A
:1032B0002E2055736520617420796F7572206F77A9
:1032C0006E207269736B210043485942413A20468F
:1032D000696C616D656E742073656E7A6F72206EB5
:1032E0006572656167756A652C207A6B6F6E7472A2
:1032F0006F6C756A7465207A61706F6A656E692E8D
:10330000004552524F523A2046696C616D656E74A9
:103310002073656E736F72206973206E6F742072F4
:103320006573706F6E64696E672C20706C65617375
:103330006520636865636B20636F6E6E6563746997
:103340006F6E2E00462E206175746F7A61762E2086
:103350005B7A61705D00462E206175746F6C6F61E1
:103360006420205B6F6E5D00462E206175746F7A5D
:1033700061762E205B7679705D00462E2061757433
:103380006F6C6F6164205B6F66665D00462E206126
:1033900075746F7A61762E205B4E2F415D00462E4C
:1033A000206175746F6C6F6164205B4E2F415D000E
:1033B00046696C2E2073656E7A6F72205B7A61703D
:1033C0005D0046696C2E2073656E736F7220205B02
:1033D0006F6E5D0046696C2E2073656E7A6F722089
:1033E0005B7679705D0046696C2E2073656E736F35
:1033F00072205B6F66665D0046696C2E2073656E99
:103400007A6F72205B4E2F415D0046696C2E2073EF
:10341000656E736F72205B4E2F415D0020467265B2
:1034200065204D656D6F72793A20005469736B6148
:10343000726E61206E6562796C61206A6573746575
:10344000207A6B616C6962726F76616E612E2050BA
:103450006F73747570756A74652070726F73696DBF
:1034600020706F646C65206D616E75616C752C20C9
:103470006B617069746F6C61205A6163696E616D14
:10348000652C206F6473746176656320506F73746C
:103490007570206B616C6962726163652E00507299
:1034A000696E74657220686173206E6F7420626546
:1034B000656E2063616C6962726174656420796510
:1034C000742E20506C6561736520666F6C6C6F772D
:1034D00020746865206D616E75616C2C2063686175
:1034E00070746572204669727374207374657073AA
:1034F0002C2073656374696F6E2043616C6962721E
:103500006174696F6E20666C6F772E0050727574EF
:103510006F6B00466C6F7700446F6B6F6E636F76F6
:10352000616E6920706F687962750046696E6973B3
:1035300068696E67206D6F76656D656E74730020C7
:103540007A203400206F66203400486C6564616D19
:10355000206B616C69627261636E6920626F6420C6
:10356000706F646C6F7A6B79005365617263686920
:103570006E67206265642063616C69627261746960
:103580006F6E20706F696E74004974657261636557
:103590002000497465726174696F6E2000446F6E1B
:1035A0006520736176696E672066696C652E0044DC
:1035B0006F6E65207072696E74696E672066696CE3
:1035C0006500536F75626F72206E656B6F6D706C06
:1035D00065746E692E20506F6B7261636F766174D3
:1035E0003F0046696C6520696E636F6D706C657431
:1035F000652E20436F6E74696E756520616E7977F4
:1036000061793F004E656B7465726520736F7562FA
:103610006F7279206E656275646F75207365747260
:103620006964656E792E204D6178696D616C6E6993
:1036300020706F63657420736F75626F7275207090
:10364000726F20736574726964656E69206A6520A3
:103650003130302E00536F6D652066696C657320C4
:1036600077696C6C206E6F7420626520736F727462
:1036700065642E204D61782E204E6F2E206F6620BF
:1036800066696C657320696E203120666F6C6465B5
:103690007220666F7220736F7274696E672069732F
:1036A000203130302E0053656E7A6F722066696C5F
:1036B000616D656E74750046696C616D656E742030
:1036C00073656E736F720046696C616D656E742010
:1036D0007679746C6163656E2061207370726176B7
:1036E0006E652062617276793F0046696C616D6536
:1036F0006E7420657874727564696E672026207711
:1037000069746820636F727265637420636F6C6F95
:10371000723F0056796D656E69742066696C616DE3
:10372000656E74004368616E67652066696C616DE3
:10373000656E7400527963686C6F73742076656E81
:10374000742E0046616E207370656564004B6F6E69
:1037500074722E2076656E742E5B7A61705D004601
:10376000616E7320636865636B2020205B6F6E5D04
:10377000004B6F6E74722E2076656E742E5B7679B8
:10378000705D0046616E7320636865636B20205B2B
:103790006F66665D00656E717565696E67202200F3
:1037A0004578747275646572002045787465726E30
:1037B000616C205265736574005072696E74657235
:1037C0002073746F707065642064756520746F2059
:1037D0006572726F72732E20466978207468652056
:1037E0006572726F7220616E6420757365204D3949
:1037F000393920746F20726573746172742E2028B9
:1038000054656D706572617475726520697320729C
:10381000657365742E205365742069742061667425
:1038200065722072657374617274696E6729004EE7
:103830006F204C696E65204E756D626572207769E8
:10384000746820636865636B73756D2C204C6173BD
:1038500074204C696E653A20004E6F2043686563A2
:103860006B73756D2077697468206C696E65206E66
:10387000756D6265722C204C617374204C696E65A5
:103880003A200020746F6F206C6F6E67206578742B
:10389000727573696F6E2070726576656E7465649B
:1038A000004C696E65204E756D62657220697320EB
:1038B0006E6F74204C617374204C696E65204E7578
:1038C0006D6265722B312C204C617374204C696ED3
:1038D000653A20005072696E7465722068616C747C
:1038E00065642E206B696C6C28292063616C6C65A3
:1038F00064210020636F6C6420657874727573694D
:103900006F6E2070726576656E74656400636865BD
:10391000636B73756D206D69736D617463682C20C2
:103920004C617374204C696E653A200043485942DB
:10393000413A004552524F523A00456E6420666942
:103940006C65206C697374006F70656E0054524929
:1039500047474552454400656E6473746F70732029
:103960006869743A2000536C6565702E2E2E0056DF
:1039700079706E6F7574206D6F746F727900446921
:103980007361626C65207374657070657273004E4C
:10399000616872616E6F20767963686F7A69206EF4
:1039A0006173746176656E690044656661756C74F7
:1039B0002073657474696E6773206C6F61646564ED
:1039C00000446174756D3A00446174653A00506F4B
:1039D000757A6520616B7475616C6E6900437572F0
:1039E00072656E74001B5B324A504F5A4F523A1B3D
:1039F0005B313B3048437261736820646574656B6A
:103A000063651B5B323B30486465616B7469766F3C
:103A100076616E612076651B5B333B30485374657D
:103A2000616C7468206D6F6475001B5B324A57418E
:103A3000524E494E473A1B5B313B304843726173EB
:103A40006820646574656374696F6E1B5B323B301C
:103A50004864697361626C656420696E1B5B333B0B
:103A60003048537465616C7468206D6F6465001B29
:103A70005B324A437261736820646574656B636589
:103A8000206D757A651B5B313B3048627974207A12
:103A900061706E75746120706F757A6520761B5B3E
:103AA000323B30484E6F726D616C206D6F647500F3
:103AB0001B5B324A4372617368206465746563748A
:103AC000696F6E2063616E1B5B313B30486265201D
:103AD0007475726E6564206F6E206F6E6C792069EC
:103AE0006E1B5B323B30484E6F726D616C206D6FA8
:103AF000646500446574656B6F76616E206E6172FB
:103B0000617A2E0043726173682064657465637422
:103B100065642E004372617368206465742E2020F2
:103B20005B7A61705D004372617368206465742E16
:103B30002020205B6F6E5D004372617368206465B6
:103B4000742E20205B7679705D004372617368206B
:103B50006465742E20205B6F66665D00437261733E
:103B600068206465742E20205B4E2F415D00204349
:103B70006F756E7420583A200056796D656E61201D
:103B80006F6B3F004368616E67656420636F72729C
:103B90006563746C793F005A63686C616469740092
:103BA000436F6F6C646F776E0050726F2075737027
:103BB00065736E6F75206B616C69627261636920F9
:103BC0006F636973746574652070726F73696D20BB
:103BD0007469736B6F766F7520747279736B752E61
:103BE00020506F74767264746520746C61636974BC
:103BF0006B656D2E00506C6561736520636C65614B
:103C00006E20746865206E6F7A7A6C6520666F72BC
:103C10002063616C6962726174696F6E2E20436CFF
:103C200069636B207768656E20646F6E652E002077
:103C30004C61737420557064617465643A20005659
:103C40007962657274652065787472756465723A1C
:103C50000043686F6F736520657874727564657270
:103C60003A0050726F73696D206F74657672657477
:103C7000652069646C65722061206D616E75616C90
:103C80006E65206F64737472616E74652066696C12
:103C9000616D656E742E00506C65617365206F7088
:103CA000656E2069646C657220616E642072656D5A
:103CB0006F76652066696C616D656E74206D616EEE
:103CC00075616C6C792E005A6D656E61207573702C
:103CD00065736E6121004368616E6765207375636B
:103CE0006365737321005469736B207A2053440019
:103CF0005072696E742066726F6D20534400546573
:103D0000706C6F742E206B616C6962726163650008
:103D100054656D702E2063616C6962726174696FA5
:103D20006E004B616C696272756A69205A0043616A
:103D30006C6962726174696E67205A005A6B616CBB
:103D40006962726F7661740043616C69627261745A
:103D5000650052657365742058595A206B616C690F
:103D600062722E0052657365742058595A2063613F
:103D70006C6962722E004B616C69627261636520CE
:103D800058595A0043616C696272617465205859D0
:103D90005A002042726F776E206F757420526573DF
:103DA000657400426567696E2066696C65206C69A0
:103DB0007374004B616C6962726163652058595A73
:103DC000206E65707265736E612E204C6576792069
:103DD000707265646E6920626F64206D6F63207617
:103DE00070726564752E0058595A2063616C69625F
:103DF000726174696F6E20636F6D70726F6D69733D
:103E000065642E204C6566742066726F6E74206344
:103E1000616C6962726174696F6E20706F696E7433
:103E2000206E6F7420726561636861626C652E003C
:103E30004B616C6962726163652058595A206E65E6
:103E4000707265736E612E20507265646E69206BAE
:103E5000616C69627261636E6920626F6479206D62
:103E60006F63207670726564752E0058595A20630E
:103E7000616C6962726174696F6E20636F6D7072DC
:103E80006F6D697365642E2046726F6E7420636176
:103E90006C6962726174696F6E20706F696E7473A1
:103EA000206E6F7420726561636861626C652E00BC
:103EB0004B616C6962726163652058595A207620A3
:103EC000706F7261646B752E20582F59206F737953
:103ED000206D69726E65207A6B6F73656E652E203A
:103EE000446F627261207072616365210058595A93
:103EF0002063616C6962726174696F6E20616C6CC1
:103F00002072696768742E20582F59206178657374
:103F10002061726520736C696768746C7920736BBB
:103F2000657765642E20476F6F64206A6F62210099
:103F30004B616C6962726163652058595A20762022
:103F4000706F7261646B752E205A6B6F73656E694A
:103F50002062756465206175746F6D617469636B4F
:103F600079207679726F766E616E6F20707269203B
:103F70007469736B752E0058595A2063616C6962BD
:103F8000726174696F6E20616C6C2072696768740D
:103F90002E20536B65772077696C6C2062652063F7
:103FA0006F72726563746564206175746F6D61749E
:103FB0006963616C6C792E004B616C69627261633C
:103FC000652058595A2073656C68616C612E204BCE
:103FD000616C69627261636E6920626F6420706FE8
:103FE000646C6F7A6B79206E656E616C657A656E54
:103FF0002E0058595A2063616C6962726174696F4E
:104000006E206661696C65642E2042656420636180
:104010006C6962726174696F6E20706F696E742072
:10402000776173206E6F7420666F756E642E004B1F
:10403000616C6962726163652058595A20762070FC
:104040006F7261646B752E20582F59206F73792021
:104050006A736F75206B6F6C6D652E20477261748B
:10406000756C756A69210058595A2063616C6962E0
:10407000726174696F6E206F6B2E20582F5920610A
:10408000786573206172652070657270656E646911
:1040900063756C61722E20436F6E67726174756C0C
:1040A0006174696F6E7321004B616C696272616348
:1040B000652058595A2073656C68616C612E204EDA
:1040C00061686C65646E65746520646F206D616EF7
:1040D00075616C752E0058595A2063616C69627263
:1040E0006174696F6E206661696C65642E20506C26
:1040F0006561736520636F6E73756C742074686599
:10410000206D616E75616C2E004B616C696272612D
:1041100063652058595A2073656C68616C612E2064
:104120004C65767920707265646E6920626F6420D8
:104130006D6F63207670726564752E2053726F7692
:104140006E656A7465207469736B61726E752E009A
:1041500058595A2063616C6962726174696F6E208C
:104160006661696C65642E204C6566742066726FAA
:104170006E742063616C6962726174696F6E207025
:104180006F696E74206E6F7420726561636861621E
:104190006C652E004B616C696272616365205859D1
:1041A0005A2073656C68616C612E20507265646E74
:1041B00069206B616C69627261636E6920626F6411
:1041C00079206D6F63207670726564752E2053724E
:1041D0006F766E656A7465207469736B61726E7553
:1041E0002E0058595A2063616C6962726174696F5C
:1041F0006E206661696C65642E2046726F6E742055
:1042000063616C6962726174696F6E20706F696E50
:104210007473206E6F7420726561636861626C658F
:104220002E004B616C696272616365205A20736570
:104230006C68616C612E2053656E736F72206A65C5
:10424000206F64706F6A656E79206E65626F207092
:104250007265727573656E79206B6162656C2E2074
:1042600043656B616D206E612072657365742E000D
:10427000426564206C6576656C696E67206661696D
:104280006C65642E2053656E736F7220646973636E
:104290006F6E6E6563746564206F72206361626C1B
:1042A000652062726F6B656E2E2057616974696E4E
:1042B0006720666F722072657365742E004B616CA7
:1042C000696272616365205A2073656C68616C6114
:1042D0002E2053656E736F72206E657365706E75F8
:1042E0006C2E205A6E6563697374656E61207472FA
:1042F00079736B613F2043656B616D206E61207245
:10430000657365742E00426564206C6576656C6922
:104310006E67206661696C65642E2053656E736FED
:1043200072206469646E7420747269676765722EA6
:1043300020446562726973206F6E206E6F7A7A6CAA
:10434000653F2057616974696E6720666F722072DD
:10435000657365742E004B616C69627261636520E0
:104360005A2073656C68616C612E2053656E736FA3
:1043700072207365706E756C207072696C69732041
:104380007679736F6B6F2E2043656B616D206E6164
:104390002072657365742E00426564206C657665D5
:1043A0006C696E67206661696C65642E2053656E6A
:1043B000736F722074726967676572656420746FC9
:1043C0006F20686967682E2057616974696E67207D
:1043D000666F722072657365742E005A6168726927
:1043E00076616E692062656400426564204865619B
:1043F00074696E6700426564204F4B2E004265640D
:1044000020646F6E650056707261766F205B756D0B
:104410005D00526967687420736964655B756D5DE2
:1044200000526573657400567A61647520205B756F
:104430006D5D00526561722073696465205B756D06
:104440005D004B6F72656B636520706F646C6F7A93
:104450006B7900426564206C6576656C20636F72D1
:104460007265637400566C65766F20205B756D5DB8
:10447000004C6566742073696465205B756D5D0032
:10448000567072656475205B756D5D0046726F6E67
:104490007420736964655B756D5D00426564004EF0
:1044A000656E69207A6B616C6962726F76616E61AC
:1044B00020767A64616C656E6F73742074727973A0
:1044C0006B79206F64207469736B6F766520706FF1
:1044D000646C6F7A6B792E20506F73747570756A87
:1044E00074652070726F73696D20706F646C6520E5
:1044F0006D616E75616C752C206B617069746F6C89
:1045000061205A6163696E616D652C206F647374FC
:1045100061766563204E6173746176656E692070A3
:1045200072766E69207672737476792E00446973A0
:1045300074616E6365206265747765656E20746969
:1045400070206F6620746865206E6F7A7A6C6520C3
:10455000616E64207468652062656420737572669C
:1045600061636520686173206E6F74206265656E9B
:1045700020736574207965742E20506C65617365B5
:1045800020666F6C6C6F7720746865206D616E7546
:10459000616C2C2063686170746572204669727367
:1045A000742073746570732C2073656374696F6E07
:1045B000204669727374206C617965722063616C46
:1045C0006962726174696F6E2E00446F6C6164651C
:1045D0006E69206F7379205A004C6976652061649A
:1045E0006A757374205A0041646A757374696E67E2
:1045F000205A004175746F20686F6D6500417574B5
:104600006F5A61766564656E692066696C2E00413B
:1046100075746F4C6F61642066696C616D656E7452
:10462000004175746F6D617469636B65207A6176A2
:104630006164656E692066696C616D656E74752074
:10464000646F737475706E6520706F757A65207015
:104650007269207A61706E7574656D2066696C612F
:104660006D656E742073656E7A6F72752E2E2E00D6
:104670004175746F6C6F6164696E672066696C6107
:104680006D656E7420617661696C61626C65206F26
:104690006E6C79207768656E2066696C616D656EF9
:1046A000742073656E736F72206973207475726EF7
:1046B0006564206F6E2E2E2E004175746F6D6174CF
:1046C00069636B65207A61766164656E69206669ED
:1046D0006C616D656E747520616B7469766E692CA2
:1046E00020737469736B6E65746520746C616369A3
:1046F000746B6F206120766C6F7A74652066696CCC
:10470000616D656E742E2E2E004175746F6C6F6135
:1047100064696E672066696C616D656E742069738B
:10472000206163746976652C206A757374207072D9
:1047300065737320746865206B6E6F6220616E64B0
:1047400020696E736572742066696C616D656E7444
:104750002E2E2E00207C20417574686F723A200046
:1047600056736500416C6C00416374697665204541
:10477000787472756465723A20000B12FB111F1277
:1047800027122F12381240125D124812761272123E
:104790007A1282129B128A12C612AC121C13E412F5
:1047A0007A135A13FE139D130C1561140316C015CA
:1047B000A91650165C17F0160718BB179B18581847
:1047C000EC18D8185A190019F119A2195F1A3B1AD6
:1047D000941A7F1AB71AA81A021BD41A8D1B301B01
:1047E000ED1BF41B0E1C041C421C1A1C771C651CC0
:1047F000881CAD1C991CE01CBF1C111D001D331D25
:10480000211D461D5F1D591D641D761D881DE11D5E
:10481000CF1D051EF31D521E171E9F1E8A1EBC1E95
:10482000B41ED01EC81EE61ED81EF11EFB1E2B1F76
:104830000F1F541F461F791F671F981F8A1FB31F22
:10484000A61FD11FC41F0720DE1F3B20322053208C
:104850004120772065209B208920BD20AD20CB20E2
:10486000EA20DB200921F7202D211B2150213F21A7
:104870006E215F218D217B21A8219E21C021B121A4
:10488000D721CD21DF210022F1211A220B2229225A
:1048900045223622532259227D226B2296228E22D5
:1048A000A9229F22C822B622E922D8220423F2227A
:1048B000222316234523302356236723772380237F
:1048C0009D238823C023AE23E423D2230824F62388
:1048D0002C241A244F243E247324612497248524F5
:1048E000BB24A924CD24E424DA24F424F024F924DC
:1048F0001D250B2541252F255325652578258E253A
:1049000080259B25AD25C125DF25D125ED25FA255F
:10491000082616262C26372654264D266C265B267E
:104920008A267B26A4269926B126E326BA26322794
:104930000B2769275427A0277E27D627C527F927C5
:10494000E82716280B28322822284D283F285B28E4
:10495000A1287028FF28CA283F292A296629522918
:1049600084297A298C29A3299429D529AF290E2AAB
:10497000F529262A652A3D2A9A2A8A2ABC2AA82AA3
:10498000E22AD02A022BF42A222B122BB52B2E2B13
:104990004B2C4E2C522C6A2C5B2C7C2C752C962C80
:1049A000832CBB2CAA2CD02CCD2CE82CD32C132D53
:1049B000F82C3E2D332D502D452D622D572D692D70
:1049C0007F2D722D892DA22D9B2DB32DAB2DCA2DA0
:1049D000C02DE22DD62DF32DEE2D222EF92D622E97
:1049E000522E802E712E852E9C2EB32ECA2EFA2E7C
:1049F000E32E102FED2F04301B3045303230623063
:104A0000523083307030A2309430B630B030C9307C
:104A1000BC30E130D930E930F230133103312F317D
:104A2000233148313B3154316731623191316D313D
:104A3000BD31B131D831CB31F631E93110320232EA
:104A400028321E327F3230320133C832563344337B
:104A50007A3368339E338C33C233B033E633D43386
:104A60000A34F8331C349E342B3413350C352B3573
:104A7000183544353F3569354A35923589359D3588
:104A8000AF35E235C23555360436B736A636EA3686
:104A9000C73624371337433734375F374D378337BB
:104AA00071379537A037A937B9372F385938833838
:104AB000A138D438F3380D3933392C393A394839DB
:104AC0004D39573966397E396F39A9398F39C83927
:104AD000C139DD39CE392A3AE539B03A6F3A043B6B
:104AE000F33A263B143B4A3B383B5C3B6E3B843BF2
:104AF000793BA03B973BF53BA93B2F3C513C3F3CCE
:104B0000973C623CD63CC73CF03CE63C103DFE3C4A
:104B10002E3D223D483D3C3D643D523D843D763D29
:104B2000923DA33DE73DB33D6B3E303EED3EB03E92
:104B3000773F303FF23FB83F67402F40D640A84014
:104B400050410941E2419441704222420643BD4234
:104B500098435643E943DB43FD43F543124406447F
:104B600021443344274453444244714465448C44B3
:104B700080449B442D459F44D945CA45E745F345AC
:104B80000F46FD45704621460947B94654476447DC
:104B900060476847457872656D65207370616E2067
:104BA0006F6620746865205A2076616C7565732184
:104BB0000043616C63756C6174696F6E206F662071
:104BC000746865206D616368696E6520736B6577D5
:104BD00020616E64206F6666736574206661696C1F
:104BE00065642E00203C20005741524E494E473A02
:104BF0002046726F6E7420706F696E74206E6F74D1
:104C000020726561636861626C652E205920636F54
:104C10006F7264696E6174653A000049746572610F
:104C200074696F6E3A200000004041FFFFBF4000F2
:104C3000005C43FFFFBF4000005C430000464300B0
:104C40000040410000464300004041FFFFBF4000DC
:104C500000E442FFFFBF4000005743FFFFBF40009A
:104C60000057430000CC420000E4420000CC420068
:104C70000040410000CC420000404100004643009B
:104C800000E442000046430000574300004643064C
:104C90002833D036C23E013F154132423B43F244F5
:104CA0003B45F24622473B48F2493B4AF058985967
:104CB0000C5A085B0C5C086110679B6E22710772CE
:104CC00008FF095A0D000EFF19045E0820642B6DC1
:104CD000322FFF5A00205A3A00590020593A005802
:104CE0000020583A0024F4D43050C38E20C2A24091
:104CF00017828B7011127A910D816CD90AA861E12B
:104D000008C7586607615143061E4B5D05C145A79C
:104D1000041A411104093D9803713931034036DB0F
:104D20000265339102D4305402802E1D02632CEEB2
:104D300001752AC501B028A001102781018F2564C3
:104D4000012B244B01E0223401AC211F018D200DE9
:104D500001801FFC00841EED00971DDF00B81CD2EF
:104D600000E61BC600201BBC00641AB200B219A8E2
:104D7000000A19A0006A189900D117910040178BFA
:104D800000B516840031167E00B31579003A15730C
:104D900000C7146F0058146A00EE1366008813638E
:104DA0000025135E00C7125B006C125700151254E9
:104DB00000C111510070114F0021114B00D6104954
:104DC000008D1047004610440002104200C00F4002
:104DD00000800F3E00420F3C00060F3B00CB0E3818
:104DE00000930E37005C0E3500270E3400F30D32B1
:104DF00000C10D3100900D3000600D2E00320D2DE0
:104E000000050D2C00D90C2B00AE0C2900850C29B7
:104E1000005C0C2700350C27000E0C2600E80B2444
:104E200000C40B2400A00B23007D0B23005A0B2190
:104E300000390B2100180B2000F80A1F00D90A1EA8
:104E400000BB0A1E009D0A1D00800A1D00630A1C8B
:104E500000470A1B002C0A1B00110A1A00F7091A46
:104E600000DD091900C4091900AB091900920917DE
:104E7000007B091800630917004C09160036091653
:104E800000200916000A091500F5081500E00814AD
:104E900000CC081400B8081400A4081400900813EB
:104EA000007D0812006B0813005808120046081213
:104EB0000034081100230811001208110001081124
:104EC00000F0071000E0071000D0071000C0071026
:104ED00000B0070F00A107100091070E0083070F15
:104EE0000074070F0065070E0057070E0049070EF4
:104EF000003B070D002E070E0020070D0013070DC5
:104F00000006070D00F9060C00ED060D00E0060C8A
:104F100000D4060C00C8060C00BC060C00B0060C41
:104F200000A4060B0099060C008D060B0082060BF0
:104F30000077060B006C060B0061060A0057060B93
:104F4000004C060A0042060A0038060A002E060A2D
:104F50000024060A001A060A001006090007060ABD
:104F600000FD050900F4050900EB050900E205094B
:104F700000D9050900D0050900C7050900BE0509CB
:104F800000B5050800AD050800A50509009C050849
:104F900000940508008C050800840508007C0508BD
:104FA00000740508006C050700650508005D05072D
:104FB00000560508004E0507004705070040050894
:104FC0000038050700310507002A050700230507FB
:104FD000001C050600160507000F0507000805065A
:104FE0000002050700FB040600F5040700EE0406B6
:104FF00000E8040600E2040700DB040600D504060E
:1050000000CF040600C9040600C3040600BD040660
:1050100000B7040600B1040500AC040600A60406AF
:1050200000A00405009B04060095040500900406FA
:10503000008A04050085040500800406007A040542
:105040000075040500700405006B04050066040586
:1050500000610405005C04050057040500520405C6
:10506000004D04050048040500430405003E040407
:10507000003A04050035040500300404002C040542
:105080000027040400230405001E0404001A04047D
:105090000016040500110404000D040400090405B1
:1050A000000404040000040400FC030400F80304EA
:1050B00000F4030400F0030400EC030400E803041C
:1050C00000E4030400E0030400DC030400D803044C
:1050D00000D4030400D0030400CC030400C803037D
:1050E00000C503030024F404D9201BC40C5C0E98F3
:1050F00004C4095F0265077101F405F900FB04B3FC
:105100000048048700C103690058035500030345A4
:1051100000BE023A008402310053022A002902250F
:105120000004022000E4011C00C8011900AF0117AF
:105130000098011400840113007101100061011036
:105140000051010E0043010D0036010B002B010B35
:105150000020010B00150109000C010900030108E2
:1051600000FB000800F3000800EB000700E4000665
:1051700000DE000600D8000600D2000600CC0005C4
:1051800000C7000500C2000500BD000400B900040E
:1051900000B5000400B1000400AD000400A9000443
:1051A00000A5000300A20003009F0004009B000371
:1051B0000098000300950002009300030090000394
:1051C000008D0002008B00030088000200860002B0
:1051D0000084000300810002007F0002007D0002C5
:1051E000007B0002007900020077000100760002D7
:1051F000007400020072000100710002006F0002E2
:10520000006D0001006C0002006A000100690002EC
:1052100000670001006600010065000100640002F3
:10522000006200010061000100600001005F0002F7
:10523000005D0001005C0001005B0001005A0001FC
:1052400000590001005800010057000100560001FC
:1052500000550001005400010053000000530001FC
:10526000005200010051000100500001004F0001F8
:10527000004E0000004E0001004D0001004C0001F6
:10528000004B0000004B0001004A000100490001F2
:1052900000480000004800010047000100460000EF
:1052A00000460001004500000045000100440001E7
:1052B00000430000004300010042000000420001E2
:1052C000004100000041000100400001003F0000DB
:1052D000003F0001003E0000003E0001003D0000D4
:1052E000003D0001003C0000003C0000003C0001CB
:1052F000003B0000003B0001003A0000003A0001C2
:1053000000390000003900010038000000380000BA
:1053100000380001003700000037000100360000AF
:1053200000360000003600010035000000350000A6
:10533000003500010034000000340000003400019A
:105340000033000000330000003300010032000091
:105350000032000000320001003100000031000086
:10536000003100010030000000300000003000017A
:10537000002F0000002F0000002F0000002F000170
:10538000002E0000002E0000002E0001002D000065
:10539000002D0000002D0000002D0001002C000059
:1053A000002C0000002C0000002C0001002B00004D
:1053B000002B0000002B0000002B0001002A000041
:1053C000002A0000002A0000002A00010029000035
:1053D0000029000000290000002900000029000128
:1053E000002800000028000000280000002800001D
:1053F000002800010027000000270000002700000F
:105400000027000000270001002600000026000001
:1054100000260000002600000026000100250000F4
:1054200000250000002500000025000000250000E8
:1054300000250001002400000024000000240000DA
:1054400000240000002400010023000000230000CD
:1054500000230000002300000023000000230000C0
:1054600000230001002200000022000000220000B2
:1054700000220000002200000022000100210000A4
:105480000021000000210000002100000021000098
:105490000021000000210001002000000020000089
:1054A000002000000020000000200000002000007C
:1054B0000020000000200001001F0000001F00006D
:1054C000001F0000001F0000001F0000001F000060
:1054D000001F0001001E0000001E0000001E000052
:1054E000001E0000004572723A204D494E54454D51
:1054F00050204245440054656D7065726174757248
:1055000065206865617465642062656420737769ED
:105510007463686564206F66662E204D494E54455D
:105520004D5020747269676765726564202100457B
:1055300072723A204D415854454D50204245440026
:1055400054656D706572617475726520686561740B
:10555000656420626564207377697463686564209C
:105560006F66662E204D415854454D502074726927
:105570006767657265642021004572723A204D4963
:105580004E54454D50003A204578747275646572EA
:10559000207377697463686564206F66662E204D9A
:1055A000494E54454D502074726967676572656451
:1055B0002021004572723A204D415854454D50000B
:1055C0003A204578747275646572207377697463E4
:1055D000686564206F66662E204D415854454D50D5
:1055E0002074726967676572656420210020484FE6
:1055F00054454E4420544845524D414C2052554E3E
:10560000415741590020484541544245442054489F
:1056100045524D414C2052554E4157415900544836
:1056200045524D414C2052554E415741590042453B
:105630004420544845524D414C2052554E4157410B
:10564000590020544845524D414C2052554E415727
:1056500041592028205052454845415420484F5434
:10566000454E44290020544845524D414C20525546
:105670004E41574159202820505245484541542019
:1056800048454154424544290050524548454154FB
:10569000204552524F520042454420505245484501
:1056A0004154204552524F52004572723A20505296
:1056B000494E542046414E204552524F520050729E
:1056C000696E742066616E2073706565642069730D
:1056D000206C6F776572207468656E2065787065E0
:1056E00063746564004572723A20455854522E2006
:1056F00046414E204552524F5200457874727564AF
:1057000065722066616E2073706565642069732020
:105710006C6F776572207468656E2065787065635C
:10572000746564002F2F20616374696F6E3A706135
:1057300075736500504944204175746F74756E65CA
:105740002066696E697368656421205075742074E1
:105750006865206C617374204B702C204B6920614C
:105760006E64204B6420636F6E7374616E7473207B
:1057700066726F6D2061626F766520696E746F204E
:10578000436F6E66696775726174696F6E2E68002B
:10579000504944204175746F74756E652066616967
:1057A0006C6564212074696D656F75740020403AE2
:1057B00000543A00423A00504944204175746F74D5
:1057C000756E65206661696C6564212054656D7035
:1057D0006572617475726520746F6F20686967689F
:1057E00000204B643A2000204B693A2000204B7087
:1057F0003A200020436C6173736963205049442050
:10580000002054753A2000204B753A2000206D612D
:10581000783A2000206D696E3A200020643A20001A
:1058200020626961733A200090137D00B015780002
:10583000F0177300601A6E00F01C6900A01F64006E
:1058400050225F0020255A00E0275500902A500082
:10585000202D4B00A02F4600F031410010343C00B9
:10586000F0353700A037320020392D00603A28008B
:10587000703B2300603C1E00203D1900C03D140019
:10588000403E0F00A03E0A00F03E0500403F0000F1
:10589000703FFBFF903FF6FFB03FF1FFC03FECFFD2
:1058A000D03FE7FFE03FE2FFF03FDDFFF03FD8FFF2
:1058B0001000C90210012C014001220170011801E1
:1058C000B0010E01F00104015002FA00B002F00034
:1058D0003003E600D003DC009004D2007005C8005D
:1058E000A006BE000008B400B009AA00D00BA000BA
:1058F000600E960060118C0000158200201978005F
:10590000C01D6E00A0226400B0275A00902C5000E9
:1059100000314600E0343C0010383200903A280054
:10592000603C1E00A03D1400803E0A00203F0000A5
:1059300070012C0190012701B0012201C0011D015D
:10594000F00118011002130130020E01600209017A
:1059500090020401C002FF000003FA004003F500BA
:105960008003F000D003EB002004E6007004E100A7
:10597000E004DC004005D700C005D2004006CD00A1
:10598000D006C8008007C3003008BE00F008B90088
:10599000C009B400B00AAF00B00BAA00D00CA5003B
:1059A000000EA000500F9B00C010960050129100F6
:1059B00000148C00C0158700B0178200B0197D005C
:1059C000D01B7800001E730040206E0090226900FA
:1059D000F024640040275F0090295A00E02B550016
:1059E000102E500020304B0010324600E0334100B2
:1059F00090353C001037370070383200A0392D0048
:105A0000B03A2800A03B2300603C1E00103D190066
:105A1000903D1400103E0F00703E0A00C03E05008D
:105A2000003F0000746D63323133305F7072696E15
:105A3000745F63757272656E747328290A09480968
:105A4000520A580925640925640A5909256409255B
:105A5000640A5A0925640925640A4509256409254B
:105A6000640A00746D63323133305F7365745F6351
:105A7000757272656E745F7228617869733D256412
:105A80002C2063757272656E743D25640A00746D16
:105A900063323133305F7365745F63757272656E44
:105AA000745F6828617869733D25642C2063757282
:105AB00072656E743D25640A00544D43204452497A
:105AC000564552204F56455254454D502000746D56
:105AD00063323133305F696E697428292C206D6F11
:105AE00064653D25530A004E4F524D414C005354BE
:105AF00045414C544800436F6E74696E756520775C
:105B000069746820616E6F7468657220626F776473
:105B1000656E3F0053746174653A20004737360064
:105B20004D3435205A004D343500473830002000C0
:105B30003E003E0020003E003E003E003E002000B1
:105B40003E003E00200000002D2D2D2D2D2D2D2D51
:105B50002D2D2D2D2D2D2D2D2D2D2D2D004E2F416B
:105B6000004E2F41006D6D00004D373031004D3734
:105B7000303200496E76616C69642050494420637C
:105B8000616C2E20726573756C74732E204E6F7469
:105B90002073746F72656420746F20454550524FB6
:105BA0004D2E004D353030004731205A31352046DA
:105BB00031353030004739310047312058353020F9
:105BC00059313930204530204637303030004739A0
:105BD00030004D373032004D3730322043004D37E2
:105BE00030322055004D373032004731205A3135A0
:105BF00020463135303000473931004731205835A3
:105C0000302059313930204530204637303030008F
:105C10004D383300473930004D3834004D31303481
:105C2000205330004D38340047312058313020594E
:105C3000313830204634303030004731205A31304E
:105C40002046313330302E303030004D313430206A
:105C50005330004D313034205330004D3130370057
:105C6000473120452D302E30373530302046323107
:105C700030302E3030303030004731205835302031
:105C80005935352045332E363237373300473120EA
:105C900058323030205935352045302E343933389C
:105CA00036004731205832303020593735204533BF
:105CB0002E363237373300473120583530205937A8
:105CC000352045302E3439333836004731205835A9
:105CD00030205939352045332E3632373733004797
:105CE000312058323030205939352045302E343962
:105CF0003338360047312058323030205931313571
:105D00002045332E3632373733004731205835306F
:105D100020593131352045302E343933383600475B
:105D2000312058353020593133352045332E363225
:105D3000373733004731205832303020593133352E
:105D40002045302E36363137340047312058323036
:105D50003020593135352045322E36323737330031
:105D60004731205831303020593135352045320007
:105D700047312058373520593135352045322E35B9
:105D80000047312046313038300047312058353017
:105D90002059313535004731204634303030004D00
:105DA000323034205331303030004731205A302ED9
:105DB0003135302046373230302E303030004731E8
:105DC00020452D312E3530303030204632313030C4
:105DD0002E3030303030004D3833004739300047F6
:105DE0003231004739322045302E300047312058BB
:105DF0003130302E30204531322E35204631303092
:105E0000302E30004731205836302E302045392E84
:105E1000302046313030302E300047393220453086
:105E20002E300047323800473837004D31303920A6
:105E300053323135004D31393020533630004D3139
:105E4000343020533630004D313034205332313528
:105E5000004D31303700473930004731204531009F
:105E60004D3832004731204531004D3833004D3137
:105E7000303620532564004D3232302053256400E3
:105E80003A20002020202020202020202020202018
:105E900020202020202000203A2000202020202028
:105EA0002020202020202020202020202020200012
:105EB00020202020202020202020202020002573AA
:105EC000002020002D2D3A2D2D0020002000200044
:105ED0004C002020002046002D2D2D003E55534221
:105EE000005344002D2D00252020202020002020BC
:105EF000002020000120002020202D2D2D2000201A
:105F0000205A002020000120004D36303000464C41
:105F10004558202D20203234302F3530005050206D
:105F200020202D20203235342F3130300048495088
:105F300053202D20203232302F3130300041425357
:105F400020202D20203235352F313030005045545F
:105F500020202D20203233302F383500504C412066
:105F6000202D20203231352F3630006661726D20B1
:105F7000202D20203235302F3430004D3234004D6A
:105F8000323320257300052E2E00580059005A0088
:105F900045787472756465720047393900446973D5
:105FA00061626C65206661726D206D6F64653F0093
:105FB00044697361626C65206661726D206D6F6407
:105FC00065004661726D206E756D626572004D38B8
:105FD000340041786973206C656E67746820646969
:105FE00066666572656E63653A004D6561737572CC
:105FF00065642061786973206C656E6774683A0027
:1060000025632041584953205347313D25640A00F8
:106010004D3834004731205A313500473238205747
:10602000005A30005A3100593000593100583000C0
:10603000583100456E642073746F70732064696119
:1060400067004D3434004732382057001B5B303B2B
:1060500030484C617374207072696E742066616997
:106060006C757265731B5B313B3148506F7765729D
:10607000206661696C757265732020252D33641B61
:106080005B323B314846696C616D2E2072756E6FD4
:106090007574732020252D33641B5B333B314843DB
:1060A0007261736820205820252D336420205920E8
:1060B000252D3364001B5B303B3048546F74616C9A
:1060C000206661696C757265731B5B313B314850AA
:1060D0006F776572206661696C7572657320202523
:1060E0002D33641B5B323B314846696C616D2E2059
:1060F00072756E6F7574732020252D33641B5B33AE
:106100003B3148437261736820205820252D336449
:1061100020205920252D336400546F74616C004C8D
:10612000617374207072696E74001B5B303B314880
:1061300042656C74207374617475731B5B313B3200
:1061400048582025641B5B323B32485920256400A7
:106150001B5B323B3148416D6269656E743A2020A9
:10616000256425631B5B333B314850494E44413A1B
:106170002020202025642563001B5B303B31484EE6
:106180006F7A7A6C653A202020256425631B5B3189
:106190003B31484265643A20202020202025642598
:1061A00063001B5B313B31485057523A202020207E
:1061B000202025642E2530316456002D2D2D2D2DC7
:1061C0002D2D2D2D2D2D2D00466C6173684169728A
:1061D00020495020416464723A002D2D2D2D2D2D23
:1061E0002D2D2D2D2D2D00466562202031203230A1
:1061F0003138002D2D2D2D2D2D2D2D2D2D2D2D001A
:10620000453344763666756C6C0045494E53795F6C
:1062100031306100315F37356D6D5F4D4B33002D8F
:106220002D2D2D2D2D2D2D2D2D2D2D002072657018
:106230006F20507275736133442F4D4B3300203300
:106240002E312E312D5243352D31353100466972B4
:106250006D776172653A0025642E25642E25642EC3
:106260002564004661696C20737461747300466133
:10627000726D206E756D62657200007263006265FA
:10628000746100616C7068610064657600505255FD
:1062900053413344465700332E312E312D5243356E
:1062A0000000000A0B02090C0D0E08070304010090
:1062B00000000000000000000000000000000000DE
:1062C000000000000000000000000000001211109B
:1062D00000000000000000000000000000000000BE
:1062E00000000000000000000000000000000000AE
:1062F000000000000000000102102020080810200B
:106300004010204080020102010804020101020441
:106310000810204080804020100804020180040200
:106320000180402010080402010804020101020457
:10633000081020408001020408102040801008044A
:10634000088010204004408010204004800505058E
:1063500005070508080808020202020A0A080804DC
:10636000040404010101010101010103030303030A
:10637000030303040707070C0C0C0C0C0C0C0C0299
:1063800002020206060606060606060B0B0B0B0BA0
:106390000B0B0B07070A0A0A0A0A0A05050504047B
:1063A000040808000020002300260029002C002FEC
:1063B0000032000001000003010601090100002273
:1063C00000250028002B002E0031003400020100BF
:1063D00000050108010B0100002100240027002A0C
:1063E000002D003000330001010000040107010A04
:1063F00001024E414E494E495459494E46CDCCCCEE
:106400003D0AD7233C17B7D13877CC2B329595E688
:10641000241FB14F0A000020410000C84200401C68
:106420004620BCBE4CCA1B0E5AAEC59D7400407AB5
:1064300010F35A00A0724E18090010A5D4E800000D
:10644000E87648170000E40B54020000CA9A3B00AB
:106450000000E1F505000080969800000040420F22
:10646000000000A08601000000102700000000E8E6
:1064700003000000006400000000000A00000000AB
:10648000000100000000002C76D888DC674F08234C
:10649000DFC1DFAE59E1B1B796E5E3E453C63AE6B2
:1064A00051997696E8E6C28426EB898C9B62ED4092
:1064B0007C6FFCEFBC9C9F40F2BAA56FA5F49005E1
:1064C0005A2AF75C936B6CF9676DC11BFCE0E40D15
:1064D00047FEF520E6B500D0ED902E030094357709
:1064E000050080841E080000204E0A000000C80C31
:1064F000333333330F986E12831141EF8D2114899A
:106500003BE65516CFFEE6DB18D1844B381BF77CF3
:106510001D901DA4BBE424203284725E228100C938
:10652000F124ECA1E53D2700D4A2C5CA63FCB80163
:1065300005A311241FBECFEFD1E2DEBFCDBF00E027
:106540000CBF17E0A0E0B2E0E8EEFCE903E00BBF0F
:1065500002C007900D92A43DB107D9F72AE1A4ED3E
:10656000B7E001C01D92A834B207E1F715E6C0E319
:10657000D5E600E006C022970109FE010BBF0F948B
:1065800028C4C832D10780E00807A9F70F9400BEDD
:106590000D9462CE0C94000010923B1A10922A1AAD
:1065A00040912B1A50912C1AEDE2FAE180E090E034
:1065B00061E070E09B01082E02C0220F331F0A9495
:1065C000E2F724233523232B11F411821082019644
:1065D00032968730910571F7089587E793E00F941D
:1065E0006DC810922C1A10922B1AEAE7F0E0808105
:1065F00087608083ACE7B0E08C9180648C9380816D
:10660000806880838FE580937E0082E080937D00A8
:10661000C3CF282F2F7090917B0083FF02C098601A
:1066200001C0977F90937B0090917C00822F8770B0
:10663000987F892B80937C000895982F21E030E08B
:1066400080E0A9014F755270452B29F04FEF490F9B
:10665000911102C00895492F220F331F8F5F80319F
:1066600011F0942FEECF0895CF93C0913B1AC7FF3E
:1066700036C0CF70EC2FF0E021E030E00C2E02C0ED
:10668000220F331F0A94E2F740912B1A50912C1AD3
:1066900024233523232B71F4409178005091790005
:1066A000EE0FFF1FE35DF54E20813181240F351F72
:1066B00031832083C73010F4CF5F0BC080912A1A3A
:1066C0008F5F80932A1A803118F00F94663264DF4E
:1066D000C0E08C2FB2DF9DDFC0933B1A0AC08091CF
:1066E0007A00806480937A0080913B1A806880935E
:1066F0003B1ACF91089590915908911107C090913C
:10670000C00095FFFCCF8093C6000895913031F40E
:106710009091C80095FFFCCF8093CE000895CF9252
:10672000DF92EF92FF920F931F93CF93DF938C0131
:10673000D42EC62FD72FD60EDC1671F1F801E080CB
:10674000F180C990C7010F9423CBC816F1F06C2DCE
:10675000C7010F9453CBC7010F9423CB8C15A9F01D
:10676000E7E4F7E08491EF01882329F0C4DF219664
:10677000FE018491F9CF8AE0DF91CF911F910F91B3
:10678000FF90EF90DF90CF90B6CFF801808191819C
:10679000019691838083D0CFDF91CF911F910F918C
:1067A000FF90EF90DF90CF900895EF92FF920F93BC
:1067B0001F93CF93DF931F92CDB7DEB78C017B0180
:1067C000460FF8018081918149830F9423CBF70113
:1067D00081937F01F801808191810196918380836B
:1067E00049814E11EECF0F90DF91CF911F910F9104
:1067F000FF90EF9008950F931F93CF93DF93CDB742
:10680000DEB72C970FB6F894DEBF0FBECDBF8C015C
:1068100040E350E360E370E04D835E836F837887ED
:106820009C878B8744E0BE016B5F7F4FCE010B9648
:1068300076DF40E16AEA77E1CE010B9670DF40E156
:106840006AEB77E1CE010B966ADF40E16AE977E116
:10685000CE010B9664DF44E062E977E1CE010B964E
:106860005EDF44E06EE877E1CE010B9658DF44E04E
:1068700066E977E1CE010B9652DF44E06AE777E103
:10688000CE010B964CDF44E06AEC77E1CE010B962B
:1068900046DF44E06EE777E1CE010B9640DF44E04F
:1068A00062E877E1CE010B963ADF44E066E877E1F3
:1068B000CE010B9634DF44E06AE877E1CE010B9617
:1068C0002EDF4CE06AE279E0CE010B9628DF44E04F
:1068D00063E279E0CE010B9622DF44E06AEA72E0DF
:1068E000CE010B961CDF44E066EA72E0CE010B9607
:1068F00016DF44E062EA72E0CE010B9610DF44E05E
:106900006AE972E0CE010B960ADF44E066E972E0C4
:10691000CE010B9604DF44E062E972E0CE010B96F3
:10692000FEDE80E290E09A87898742E0BE01675FE1
:106930007F4FCE010B96F3DE41E06FE179E0CE01AF
:106940000B96EDDE44E066E272E0CE010B96E7DEE8
:1069500044E06EE172E0CE010B96E1DE44E06AE1D4
:1069600079E0CE010B96DBDE44E066E179E0CE0112
:106970000B96D5DE44E06AE172E0CE010B96CFDEE5
:1069800041E066E479E0CE010B96C9DE44E066E4BE
:1069900072E0CE010B96C3DE46E552E360E070E0A4
:1069A00049835A836B837C831C870B8744E0BE0139
:1069B0006F5F7F4FCE010B96B2DEE4E5FEE084917F
:1069C0008F01882331F097DE0F5F1F4FF80184910C
:1069D000F8CFE7E3F7E084918F01882331F08BDE75
:1069E0000F5F1F4FF8018491F8CF8AE084DE2C9668
:1069F0000FB6F894DEBF0FBECDBFDF91CF911F91D0
:106A00000F9108950F931F93CF93DF93C4E5DEE0BA
:106A1000FE0184918E01882331F06DDE0F5F1F4FE0
:106A2000F8018491F8CFE7E2F7E084918F018823A1
:106A300031F061DE0F5F1F4FF8018491F8CF8AE0DB
:106A40005ADEFE01849104E51EE0882331F053DE16
:106A50000F5F1F4FF8018491F8CF4091AA17509112
:106A6000AB176091AC177091AD178FE197E00E9462
:106A7000F4464091AE175091AF176091B0177091E6
:106A8000B1178CE197E00E94F4464091B217509103
:106A9000B3176091B4177091B51789E197E00E9420
:106AA000F4464091B6175091B7176091B81770919E
:106AB000B91786E197E00E94F4468AE01CDEFE01E9
:106AC000849104E51EE0882331F015DE0F5F1F4F2F
:106AD000F8018491F8CFECEFF6E084918F018823E0
:106AE00031F009DE0F5F1F4FF8018491F8CF8AE083
:106AF00002DEFE01849104E51EE0882331F0FBDD17
:106B00000F5F1F4FF8018491F8CF4091BA17509151
:106B1000BB176091BC177091BD1783EF96E00E9480
:106B2000F4464091BE175091BF176091C017709105
:106B3000C11780EF96E00E94F4464091C217509131
:106B4000C3176091C4177091C5178DEE96E00E942F
:106B5000F4464091C6175091C7176091C8177091BD
:106B6000C9178AEE96E00E94F4468AE0C4DDFE0171
:106B7000849104E51EE0882331F0BDDD0F5F1F4FD7
:106B8000F8018491F8CFECECF6E084918F01882332
:106B900031F0B1DD0F5F1F4FF8018491F8CF8AE02B
:106BA000AADDFE01849104E51EE0882331F0A3DD17
:106BB0000F5F1F4FF8018491F8CF40919A175091C1
:106BC0009B1760919C1770919D1783EC96E00E9433
:106BD0001C4740919E1750919F176091A01770918C
:106BE000A11780EC96E00E941C474091A21750919B
:106BF000A3176091A4177091A5178DEB96E00E94E2
:106C00001C474091A6175091A7176091A817709143
:106C1000A9178AEB96E00E941C478AE06CDDFE0112
:106C2000849104E51EE0882331F065DD0F5F1F4F7E
:106C3000F8018491F8CFE5E8F6E084918F0188238C
:106C400031F059DD0F5F1F4FF8018491F8CF8AE0D2
:106C500052DDFE01849104E51EE0882331F04BDD16
:106C60000F5F1F4FF8018491F8CF40919217509118
:106C7000931760919417709195178CE796E00E9496
:106C8000F44640918E1750918F1760919017709134
:106C9000911789E796E00E94F4468AE02CDDFE0118
:106CA000849104E51EE0882331F025DD0F5F1F4F3E
:106CB000F8018491F8CFE6ECF5E084918F01882308
:106CC00031F019DD0F5F1F4FF8018491F8CF8AE092
:106CD00012DDFE01849104E51EE0882331F00BDD16
:106CE0000F5F1F4FF8018491F8CF40919617509194
:106CF000971760919817709199178DEB95E00E9406
:106D0000F44640917A1750917B1760917C177091EF
:106D10007D178AEB95E00E94F4464091CA17509186
:106D2000CB176091CC177091CD1787EB95E00E943F
:106D30001C4740917E1750917F176091801770918A
:106D4000811784EB95E00E94F446409182175091A0
:106D50008317609184177091851781EB95E00E94ED
:106D6000F44640918617509187176091881770916B
:106D700089178EEA95E00E94F44640918A17509157
:106D80008B1760918C1770918D178BEA95E00E949C
:106D9000F4468AE0B0DCFE01849104E51EE088231D
:106DA00031F0A9DC0F5F1F4FF8018491F8CFE9E9BA
:106DB000F5E084918F01882331F09DDC0F5F1F4F38
:106DC000F8018491F8CF8AE096DCFE01849104E515
:106DD0001EE0882331F08FDC0F5F1F4FF801849194
:106DE000F8CF40912A0950912B0960912C0970919C
:106DF0002D0980E995E00E94F44640912E095091BA
:106E00002F0960913009709131098DE895E00E9459
:106E1000F4464091320950913309609134097091E0
:106E200035098AE895E00E94F4468AE064DCFE01B8
:106E3000849104E51EE0882331F05DDC0F5F1F4F75
:106E4000F8018491F8CFECE7F5E084918F01882375
:106E500031F051DC0F5F1F4FF8018491F8CF8AE0C9
:106E60004ADCFE01849104E51EE0882331F043DC16
:106E70000F5F1F4FF8018491F8CF4091AA02509103
:106E8000AB026091AC027091AD0282E795E00E9486
:106E9000F4466091A6027091A7028091A802909199
:106EA000A9020F94A133AB01BC018FE695E00E94CB
:106EB000F4466091A2027091A3028091A402909185
:106EC000A5020F94AD33AB01BC018CE695E00E94A6
:106ED000F4468AE010DCFE01849104E51EE088237C
:106EE00031F009DC0F5F1F4FF8018491F8CFE6E520
:106EF000F5E084918F01882331F0FDDB0F5F1F4F98
:106F0000F8018491F8CF8AE0F6DBFE01849104E574
:106F10001EE0882331F0EFDB0F5F1F4FF8018491F3
:106F2000F8CF40919A0250919B0260919C0270911F
:106F30009D028CE495E00E94F44660919602709167
:106F4000970280919802909199020F94A133AB011E
:106F5000BC0189E495E00E94F44660919202709130
:106F6000930280919402909195020F94AD33AB01FE
:106F7000BC0186E495E00E94F4468AE0BCDBFE0199
:106F8000849104E51EE0882331F0B5DB0F5F1F4FCD
:106F9000F8018491F8CFE2E1F5E084918F01882334
:106FA00031F0A9DB0F5F1F4FF8018491F8CF8AE021
:106FB000A2DBFE01849104E51EE0882331F09BDB17
:106FC0000F5F1F4FF8018491F8CF40912602509136
:106FD0002702609128027091290288E095E00E94C2
:106FE000F44620E030E040E752E460911E027091E8
:106FF0001F0280912002909121020F94BDC1AB012C
:10700000BC0185E095E00E94F44640911A09509138
:107010001B0960911C0970911D0982E095E00E9496
:10702000F4468AE068DBFE01849104E51EE08823D3
:1070300031F061DB0F5F1F4FF8018491F8CFE6ED6F
:10704000F4E084918F01882331F055DB0F5F1F4FEF
:10705000F8018491F8CF8AE04EDBFE01849104E5CB
:107060001EE0882331F047DB0F5F1F4FF80184914A
:10707000F8CF409116095091170960911809709145
:1070800019098CEC94E00E94F44620E030E040E7DF
:1070900052E460911A0270911B0280911C0290913F
:1070A0001D020F94BDC1AB01BC0189EC94E00E94AC
:1070B000F4468AE020DBFE01849104E51EE088238B
:1070C00031F019DB0F5F1F4FF8018491F8CFEFE625
:1070D000F4E084918F01882331F00DDB0F5F1F4FA7
:1070E000F8018491F8CF8AE006DBFE01849104E583
:1070F0001EE0882331F0FFDA0F5F1F4FF801849103
:10710000F8CF40911F0950E060E070E085E694E020
:107110000E941C478AE0EFDAFE01849104E51EE03C
:10712000882331F0E8DA0F5F1F4FF8018491F8CF20
:1071300080914609882339F1E2E5F4E084918F01DA
:10714000882331F0D8DA0F5F1F4FF8018491F8CF10
:107150008AE0D1DAFE01849104E51EE0882331F053
:10716000CADA0F5F1F4FF8018491F8CF40914602B1
:1071700050914702609148027091490288E494E07E
:107180000E94F4460BC0ECE2F4E08491EF01882306
:1071900029F0B1DA2196FE018491F9CF8AE0DF91DE
:1071A000CF911F910F91A7CAAF92BF92CF92DF925A
:1071B000EF92FF920F931F93CF93DF93CDB7DEB77C
:1071C000E0970FB6F894DEBF0FBECDBF80E1E7EECB
:1071D000F2E0DE01919601900D928A95E1F780E14F
:1071E000E7EFF2E0DE01519601900D928A95E1F70A
:1071F00080E1E7E0F3E0DE01119601900D928A95BF
:10720000E1F76E0181E2C80ED11C8AEAE82E87E11F
:10721000F82E8E010F5E1F4F6AEB77E1AE014F5FD4
:107220005F4F9AE9A92E97E1B92E20E030E0F601F0
:1072300081919191A191B1916F01F7018193919306
:10724000A193B1937F01F80181919191A191B191A5
:107250008F01FB0181939193A193B193BF01FA0137
:1072600081919191A191B191AF01F5018193919398
:10727000A193B1935F012F5F3F4F24303105B9F6E1
:107280000F94331380E090E4ACE9B4E48093921758
:1072900090939317A0939417B093951780938E179C
:1072A00090938F17A0939017B09391171092961701
:1072B00010929717109298171092991780E29EE4F7
:1072C000A0E0B0E08093CA179093CB17A093CC179F
:1072D000B093CD1710927A1710927B1710927C17EB
:1072E00010927D1780E090E0A0E2B1E480937E17D9
:1072F00090937F17A0938017B09381178093821784
:1073000090938317A0938417B09385178DEC9CEC12
:10731000ACECBEE38093861790938717A0938817F1
:10732000B093891780E090E0A0E2B0E480938A17E0
:1073300090938B17A0938C17B0938D1710923209EE
:1073400010923309109234091092350910922E09C7
:1073500010922F09109230091092310910922A09C7
:1073600010922B0910922C0910922D098DE39AE0AE
:10737000A1E8B1E48093AA029093AB02A093AC027F
:10738000B093AD026DEC7CEC84E99FE30F949B33EA
:107390006093A6027093A7028093A8029093A9021B
:1073A00065E87BEE80E692E40F94A7336093A20237
:1073B0007093A3028093A4029093A5020F94B82324
:1073C00080E090E0A0E8BFE380939E0290939F024C
:1073D000A093A002B093A10210921F0980E090E058
:1073E000A0E4B0E48093260290932702A0932802A1
:1073F000B093290240E050E064E372E440931E023F
:1074000050931F02609320027093210210921A0978
:1074100010921B0910921C0910921D091092160956
:1074200010921709109218091092190940E050E0C3
:1074300060E071E440931A0250931B0260931C02B7
:1074400070931D0210924609809346029093470262
:10745000A0934802B09349020E94305CE4E5FEE04C
:1074600084918F01882331F046D90F5F1F4FF801B7
:107470008491F8CFE0EFF3E084918F01882331F01D
:107480003AD90F5F1F4FF8018491F8CF8AE0E09658
:107490000FB6F894DEBF0FBECDBFDF91CF911F9125
:1074A0000F91FF90EF90DF90CF90BF90AF9023C9E6
:1074B0000F931F93CF93DF93CDB7DEB72C970FB603
:1074C000F894DEBF0FBECDBF8C019C878B8746E54D
:1074D00052E360E070E049835A836B837C8344E02D
:1074E000BE016B5F7F4FCE010B965FD943E050E04A
:1074F000BE016B5F7F4FCE0101960F94CAC7892BE7
:1075000009F009C140E16AEA77E1CE010B964DD955
:1075100040E16AEB77E1CE010B9647D940E16AE999
:1075200077E1CE010B9641D90F94331344E062E921
:1075300077E1CE010B9639D944E06EE877E1CE01D0
:107540000B9633D944E066E977E1CE010B962DD94D
:1075500044E06AE777E1CE010B9627D944E06AEC74
:1075600077E1CE010B9621D944E06EE777E1CE01B9
:107570000B961BD944E062E877E1CE010B9615D952
:1075800044E066E877E1CE010B960FD944E06AE863
:1075900077E1CE010B9609D920E030E040E251E4DA
:1075A00060917E1770917F1780918017909181175D
:1075B0000F94EBC0181664F480E090E0A0E2B1E410
:1075C00080937E1790937F17A0938017B0938117B5
:1075D00020E030E040E251E460918217709183171F
:1075E00080918417909185170F94EBC0181664F45E
:1075F00080E090E0A0E2B1E480938217909383173B
:10760000A0938417B09385174CE06AE279E0CE012D
:107610000B96CBD844E063E279E0CE010B96C5D857
:1076200044E06AEA72E0CE010B96BFD844E066EA15
:1076300072E0CE010B96B9D844E062EA72E0CE0166
:107640000B96B3D844E06AE972E0CE010B96ADD850
:1076500044E066E972E0CE010B96A7D844E062E907
:1076600072E0CE010B96A1D842E0BE01675F7F4F6A
:10767000CE010B969AD841E06FE179E0CE010B96EE
:1076800094D844E066E272E0CE010B968ED844E0D6
:107690006EE172E0CE010B9688D844E06AE179E0B1
:1076A000CE010B9682D844E066E179E0CE010B96DC
:1076B0007CD844E06AE172E0CE010B9676D841E0D6
:1076C00066E479E0CE010B9670D844E066E472E09F
:1076D000CE010B966AD80F94B823E4E5FEE08491BE
:1076E0008F01882331F007D80F5F1F4FF801849175
:1076F000F8CFE2E1F4E084918F01882339F00E9411
:107700007B330F5F1F4FF8018491F7CF8AE00E940F
:107710007B3391E014C048DDC8010F9423CB8F3F29
:1077200069F4C80101960F9423CB8F3F39F4C80147
:1077300002960F9423CB91E08F3F09F090E0892FC0
:107740002C960FB6F894DEBF0FBECDBFDF91CF9160
:107750001F910F910895CF93DF93EC0160E08E812C
:107760000F9435B881E090E00F9477B661E08E8198
:107770000F9435B881E090E00F9477B660E08E8189
:107780000F9435B884E690E0DF91CF910D9477B6F1
:10779000CF92DF92EF92FF920F931F93CF93DF93DD
:1077A0007C01C0E0D0E0C62ED12C87010C0F1D1F3C
:1077B00061E0F80187810F94FCB7B6010C2E02C07E
:1077C000759567950A94E2F76170F80187810F94C7
:1077D00035B82196C430D10541F7C701DF91CF916B
:1077E0001F910F91FF90EF90DF90CF90B4CFCF9289
:1077F000DF92EF92FF920F931F93CF93DF937C0161
:10780000C0E0D0E0C62ED12C87010C0F1D1F61E017
:10781000F80187810F94FCB7B6010C2E02C0759554
:1078200067950A94E2F76170F80187810F9435B883
:107830002196C830D10541F7C701DF91CF911F9143
:107840000F91FF90EF90DF90CF9085CF1F93CF9354
:10785000DF93EC01162F642F8C810F9435B88D8146
:107860008F3F19F060E00F9435B88F85612F84FF4A
:1078700005C0CE01DF91CF911F91B9CF70E084E0B8
:10788000759567958A95E1F7CE0182DF612FCE016C
:10789000DF91CF911F917CCF40E0D8CF61E0FCDF3A
:1078A00080E496E00D9477B662E0F6DF80E496E03F
:1078B0000D9477B6CF93DF93CDB7DEB728970FB689
:1078C000F894DEBF0FBECDBF28E0E7E1F3E0DE01B4
:1078D000119601900D922A95E1F7FC012389421738
:1078E00010F04FEF420FFE013196E40FF11DE40F4F
:1078F000F11D2081260F2068622F28960FB6F8947C
:10790000DEBF0FBECDBFDF91CF91C6CFFC01608936
:10791000262F2460208B6C60BFCFCF93DF93EC01C8
:10792000423018F08F8588608F874B8B1C8A22230A
:1079300029F0413019F48F8584608F8780E593ECBE
:107940000F9477B660E08C810F9435B860E08E813B
:107950000F9435B88D818F3F19F060E00F9435B8E2
:107960006F8564FD19C063E0CE0112DF84E991E107
:107970000F9477B663E0CE010BDF84E991E10F94B9
:1079800077B663E0CE0104DF86E990E00F9477B626
:1079900062E0CE01FDDE13C06062CE017DDF84E9CE
:1079A00091E10F9477B66F856062CE0175DF86E94D
:1079B00090E00F9477B66F856062CE016DDF6F85C2
:1079C0006062CE0169DF8CE390E00F9477B684E0CB
:1079D000888BCE019BDF8CE390E00F9477B6CE01CD
:1079E0005DDF88EB9BE00F9477B682E0898B66E0E1
:1079F000CE0152DF8CE390E00F9477B61D8ADF91C1
:107A0000CF9108956F927F928F92AF92CF92EF9223
:107A10000F931F93CF93DF93CDB7DEB73C01162FA3
:107A2000842F5E854F8538899989F3018483258366
:107A30000683E782C086A18682865387448735877E
:107A4000968761E00F94FCB7F30185818F3F19F0B1
:107A500061E00F94FCB761E0F30186810F94FCB7FD
:107A6000112319F0F301178603C080E1F301878722
:107A700020E041E060E1C301DF91CF911F910F91C0
:107A8000EF90CF90AF908F907F906F9046CF8F9276
:107A9000AF92CF92EF920F93DC0113961C921E923D
:107AA0001297E4E8F3E0ED93FC931F921F921F926C
:107AB0001F928C2CAE2CC02EE22E042F2FEF462FBF
:107AC00061E0A0DF0F900F900F900F900F91EF905B
:107AD000CF90AF908F900895CF93DF93EC01423019
:107AE00018F08F8588608F874B8B1C8A222329F0A2
:107AF000413019F48F8584608F8780E593EC0F9473
:107B000077B660E08C810F9435B860E08E810F9479
:107B100035B88D818F3F19F060E00F9435B86F85CF
:107B200064FD19C063E0CE0133DE84E991E10F9476
:107B300077B663E0CE012CDE84E991E10F9477B64D
:107B400063E0CE0125DE86E990E00F9477B662E02F
:107B5000CE011EDE13C06062CE019EDE84E991E19B
:107B60000F9477B66F856062CE0196DE86E990E06D
:107B70000F9477B66F856062CE018EDE6F8560628E
:107B8000CE018ADE8CE390E00F9477B684E0888B98
:107B9000CE01BCDE8CE390E00F9477B6CE0184DE9C
:107BA00080E496E00F9477B682E0898B66E0CE01A0
:107BB00073DE8CE390E00F9477B640E068E0CE018E
:107BC00079DE6FE077E0CE010F94D0B841E068E055
:107BD000CE0170DE6FE077E0CE010F94D0B842E0C6
:107BE00066E0CE0167DE6DE077E0CE01DF91CF91F8
:107BF0000D94D0B8FC0160896D7F608B68604CCEBD
:107C0000CF93DF93EC01262F8D898230B0F0FE01F7
:107C1000E80FF11D658B3E8980ED860F8A3058F4A0
:107C2000316081E090E00D8802C0880F991F0A94AE
:107C3000E2F7382B01C03E7F3E8B4D8981E0840FF7
:107C40008D8B50E04830510508F0B6C0FA01EE586F
:107C5000FF4F0D94FDC32B3109F0AEC0AEC01E8A9C
:107C60002B3509F0A9C0A9C0223309F4A6C02F33CF
:107C700009F4A3C08E897AC08F89823331F08F33A3
:107C800049F4223309F098C098C02A3419F4CE017F
:107C900005DE92C08E8982FF8FC02B3309F066C04B
:107CA0008CC08F898F3341F4888D823309F084C072
:107CB000253309F081C081C08E8982FF7DC0988DF7
:107CC0009B3311F480FD79C083FF76C02B3309F01C
:107CD00073C073C04F894F3371F4888D823309F0BC
:107CE0006BC0898D853309F067C02C3609F064C0FC
:107CF000CE0180DF61C08E8982FF5EC0988D9B338C
:107D000039F484FF05C0283489F54053698D2CC0AF
:107D100083FF52C0998D9B3309F04EC027C08E89D6
:107D200082FF4AC0488D4B3361F4982F9073903393
:107D300041F4283431F44F8940536A8D6053898D62
:107D400032C083FF39C0998D9B33B1F585FF34C0B4
:107D5000283461F440538F89880F8056982F990FEB
:107D6000990F980F490F6A8D605324C080FF24C07B
:107D700024C08E89982F9C709C30F1F4998D9B3390
:107D8000D9F480768036C1F42834B1F4488D40535C
:107D90008F89880F8056982F990F990F980F490F48
:107DA0006B8D60538A8D880F8056982F990F990F8D
:107DB000980F690FCE017EDD1D8A81E090E0DF9192
:107DC000CF910895CF92DF92EF92FF920F931F937E
:107DD000CF93DF931F921F92CDB7DEB78C016770F0
:107DE00088E0689FB00111246064C80149835A8308
:107DF00053DD4981C42E5A81D52EE12CF12CD601B8
:107E00006D916D01D801ED91FC910190F081E02D13
:107E1000C8011995BFEFEB1AFB0AE8E0EE16F10472
:107E200071F70F900F90DF91CF911F910F91FF90FD
:107E3000EF90DF90CF900895FC012589211102C0B9
:107E40006B3109F4DDCE41E001DD81E090E0089581
:107E500090915908911107C09091C00095FFFCCFF7
:107E60008093C6000895913031F49091C80095FF39
:107E7000FCCF8093CE0008951F920F920FB60F9201
:107E800011240BB60F922F933F934F935F936F93F1
:107E90008F939F93EF93FF938091C00084FF03C063
:107EA0008091C6001DC06091C60080915908811163
:107EB00017C02091550830915608C90101968F7757
:107EC000992740915708509158088417950741F019
:107ED000F901EB52F84F6083909356088093550850
:107EE000FF91EF919F918F916F915F914F913F9192
:107EF0002F910F900BBE0F900FBE0F901F901895F3
:107F00001F920F920FB60F9211240BB60F922F9360
:107F10003F934F935F936F938F939F93EF93FF9351
:107F20008091C80084FF03C08091CE001DC0609185
:107F3000CE00809159088130B9F4209155083091D4
:107F40005608C90101968F7799274091570850919B
:107F500058088417950741F0F901EB52F84F6083F8
:107F60009093560880935508FF91EF919F918F91C0
:107F70006F915F914F913F912F910F900BBE0F909A
:107F80000FBE0F901F901895CF92DF92EF92FF9245
:107F90006A017B01411581EE58076105710509F4FD
:107FA00063C082E08093C00060E079E08DE390E000
:107FB000A70196010F94E1C32150310941095109EC
:107FC000CA01B90122E030E040E050E00F94E1C383
:107FD00091E03093C5002093C4008091C10080617E
:107FE0008093C1008091C10088608093C10080911E
:107FF000C10080688093C100809159088130D1F51B
:10800000992341F082E08093C80060E079E08DE33D
:1080100090E006C01092C80060E874E88EE190E03D
:10802000A70196010F94E1C321503109410951097B
:10803000CA01B90122E030E040E050E00F94E1C312
:108040003093CD002093CC008091C9008061809353
:10805000C9008091C90088608093C9008091C900DF
:1080600080688093C90006C01092C00090E020E1B3
:1080700030E0AFCFFF90EF90DF90CF900895209148
:1080800057083091580880915508909156088217EA
:10809000930771F0F901EB52F84F80812F5F3F4F4A
:1080A0002F773327309358082093570890E008958E
:1080B0008FEF9FEF08958091570890915808909303
:1080C00056088093550808954F925F926F927F9261
:1080D0008F929F92AF92BF92CF92DF92EF92FF92D8
:1080E0000F931F93CF93DF93CDB7DEB7A0970FB653
:1080F000F894DEBF0FBECDBF411551056105710576
:10810000C1F480E3A0960FB6F894DEBF0FBECDBFDA
:10811000DF91CF911F910F91FF90EF90DF90CF9063
:10812000BF90AF909F908F907F906F905F904F9097
:108130008FCECE0101967C01812C912C54018C01B3
:10814000422E512C612C712C9FEF891A990AA90A91
:10815000B90ACB01BA01A30192010F94BFC3CA01AE
:10816000F70161937F01A901BC014115510561052A
:10817000710551F775016401F1E0CF1AD108E108EA
:10818000F108F801EC0DFD1D80818A3010F4805D4E
:1081900001C0895C5DDE81E0C81AD108E108F10800
:1081A0009FEFC916D906E906F90659F7A0960FB64A
:1081B000F894DEBF0FBECDBFDF91CF911F910F911D
:1081C000FF90EF90DF90CF90BF90AF909F908F90F7
:1081D0007F906F905F904F9008952115310511F4B5
:1081E000842F36CE71CF0F931F93CF93DF9300D0A0
:1081F0001F92CDB7DEB78C0177FF11C08DE24983A6
:108200005A836B837C8324DE49815A816B817C8114
:1082100070956095509541955F4F6F4F7F4F2AE065
:10822000C8010F900F900F900F90DF91CF911F9189
:108230000F914ACF2115310511F4842F09CE2A3030
:10824000310509F4D0CF40CF9A01462F552747FD7D
:108250005095652F752FEECF9A01AB01662757FD1C
:108260006095762FE7CF8DE0F3DD8AE0F1CD0F93B7
:108270001F93CF93DF938C01EB018991882311F039
:10828000E7DDFBCFC801DF91CF911F910F91EBCFBD
:10829000CF93DF93EC019A01AB01662757FD609500
:1082A000762FC8DFCE01DF91CF91DDCFCF93DF9363
:1082B000EC019A01462F50E060E070E08EDFCE01C5
:1082C000DF91CF91D0CFCF93DF93EC019A01AB0137
:1082D00060E070E082DFCE01DF91CF91C4CFCF9319
:1082E000DF93EC017ADFCE01DF91CF91BCCF8F928B
:1082F0009F92AF92BF92CF92DF92EF92FF921F9325
:10830000CF93DF93EC016A017B01122F20E030E074
:10831000A901C701B6010F94E8BE87FF06C08DE230
:1083200097DDF7FAF094F7F8F094B12C60E070E084
:1083300080E09FE3B11641F020E030E040E251E4FC
:108340000F94EFBEB394F6CF9B01AC01C701B60109
:108350000F940FBE6B017C010F945CBF4B015C015D
:108360000F9488BF9B01AC01C701B6010F940EBEEC
:108370006B017C012AE0B501A401CE01A5DE112329
:1083800059F08FE2A82E85E0B82EF50181915F01AA
:10839000882311F05DDDF9CF112319F120E030E0E1
:1083A00040E251E4C701B6010F94BDC16B017C01ED
:1083B0000F9457BF4B01AA2497FCA094BA2CB50187
:1083C000A401CE0110DFC501B4010F948ABF9B0147
:1083D000AC01C701B6010F940EBE6B017C011150B8
:1083E000DBCFDF91CF911F91FF90EF90DF90CF9087
:1083F000BF90AF909F908F90089579CFCF93DF93E8
:10840000EC0175DFCE01DF91CF912DCFFC0165919D
:108410007591859194910895EF92FF920F931F9318
:10842000CF93DF93EC01CC0FDD1FCC0FDD1FCE010E
:10843000805D914FEBDF9E012A5C364F79018E0102
:10844000065D164FF80120813181428153810F94DE
:108450000FBEF7016083718382839383CE01885BB3
:10846000914FD4DF9E012A5C3D4F7901F8012081B4
:108470003181428153810F940FBEF7016083718374
:1084800082839383CE01845C914FC0DFC65DDD4F54
:10849000F80120813181428153810F940FBE68839E
:1084A00079838A839B83DF91CF911F910F91FF90F6
:1084B000EF90089520910C0F30910D0FBC01C90170
:1084C0008F5E904F0F94E7C79093030F8093020F36
:1084D00021E0892B09F420E0822F0895CF93C82F43
:1084E00040910E0250910F026091100270911102A2
:1084F0004093ED085093EE086093EF087093F008F6
:1085000020915802309159023093B7092093B6094F
:1085100024E630E030935902209358020F9411B6AC
:108520006093E8087093E9088093EA089093EB0859
:108530008C2FCF910D94CD1480E00F94CD148091A9
:10854000ED089091EE08A091EF08B091F0088093AB
:108550000E0290930F02A0931002B093110280912B
:10856000B6099091B70990935902809358020F94DD
:1085700011B66093E8087093E9088093EA08909335
:10858000EB080895682F772767FD709580910C0F91
:1085900090910D0F8F5E904F0F94AFC79093030F84
:1085A0008093020F21E0892B09F420E0822F0895A7
:1085B0008091020F9091030F4AE050E060E070E07C
:1085C00001960F94C0C5CB0108958091020F909140
:1085D000030F4AE050E060E070E001960D94C0C5E2
:1085E0008091020F9091030F60E070E001960D946E
:1085F00058C490915908911107C09091C00095FFFF
:10860000FCCF8093C6000895913031F49091C8005A
:1086100095FFFCCF8093CE000895EBDF80E090E0E3
:1086200008952F923F924F925F926F927F928F9216
:108630009F92AF92BF92CF92DF92EF92FF920F93F1
:108640001F93CF93DF93CDB7DEB760970FB6F89443
:10865000DEBF0FBECDBF1C012A013B0148015901FD
:1086600020E030E04CE052E4C301B2010F940EBEB2
:1086700025E535E547E052E40F94EFBE6B017C0140
:108680000F94C5BF0F9457BF8B0177FF12C020E036
:1086900030E040E85FE3C701B6010F94EBC0181665
:1086A0000CF05DC0C12CD12CE0E8EE2EEFE3FE2EE5
:1086B00056C066307105DCF02AEA3AE24CE453E435
:1086C000C301B2010F940EBE25E535E547E052E443
:1086D0000F94EFBE6B017C0120E030E0A9010F9404
:1086E000E8BE87FF3FC0C12CD12C76013BC0882754
:1086F00077FD8095982F0F948ABF25E535E547E0F3
:1087000052E40F94BDC120E030E04CE052E40F94FD
:108710000FBE9B01AC01C301B2010F940EBE25E553
:1087200035E547E052E40F94EFBE6B017C0120E099
:1087300030E0A9010F94E8BE87FD17C020E030E0CB
:1087400040E85FE3C701B6010F94EBC0181684F44C
:10875000C12CD12C70E8E72E7FE3F72E09C000E092
:1087600010E006C005E010E003C0C12CD12C76015A
:1087700020E030E040EC50E4C501B4010F940EBE9F
:108780002BEA3AEA42E052E40F94EFBE2B013C019F
:108790000F94C5BF0F9457BF788B6F8777FF12C0B8
:1087A00020E030E040E85FE3C301B2010F94EBC08A
:1087B00018160CF05FC0412C512C60E8662E6FE358
:1087C000762E58C0AF85B8891697E4F026E535E5D2
:1087D00049E253E4C501B4010F940EBE2BEA3AEA14
:1087E00042E052E40F94EFBE2B013C0120E030E068
:1087F000A9010F94E8BE87FD40C0E5E0F0E0F88BEA
:10880000EF8746C0882777FD8095982F0F948ABF01
:108810002BEA3AEA42E052E40F94BDC120E030E096
:1088200040EC50E40F940FBE9B01AC01C501B401B4
:108830000F940EBE2BEA3AEA42E052E40F94EFBEE8
:108840002B013C0120E030E0A9010F94E8BE87FD38
:108850001CC020E030E040E85FE3C301B2010F94A8
:10886000EBC01816ACF4412C512C50E8652E5FE398
:10887000752E0EC0188A1F860BC0412C512C320158
:1088800025E030E0388B2F8703C0412C512C32017A
:10889000A701960160E070E080E89FE30F940EBEB0
:1088A00069837A838B839C83C80101969E838D8321
:1088B000AF85B8891196BA87A987A301920160E0B4
:1088C00070E080E89FE30F940EBE6B877C878D87F6
:1088D0009E8747E02F853889429FF001439FF00D26
:1088E0001124F887EF83E00FF11FEE0FFF1FEE0F4B
:1088F000FF1FE20DF31D2181328143815481698183
:108900007A818B819C810F94BDC14B015C01EF8109
:10891000F8858D819E81E80FF91FEE0FFF1FEE0F86
:10892000FF1FE20DF31D2181328143815481C70174
:10893000B6010F94BDC19B01AC01C501B4010F94F8
:108940000FBE9B01AC016B857C858D859E850F9448
:10895000BDC14B015C0127E0E985FA852E9FD0015E
:108960002F9FB00D1124B887AF83FD01E00FF11FD9
:10897000EE0FFF1FEE0FFF1FE20DF31D218132816D
:108980004381548169817A818B819C810F94BDC11F
:1089900069837A838B839C83AF81B8858D819E8127
:1089A000A80FB91FAA0FBB1FAA0FBB1FA20DB31D93
:1089B00011962D913D914D915C911497C701B6018F
:1089C0000F94BDC19B01AC0169817A818B819C812F
:1089D0000F940FBE9B01AC01C301B2010F94BDC146
:1089E0009B01AC01C501B4010F940FBE60960FB698
:1089F000F894DEBF0FBECDBFDF91CF911F910F91D5
:108A0000FF90EF90DF90CF90BF90AF909F908F90AE
:108A10007F906F905F904F903F902F9008954F926E
:108A20005F926F927F929F92AF92BF92CF92DF92AE
:108A3000EF92FF920F931F93CF93DF937C015B0123
:108A40008A01E90190904A11911014C0FC018081C3
:108A50009181A281B381FA0180839183A283B38340
:108A6000FB0180819181A281B38188839983AA834C
:108A7000BB837FC091FE55C0FC01208131814281C2
:108A8000538160913A1170913B1180913C1190910A
:108A90003D110F94BDC12B013C01F50120813181B5
:108AA0004281538160913E1170913F11809140113C
:108AB000909141110F94BDC19B01AC01C301B20162
:108AC0000F940FBEF8016083718382839383F70153
:108AD0002081318142815381609142117091431113
:108AE00080914411909145110F94BDC16B017C019F
:108AF000F50120813181428153816091461170914D
:108B0000471180914811909149110F94BDC19B016B
:108B1000AC01C701B6010F940FBE688379838A83C5
:108B20009B8390FE26C02091221130912311409109
:108B3000241150912511F801608171818281938106
:108B40000F940FBEF8016083718382839383209119
:108B500026113091271140912811509129116881D7
:108B600079818A819B810F940FBE688379838A8380
:108B70009B83DF91CF911F910F91FF90EF90DF903A
:108B8000CF90BF90AF909F907F906F905F904F90ED
:108B900008952F923F924F925F926F927F928F92A1
:108BA0009F92AF92BF92CF92DF92EF92FF920F937C
:108BB0001F93CF93DF93CDB7DEB728970FB6F89406
:108BC000DEBF0FBECDBF8C011B019E012F5F3F4F4B
:108BD000AE014B5F5F4F23DF20E030E0A9016D81E4
:108BE0007E818F8198850F94E8BE87FF07C01D8224
:108BF0001E821F821886FF24F39401C0F12C20E00E
:108C000030E040E850EC69817A818B819C810F943F
:108C1000E8BE87FF0AC080E090E0A0E8B0EC89835E
:108C20009A83AB83BC83FF24F39420E030E04FE7CA
:108C300053E46D817E818F8198850F94EBC0181667
:108C400054F480E090E0AFE7B3E48D839E83AF837C
:108C5000B887FF24F39420E030E042E553E46981D3
:108C60007A818B819C810F94EBC018164CF480E0C4
:108C700090E0A2E5B3E489839A83AB83BC8303C00D
:108C8000FF2009F483C0C980DA80EB80FC808D80EE
:108C90009E80AF80B88470904A1171100BC0F801AB
:108CA00080829182A282B382F101C082D182E2826B
:108CB000F3826AC070FE1CC02091221130912311F2
:108CC0004091241150912511C501B4010F940EBE9D
:108CD0004B015C0120912611309127114091281100
:108CE00050912911C701B6010F940EBE6B017C0192
:108CF00071FE4AC020912A1130912B1140912C1104
:108D000050912D11C501B4010F94BDC12B013C013F
:108D100020912E1130912F1140913011509131112D
:108D2000C701B6010F94BDC19B01AC01C301B201E3
:108D30000F940FBEF8016083718382839383209127
:108D40003211309133114091341150913511C501D8
:108D5000B4010F94BDC14B015C01209136113091DB
:108D600037114091381150913911C701B6010F9454
:108D7000BDC19B01AC01C501B4010F940FBEF1014F
:108D80006083718382839383FF24F3948F2D2896CD
:108D90000FB6F894DEBF0FBECDBFDF91CF911F910C
:108DA0000F91FF90EF90DF90CF90BF90AF909F908A
:108DB0008F907F906F905F904F903F902F9008958D
:108DC000CF93DF931F92CDB7DEB7BE016F5F7F4FAA
:108DD0000F94C8880F90DF91CF910895682F87EF87
:108DE0009FE00D9435CB08950F931F93CF93DF939E
:108DF00000D01F92CDB7DEB78C01FC01849188238F
:108E000071F049835A836B837C83F3DB0F5F1F4FC1
:108E1000F80184917C816B815A814981F0CF22E0F5
:108E200030E084ED97E00F900F900F900F90DF915E
:108E3000CF911F910F91E1CA0F931F93CF93DF93AF
:108E400000D01F92CDB7DEB78C01FC01849188233E
:108E500071F049835A836B837C83CBDB0F5F1F4F99
:108E6000F80184917C816B815A814981F0CF2AE09D
:108E700030E084ED97E00F900F900F900F90DF910E
:108E8000CF911F910F91A9C9CF93C1E0C093AE02BA
:108E90006FEF89E69FE00F9435CBC093E402CF914A
:108EA00008951092AE0210920C1960E089E69FE0DE
:108EB0000F9435CB1092E4020895CF93C82F0F94EE
:108EC000891C81E00F94CD870F943D4882E00F9478
:108ED000FF84C0FF15C086E69FE00F9423CB61E0BE
:108EE000680F86E69FE00F9435CB85E09FE00F94F6
:108EF00030CBBC016F5F7F4F85E09FE00F944FCB7D
:108F0000C1FF15C088E69FE00F9423CB61E0680F96
:108F100088E69FE00F9435CB83E09FE00F9430CB41
:108F2000BC016F5F7F4F83E09FE00F944FCB81E0E8
:108F30000F94CD8782E00F94FF84E0918609F0E0E2
:108F4000EE0FFF1FE252F54B859194910F949649D5
:108F500061E08DE09EE00E9469C461E08FEF9DE0DA
:108F6000CF910C9469C41092C20960E080EC99E042
:108F70000E94A5B881E08093AE02089560E086E685
:108F80009FE00F9435CB60E088E69FE00F9435CBEF
:108F900060E085E69FE00F9435CB60E084E69FE0DB
:108FA0000D9435CBEF92FF920F931F93CF93DF93E6
:108FB0001F92CDB7DEB789830F943D4889818230F7
:108FC00009F495C00CF062C0882309F46EC08130AA
:108FD00009F025C19FB7F8948091020184608093C5
:108FE00002019FBFEFEFF1EE24E0E150F04020409E
:108FF000E1F700C000009FB7F894809102018B7FD9
:10900000809302019FBF40E050E0BA018DEE9FE0E7
:109010000F9447CB40E050E0BA0181EF9FE00F94FE
:1090200047CB60E086E69FE00F9435CB60E088E6B2
:109030009FE00F9435CB60E085E69FE00F9435CB41
:1090400060E084E69FE00F9435CB60E070E085E05F
:109050009FE00F944FCB60E070E083E09FE00F94BF
:109060004FCB60E070E081E09FE00F944FCB60E079
:1090700070E08FEF9EE00F944FCB0F90DF91CF9178
:109080001F910F91FF90EF900D948F67833009F43B
:1090900061C0843009F0C3C00F90DF91CF911F9160
:1090A0000F91FF90EF900D94BF8F9FB7F894809130
:1090B00002018460809302019FBF2FEF81EE94E054
:1090C000215080409040E1F700C000009FB7F89425
:1090D000809102018B7F809302019FBF0F90DF91EF
:1090E000CF911F910F91FF90EF900D9427490F940E
:1090F000274980EF73DE61E08FE59FE00F9453CB4B
:109100001092CA191092C9196091CB1984EC9FE092
:109110000F9435CB69EC79E181EC9FE00F947B48AB
:109120009FB7F894809102018460809302019FBFF1
:109130008FEF91EEE4E081509040E040E1F700C015
:1091400000009FB7F894809102018B7F8093020109
:109150009FBF65C081EF9DE00F946D5B40EE5DE0C9
:1091600062E081E00F94166D9FB7F8948091020140
:109170008460809302019FBFFFEF21EE84E0F150F5
:1091800020408040E1F700C000009FB7F894809134
:1091900002018B7F809302019FBF1092D40810922E
:1091A000D30849ED5DE063E083E00F94166D4091D4
:1091B000D3085091D40863E083E00F944848E12C31
:1091C000F12C09E210E06FEFC7010F9453CBC701F8
:1091D000B8010F94ACC3892BD9F48091D308909136
:1091E000D40801969093D4088093D30842ED5DE0B3
:1091F00063E083E00F94166D4091D3085091D4083A
:1092000063E083E00F94484880ED9DE00F946D5B30
:109210009FEFE91AF90AE114E0E1FE06A1F60F90CA
:10922000DF91CF911F910F91FF90EF90089565EC22
:1092300078E080EA9DE00D941DC884E090E0909372
:109240001802809317028091000186FD39C02FEF2C
:1092500083ED90E3215080409040E1F700C0000092
:109260008091000186FD2CC00F943D4882E99DE06D
:109270000F946D5B809101018460809301019FB721
:10928000F894809102018460809302019FBF8091D5
:10929000000186FFFCCF9FB7F894809102018B7F7D
:1092A000809302019FBF2FEF87EA91E62150804013
:1092B0009040E1F700C000000F94E14C60E072DEE6
:1092C00082E090E090931802809317020895E09155
:1092D0008609F0E0EE0FFF1FEC5BF54B8591949152
:1092E0000F949C9581E00D94CD871F93CF93DF93CE
:1092F0000F949700EC01DF93CF9388E29DE09F935A
:109300008F930F944AC887E69FE00F9423CB182FC2
:109310000F900F900F900F90CD2B29F481E0809348
:10932000091110E002C0109209118FE19DE00F9425
:109330009AC8112349F086E19DE00F949AC8DF9105
:10934000CF911F910C94F4CA8CE09DE00F949AC8C1
:10935000DF91CF911F910C9411CB8F929F92AF927E
:10936000BF92CF92DF92EF92FF92CF93DF938091E3
:10937000CB19811185C00F9411B66B017C0120912E
:109380001202222309F474C040911702509118026E
:109390004130510509F46CC0809113029091140280
:1093A000A0911502B091160246015701881A990A38
:1093B000AA0ABB0A30E0A8EEB3E00F9403C48616F5
:1093C0009706A806B9060CF45BC04430510541F17C
:1093D0004CF4423051050CF44BC0E4E5FEE08491BE
:1093E000EF0109C04530510509F042C0E4E5FEE057
:1093F0008491EF012BC0882329F0FBD82196FE0130
:109400008491F9CFE7EEFCE08491EF01882329F005
:10941000F0D82196FE018491F9CF8AE0EAD828C0DD
:10942000E4E5FEE08491EF01882329F0E2D821965B
:10943000FE018491F9CFE1EDFCE08491EF018823F6
:1094400061F3D7D82196FE018491F9CF882329F0C2
:10945000D0D82196FE018491F9CFEAEBFCE084910B
:10946000EF018823D1F2C5D82196FE018491F9CF6E
:10947000C0921302D0921402E0921502F0921602EA
:10948000DF91CF91FF90EF90DF90CF90BF90AF90A2
:109490009F908F90089580E1E6E3F9E0A1E0B9E0C4
:1094A00001900D928A95E1F70895CF93C0E0209145
:1094B000080F3091090F232BB9F088E893E00E9440
:1094C0005A4281110FC08CE893E00E945A428111E8
:1094D00009C08091070F811102C00E9493C31092AE
:1094E000070FE5CFC1E0F5CF8C2FCF9108952F92D4
:1094F0003F924F925F926F927F928F929F92AF9224
:10950000BF92CF92DF92EF92FF920F931F93CF9370
:10951000DF931F92CDB7DEB70F943D48E0918609E7
:10952000F0E0EE0FFF1FE05FF44B4591549161E0D6
:1095300080E00F94166D81E00F94CD148983E7E1EC
:10954000FEE0E4918E2F992781950CF490951C01F3
:1095500084E00F947536AEE3B9E01D921D921D9222
:109560001C921397EAE3F9E0208131814281538113
:10957000A6E3B9E06D917D918D919C91E2E4CE2EB0
:10958000E9E0DE2EE12CF12C87010F94981183DFA6
:109590008CE29EE00E9406422DEC3CEC4CE85FE33E
:1095A0000F94BDC14B015C01B101882777FD809507
:1095B000982F0F948ABF9B01AC01C501B4010F9491
:1095C000BDC1E9E0F9E020813181428153810F94EE
:1095D0000FBE2B013C01A9E0B9E06D937D938D9303
:1095E0009C931397E2E6F2E060817181828193811E
:1095F00060930E0270930F028093100290931102F9
:1096000020E030E040E752E40F94EFBE4B015C01F4
:10961000A5E0B9E02D913D914D915C91E1E0F9E03B
:109620006081718182819381A2E2B9E0BF93AF939F
:10963000FDE0CF2EF9E0DF2E830172010F942806A2
:109640000F94891C0F94D43680E00F94CD14AEE3B0
:10965000B9E01D921D921D921C921397EAE3F9E066
:109660002081318142815381A6E3B9E06D917D91E2
:109670008D919C91A2E4CA2EA9E0DA2EE12CF12C66
:1096800087010F94981107DF8AE0829DB001839DC6
:10969000700D1124882777FD8095982F0F948ABF2D
:1096A000E9E0F9E020813181428153810F940FBEBE
:1096B0002B013C01A9E0B9E06D937D938D939C93C0
:1096C000139720E030E040E05FE3E2E6F2E0608103
:1096D0007181828193810F94BDC160930E0270935A
:1096E0000F02809310029093110220E030E040E7D7
:1096F00052E40F94EFBE4B015C01A5E0B9E02D915F
:109700003D914D915C91E1E0F9E060817181828150
:109710009381A2E2B9E0BF93AF93BDE0CB2EB9E055
:10972000DB2E830172010F9428060F94891C898116
:109730000F94CD1480E090E0A4E5B3E4EEE3F9E00B
:1097400080839183A283B383AAE3B9E02D913D91F5
:109750004D915C91E6E3F9E06081718182819381B2
:1097600012E4C12E19E0D12EE12CF12C04E513E412
:109770000F94981181E00F900F900F900F900F9021
:10978000DF91CF911F910F91FF90EF90DF90CF90DD
:10979000BF90AF909F908F907F906F905F904F9011
:1097A0003F902F9008952F923F924F925F926F9229
:1097B0007F928F929F92AF92BF92CF92DF92EF9261
:1097C000FF920F931F93CF93DF93CDB7DEB7299707
:1097D0000FB6F894DEBF0FBECDBF3C0181E00F9401
:1097E000CD148F8382E06816710408F081C2F30102
:1097F000EB5EF14FE491D301AA0FBB1FAA0FBB1F71
:10980000BA83A983A65ABD4FBE83AD838D919D9126
:109810000D90BC91A02D80930E0290930F02A09307
:109820001002B093110281E0062C01C0880F0A9447
:10983000EAF70F947536E981FA81EA5CF64FF98709
:10984000E8871082118212821382E0903E09F09024
:109850003F09009140091091410920913A09309146
:109860003B0940913C0950913D0960913609709146
:1098700037098091380990913909E2E4CE2EE9E068
:10988000DE2E0F949811E981FA81EF5FF64F2F01D8
:1098900080E090E0A0E4B0E480839183A283B3836E
:1098A00020E030E040E752E460910E0270910F0238
:1098B00080911002909111020F94EFBE4B015C0158
:1098C000E0900909F0900A0900910B0910910C0928
:1098D0002091050930910609409107095091080926
:1098E0006091010970910209809103099091040926
:1098F000F2E22F2EF9E03F2E3F922F92ADE0CA2EDA
:10990000A9E0DA2E0F9428060F94891C0F94B51441
:1099100080E00F94CD14A885B9851D921D921D92EB
:109920001C921397E0903E09F0903F090091400986
:109930001091410920913A0930913B0940913C092D
:1099400050913D096091360970913709809138092D
:1099500090913909B2E4CB2EB9E0DB2E0F94981127
:1099600080E090E0A0E8BFEBF20180839183A283C6
:10997000B38320E030E040E752E460910E02709142
:109980000F0280911002909111020F94EFBE4B01D3
:109990005C01E0900909F0900A0900910B0910910F
:1099A0000C09209105093091060940910709509151
:1099B0000809609101097091020980910309909151
:1099C00004093F922F92EDE0CE2EE9E0DE2E0F94B7
:1099D00028060F94891C81E00F94CD1489819A8107
:1099E0008C5D914F0E9406422DEC3CEC4CE85FEB05
:1099F0000F94BDC1D2016D937D938D939C9313976A
:109A000020E030E040E752E460910E0270910F02D6
:109A100080911002909111020F94EFBE4B015C01F6
:109A2000E0900909F0900A0900910B0910910C09C6
:109A300020910509309106094091070950910809C4
:109A400060910109709102098091030990910409C4
:109A50003F922F920F9428060F94891C0F94B514EF
:109A600080E00F94CD14E885F9851082118212826E
:109A70001382E0903E09F0903F0900914009109157
:109A8000410920913A0930913B0940913C0950919C
:109A90003D0960913609709137098091380990919C
:109AA0003909F2E4CF2EF9E0DF2E0F94981180E00F
:109AB00090E0A0E2B1E4F20180839183A283B383BA
:109AC00020E030E040E752E460910E0270910F0216
:109AD00080911002909111020F94EFBE4B015C0136
:109AE000E0900909F0900A0900910B0910910C0906
:109AF0002091050930910609409107095091080904
:109B00006091010970910209809103099091040903
:109B10003F922F92ADE0CA2EA9E0DA2E0F942806CC
:109B20000F94891C0F94B51481E00F94CD1480E03C
:109B300090E0A0E7B1ECF20180839183A283B3832C
:109B400020E030E040E05FE3AD81BE816D917D912A
:109B50008D919C910F94BDC160930E0270930F0282
:109B6000809310029093110220E030E040E752E42D
:109B70000F94EFBE4B015C01E0900909F0900A09D7
:109B800000910B0910910C092091050930910609EB
:109B900040910709509108096091010970910209EB
:109BA00080910309909104093F922F920F94280607
:109BB0000F94891CC3010E940C42F301E95DF64F2A
:109BC00081E080830F94D4360F94B51480E00F9415
:109BD000CD142AE037ED43E25FE3E885F985608143
:109BE0007181828193810F940EBEA885B9856D9392
:109BF0007D938D939C931397E0903E09F0903F09DD
:109C0000009140091091410920913A0930913B0996
:109C100040913C0950913D09609136097091370996
:109C20008091380990913909B2E4CB2EB9E0DB2E4E
:109C30000F9498112AE037ED43E25FE3E885F98558
:109C400060817181828193810F940FBEA885B9854F
:109C50006D937D938D939C931397F2016083718331
:109C6000828393832AE939E949E95EE360910E0230
:109C700070910F0280911002909111020F94BDC15A
:109C800020E030E040E752E40F94EFBE4B015C016E
:109C9000E0900909F0900A0900910B0910910C0954
:109CA0002091050930910609409107095091080952
:109CB0006091010970910209809103099091040952
:109CC0003F922F92EDE0CE2EE9E0DE2E0F94280693
:109CD0000F94891C10920E0210920F021092100223
:109CE000109211020FB6F894DEBF0FBECDBF62C155
:109CF00092E06916710409F05DC1E7E1FEE074903D
:109D000010923E0910923F091092400910924109A9
:109D100020913A0930913B0940913C0950913D090D
:109D2000609136097091370980913809909139090D
:109D3000F2E4CF2EF9E0DF2EE12CF12C87010F9415
:109D400098118CE29EE00E9406424B015C01672D57
:109D5000772767FD7095872F972F0F948ABF2B0168
:109D60003C0120E030E040EC5FE3C501B4010F941A
:109D7000BDC1A30192010F94BDC169837A838B8316
:109D80009C836093090970930A0980930B0990934F
:109D90000C0960916202709163028091640290915B
:109DA000650260930E0270930F02809310029093ED
:109DB000110220E030E040E752E40F94EFBE4B0187
:109DC0005C012091050930910609409107095091E5
:109DD000080960910109709102098091030990912D
:109DE0000409A2E22A2EA9E03A2E3F922F92BDE06A
:109DF000CB2EB9E0DB2EE980FA800B811C810F9419
:109E000028060F94891C10923E0910923F09109267
:109E100040091092410920913A0930913B09409143
:109E20003C0950913D096091360970913709809144
:109E300038099091390912E4C12E19E0D12EE12C94
:109E4000F12C87010F94981180E29EE00E94064257
:109E50009058A30192010F94BDC169837A838B83CB
:109E60009C836093090970930A0980930B0990936E
:109E70000C0920E030E040E752E460910E0270915E
:109E80000F0280911002909111020F94EFBE4B01CE
:109E90005C01209105093091060940910709509114
:109EA000080960910109709102098091030990915C
:109EB00004093F922F920DE0C02E09E0D02EE980D8
:109EC000FA800B811C810F9428060F94891C80E274
:109ED0009EE00E9406429B01AC010F940FBEA301BD
:109EE00092010F94BDC12B013C016093090970934D
:109EF0000A0980930B0990930C0920E030E040E0C0
:109F00005FE36091620270916302809164029091BC
:109F100065020F94BDC160930E0270930F0280938F
:109F200010029093110220E030E040E752E40F94D9
:109F3000EFBE4B015C01209105093091060940916B
:109F400007095091080960910109709102098091F7
:109F50000309909104093F922F92830172010F949B
:109F600028060F94891C82E090E00E940C428091A8
:109F70003E0990913F09A0914009B0914109809319
:109F8000090990930A09A0930B09B0930C09109248
:109F90000E0210920F0210921002109211020F94F2
:109FA000B51481E0809329090F900F900F900F90C6
:109FB0000F900F908F8129960FB6F894DEBF0FBED9
:109FC000CDBFDF91CF911F910F91FF90EF90DF9068
:109FD000CF90BF90AF909F908F907F906F905F9049
:109FE0004F903F902F900D94CD14CF92DF92EF922F
:109FF000FF920F931F934FDA80E090E0D4DB81E073
:10A0000090E0D1DBE0903E09F0903F0900914009DB
:10A010001091410920913A0930913B0940913C0946
:10A0200050913D0960913609709137098091380946
:10A0300090913909F2E4CF2EF9E0DF2E0F949811B8
:10A040001F910F91FF90EF90DF90CF900D94B5147A
:10A050000F9411B66093E8087093E9088093EA08BA
:10A060009093EB08089520E030E0A90168EB71E0DF
:10A0700084E50F9469BA69E170E080E090E00F94A4
:10A0800040B684E50F948DBD64E170E080E090E01F
:10A090000D9440B68F929F92AF92BF92CF92DF9273
:10A0A000EF92FF920F931F93CF93DF9300D01F92F5
:10A0B000CDB7DEB71092BD181092BC181092BB1825
:10A0C0001092BA180F943D4888EF9CE00F946D5B96
:10A0D0008E010F5F1F4F7E0125E0E20EF11C84ED23
:10A0E00097E00E943F408F3FEFEF9E07C1F3F801DA
:10A0F00081938F01EE15FF0591F789809A80AB80DF
:10A10000BC808BE20E94F942C12CD12C7601809157
:10A110008509882309F447C006E718E0C814D90464
:10A12000EA04FB04A1F084ED97E00E943F408F3FDA
:10A13000FFEF9F07C1F32FEFC21AD20AE20AF20A19
:10A14000F80181938F01F8E0063B1F0739F766E7B6
:10A1500078E080EC99E00E9474B88BE20E94F942AA
:10A160000F941B29C814D904EA04FB0481F67BDF91
:10A1700060E080EC99E00E94A5B810928509EEE7B6
:10A18000FAE4E590F490F7018491882331F00E947D
:10A19000F942FFEFEF1AFF0AF6CF8AE00E94F94278
:10A1A00080E090E000C00F900F900F900F90DF9133
:10A1B000CF911F910F91FF90EF90DF90CF90BF90C4
:10A1C000AF909F908F900895CF93C82F8FEF9FE00F
:10A1D0000F9423CB8130C1F40F94891CF89491E043
:10A1E0009C27909318190F94AC37B19A1092850060
:10A1F0001092840080ED97E090938900809388000E
:10A200007894CF910D943C1ECF9108952F923F9258
:10A210004F925F926F927F928F929F92AF92BF9276
:10A22000CF92DF92EF92FF920F931F93CF93DF9322
:10A2300000D01F921F92CDB7DEB7382E81E0C4DF69
:10A24000311012C01092BB181092BA181092BD189B
:10A250001092BC181092BF181092BE181092C1181C
:10A260001092C0180F94A24880E00F94CD878BE421
:10A2700091E10E9481FA0E94B0DC0E94D2F9109212
:10A280002709109228091092290981E00E946E4244
:10A29000EEE7FBE4859194910E94E046A6DE80E023
:10A2A0000F94CD1420E030E040EA50E4609136098C
:10A2B0007091370980913809909139090F940FBE38
:10A2C0002B013C016093360970933709809338095C
:10A2D0009093390920E030E040EA50E460913A0977
:10A2E00070913B0980913C0990913D090F940FBEFC
:10A2F0006A837B838C839D8360933A0970933B09C7
:10A3000080933C0990933D0920E030E040E252E424
:10A310006091620270916302809164029091650283
:10A320000F94EFBE4B015C01E0903E09F0903F09B5
:10A33000009140091091410982E299E09F938F9327
:10A3400022E4C22E29E0D22E2A813B814C815D81FC
:10A35000C301B2010F9428060F94891CC8D80F902E
:10A360000F90882309F4A3C173DE311058C084E034
:10A3700090E09093180280931702E0918609F0E034
:10A38000EE0FFF1FE25DF74B8591949140E060E096
:10A390000F94DA8A882359F0E0918609F0E0EE0FF5
:10A3A000FF1FE65DF64B859194910F949C95E0918B
:10A3B0008609F0E0EE0FFF1FEA50F54B859194916E
:10A3C0000F949C95E0918609F0E0EE0FFF1FE45793
:10A3D000F64B859194910F949C9582E090E0909338
:10A3E000180280931702E0918609F0E0EE0FFF1F3C
:10A3F000EA58F54B859194910E94E04641E050E087
:10A4000062E080E00F944848E0918609F0E0EE0FAA
:10A41000FF1FEE58F54B859194910F946D5B80E092
:10A4200090E0A0EAB0E480933E0990933F09A093A6
:10A430004009B093410981E00F94CD14282E84E0A7
:10A440000F94753620E030E040E252E46091620201
:10A450007091630280916402909165020F94EFBE47
:10A460004B015C01E0903E09F0903F0900914009EA
:10A470001091410920913A0930913B0940913C09E2
:10A4800050913D09609136097091370980913809E2
:10A4900090913909E2E2F9E0FF93EF93E2E4CE2EE6
:10A4A000E9E0DE2E0F9428060F94891C0F94D43611
:10A4B000822D0F94CD1482E00F94F81C0F900F9012
:10A4C00020E030E040EA50E40F94E8BE8111EBC098
:10A4D00086E50E94C242882361F0E091020FF0916C
:10A4E000030F8181893039F08F7D41F00E94D8427D
:10A4F00003C01A8205C081E08A8302C091E09A837A
:10A500003320B1F00E949C420E9405DD0E9457DE7C
:10A510000E942FF3882309F4C0C087EF9FE00F94B7
:10A5200023CB803F09F0BBC081E00E94EE46B7C05C
:10A530008AEF0E94EE4660E070E088EF9FE00F94A3
:10A540004FCB1982BE016F5F7F4F8A810E94FCEF63
:10A550003C010E949C42212C312CB0EA4B2EB0E4ED
:10A560005B2E20923E0930923F0940924009509262
:10A57000410920E030E040E252E4609162027091D3
:10A58000630280916402909165020F94EFBE4B01CB
:10A590005C0120913A0930913B0940913C0950916E
:10A5A0003D09609136097091370980913809909181
:10A5B0003909A2E2B9E0BF93AF9312E4C12E19E0CA
:10A5C000D12E820171010F9428060F94891C0F90DF
:10A5D0000F9077FC47C019828BE491E10E9481FAC9
:10A5E0000E9477DC81E00E946E42FFDCAE014F5F8B
:10A5F0005F4F6A8181E00E9451F53C010E949C42BC
:10A6000020923E0930923F09409240095092410900
:10A6100020E030E040E252E4609162027091630217
:10A6200080916402909165020F94EFBE4B015C0132
:10A6300020913A0930913B0940913C0950913D09E4
:10A6400060913609709137098091380990913909E4
:10A65000A2E2B9E0BF93AF930F9428060F94891C30
:10A660000F900F906981C3010F94B3A677FC15C0BA
:10A6700086EE0E94EE468FE59FE00F9423CB81305B
:10A6800071F0E0918609F0E0EE0FFF1FEC58F44BFB
:10A69000859194910F949C9502C010E001C011E047
:10A6A0000F94D43605C083E59CE00F949C9510E090
:10A6B00081E00F94CD8780E087DD812F0F900F9090
:10A6C0000F900F900F90DF91CF911F910F91FF90FE
:10A6D000EF90DF90CF90BF90AF909F908F907F9042
:10A6E0006F905F904F903F902F900895CF93DF939E
:10A6F00084ED97E00E945B40E8E2F9E4C591D491D3
:10A70000FE018491882321F00E94F9422196F8CF1E
:10A710004091F20E5091F30E6091F40E7091F50E8F
:10A720004F5F5F4F6F4F7F4F2AE030E084ED97E03F
:10A730000E941A418AE00E94F9420F9411B6609378
:10A74000E8087093E9088093EA089093EB08E0E941
:10A75000F9E4C591D491FE018491882321F00E94EF
:10A76000F9422196F8CF8AE0DF91CF910C94F9421B
:10A77000CF93DF930F9411B66093E8087093E908C4
:10A780008093EA089093EB08E0910C0FF0910D0F85
:10A79000E25FF04F8081813089F4E0E9F9E4C5910E
:10A7A000D491FE018491882321F00E94F9422196E0
:10A7B000F8CF8AE0DF91CF910C94F942DF91CF91ED
:10A7C00008958F929F92AF92BF92CF92DF92EF92B5
:10A7D000FF920F931F93CF93DF933FEEE32E34E06E
:10A7E000F32E06E319E0C1E0D9E048EBC42E49E0BE
:10A7F000D42EF70181917F010E94C242882319F172
:10A800000E94F0424B015C01F6018081811103C07E
:10A810006091EC0801C061E070E080E090E00F948E
:10A820008ABFF80120813181428153810F94BDC1DB
:10A830009B01AC01C501B4010F940FBE68837983FD
:10A840008A839B8309C0F80180819181A281B381B1
:10A8500088839983AA83BB830C5F1F4F2496FFEFE5
:10A86000CF1ADF0A83EFE81684E0F80611F686E4D3
:10A870000E94C2428823D9F00E94F0426B017C0101
:10A880006093F1087093F2088093F3089093F408B2
:10A8900020E030E0A9010F94EBC0181644F4C092F8
:10A8A0000E02D0920F02E0921002F0921102DF919C
:10A8B000CF911F910F91FF90EF90DF90CF90BF90BD
:10A8C000AF909F908F9008957CDF89E40E94C242F0
:10A8D000882359F00E94F0426093F5087093F608BF
:10A8E0008093F7089093F80808C01092F50810922A
:10A8F000F6081092F7081092F8088AE40E94C24203
:10A90000882359F00E94F0426093F9087093FA0886
:10A910008093FB089093FC0808951092F908109218
:10A92000FA081092FB081092FC080895CF92DF926B
:10A93000EF92FF92CF93DF93EC01BC016C5F7F4FEE
:10A940000E94C94520E030E0A90160913E0270916B
:10A950003F0280914002909141020F940FBE6B0123
:10A960007C019B01AC01688579858A859B850F9464
:10A97000E8BE87FF04C0C886D986EA86FB86C090F9
:10A980003202D0903302E0903402F0903502A701F9
:10A990009601688579858A859B850F94EBC018168A
:10A9A00024F4C886D986EA86FB86DF91CF91FF9092
:10A9B000EF90DF90CF9008952F923F924F925F9249
:10A9C0006F927F928F929F92AF92BF92CF92DF92BF
:10A9D000EF92FF920F931F93CF93DF93CDB7DEB724
:10A9E000AB970FB6F894DEBF0FBECDBF9F878E87A3
:10A9F000798B688B5B8B4A8B3D8B2C8B1F8B0E8BE3
:10AA0000ED82DC018D909D90AD90BC904090360918
:10AA1000509037096090380970903909DB018D91A9
:10AA20009D910D90BC91A02D88879987AA87BB879F
:10AA3000C0903A09D0903B09E0903C09F0903D0964
:10AA400020913E0930913F094091400950914109C0
:10AA5000EA89FB8960817181828193810F940EBEA6
:10AA6000688F798F8A8F9B8F80914B11811173C072
:10AA7000AE89BF898D909D90AD90BC90EA89FB898D
:10AA8000E080F18002811381A889B9892D913D91DF
:10AA90004D915C91EE85FF8560817181828193810A
:10AAA000FE013596FF93EF93CC88DD880F9428063E
:10AAB000EE85FF8580819181A281B38180933609E3
:10AAC00090933709A0933809B0933909E889F98937
:10AAD00080819181A281B38180933A0990933B094F
:10AAE000A0933C09B0933D09EA89FB89808191815B
:10AAF000A281B38180933E0990933F09A0934009BE
:10AB0000B0934109EC89FD8980819181A281B38153
:10AB10008093420990934309A0934409B093450957
:10AB20000F900F90AB960FB6F894DEBF0FBECDBF5F
:10AB3000DF91CF911F910F91FF90EF90DF90CF9019
:10AB4000BF90AF909F908F907F906F905F904F904D
:10AB50003F902F900895A3019201C501B4010F9475
:10AB60000EBE2B013C0120E030E0A9010F94EBC0A8
:10AB700053014201181624F0B7FAB094B7F8B09414
:10AB8000A7019601688579858A859B850F940EBEFD
:10AB9000688779878A879B8720E030E0A9010F9436
:10ABA000EBC0288539854A855B8518160CF050580E
:10ABB000C501B4010F940FBE6B017C0120E030E0B1
:10ABC000A9010F94EBC018160CF052CF20E030E032
:10ABD00040EF51E4C701B6010F94EFBE0F94D5BE0C
:10ABE0000F9457BF7D876C87623071050CF440CF9E
:10ABF00020914209309143094091440950914509FF
:10AC0000AC89BD896D917D918D919C910F940EBE03
:10AC10006C8F7D8F8E8F9F8F22242394312C8C8577
:10AC20009D85AA2797FDA095BA2F88A799A7AAA7BF
:10AC3000BBA7DE011596BF83AE83B101882777FDE0
:10AC40008095982F0F948ABF6B017C0168A579A528
:10AC50008AA59BA50F948ABF9B01AC01C701B601D1
:10AC60000F94EFBE6B017C01EE89FF89808091809B
:10AC7000A280B3802C8D3D8D4E8D5F8D0F94BDC114
:10AC80009B01AC0160914209709143098091440994
:10AC9000909145090F940FBE69837A838B839C83BF
:10ACA000288D398D4A8D5B8DC701B6010F94BDC1CA
:10ACB00020913E0930913F0940914009509141094E
:10ACC0000F940FBE68A379A38AA39BA32885398517
:10ACD0004A855B85C701B6010F94BDC120913A0931
:10ACE00030913B0940913C0950913D090F940FBEB2
:10ACF0006CA37DA38EA39FA3A3019201C701B601FC
:10AD00000F94BDC12091360930913709409138091F
:10AD1000509139090F940FBEFF81FF932E812F931D
:10AD2000DE0111966D01E8A0F9A00AA11BA12CA1DA
:10AD30003DA14EA15FA10F942806BFEF2B1A3B0A3D
:10AD40000F900F90EC85FD852E163F0609F075CF0C
:10AD50008FCE4F925F926F927F928F929F92AF921F
:10AD6000BF92CF92DF92EF92FF920F931F93CF93F8
:10AD7000DF93CDB7DEB728970FB6F894DEBF0FBECE
:10AD8000CDBF81E099E0D2DD0F9411B66093E80861
:10AD90007093E9088093EA089093EB088091010989
:10ADA00090910209A0910309B09104098D839E83BB
:10ADB000AF83B8879C01AD01609136097091370966
:10ADC00080913809909139090F94E8BE811197C09C
:10ADD0004090050950900609609007097090080995
:10ADE000A301920160913A0970913B0980913C095D
:10ADF00090913D090F94E8BE811181C020E030E0C0
:10AE000040E752E460910E0270910F0280911002AF
:10AE1000909111020F94EFBE4B015C01E090090983
:10AE2000F0900A0900910B0910910C0982E299E057
:10AE30009F938F936DE0C62E69E0D62EA3019201F9
:10AE40006D817E818F8198850F9428060F900F90D9
:10AE50008091010990910209A0910309B091040920
:10AE60008093360990933709A0933809B093390934
:10AE70008091050990910609A0910709B0910809F0
:10AE800080933A0990933B09A0933C09B0933D0904
:10AE90008091090990910A09A0910B09B0910C09C0
:10AEA00080933E0990933F09A0934009B0934109D4
:10AEB00080910D0990910E09A0910F09B091100990
:10AEC0008093420990934309A0934409B0934509A4
:10AED00028960FB6F894DEBF0FBECDBFDF91CF919D
:10AEE0001F910F91FF90EF90DF90CF90BF90AF90A8
:10AEF0009F908F907F906F905F904F900895E0901B
:10AF000022096091580270915902882777FD809537
:10AF1000982F0F948ABF20910E0230910F0240911A
:10AF20001002509111020F94BDC12EE333EC4EE29A
:10AF300059E30F94BDC169837A838B839C838E010F
:10AF40000F5F1F4F2DE039E049E059E065E079E0FF
:10AF500081E099E031DD7CCF4F925F926F927F92DA
:10AF60008F929F92AF92BF92CF92DF92EF92FF9219
:10AF70000F931F93CF93C62FE0912209F0E088230F
:10AF800009F4D9C0DF01A25EB64F8C918111AFC127
:10AF90008091360990913709A0913809B09139090B
:10AFA0008093010990930209A0930309B0930409C7
:10AFB00080913A0990913B09A0913C09B0913D09DB
:10AFC0008093050990930609A0930709B093080997
:10AFD00080913E0990913F09A0914009B0914109AB
:10AFE0008093090990930A09A0930B09B0930C0967
:10AFF000C0904209D0904309E0904409F09045097F
:10B00000C0920D09D0920E09E0920F09F09210093A
:10B01000EE0FFF1FEE0FFF1FEE5BFD4F2081318112
:10B0200042815381662349F060912202709123028C
:10B03000809124029091250208C0609126027091AF
:10B04000270280912802909129020F94EFBE9B0164
:10B05000AC01C701B6010F940FBE60934209709313
:10B060004309809344099093450982E499E00F9441
:10B070000D1380900E0290900F02A0901002B090DD
:10B08000110220E030E040E752E460911E0270912E
:10B090001F0280912002909121020F94BDC1609304
:10B0A0000E0270930F028093100290931102E091B0
:10B0B0002209F0E0E25EF64F81E080834ADE2091D3
:10B0C0001A0930911B0940911C0950911D0960918A
:10B0D0003E0970913F0980914009909141090F9478
:10B0E0000EBE7B018C0160933E0970933F098093F3
:10B0F00040099093410920913A0930913B094091D0
:10B100003C0950913D096091360970913709809151
:10B11000380990913909E2E4CE2EE9E0DE2E0F9451
:10B12000981117DE80920E0290920F02A0921002E8
:10B13000B0921102DCC0E25EF64F8081882309F4F0
:10B14000D6C08090360990903709A0903809B09009
:10B1500039098092010990920209A0920309B092E4
:10B16000040940903A0950903B0960903C09709066
:10B170003D094092050950920609609207097092B4
:10B18000080960913E0970913F09809140099091B2
:10B1900041096093090970930A0980930B09909300
:10B1A0000C09009142091091430920914409309102
:10B1B000450900930D0910930E0920930F09309350
:10B1C000100920911A0930911B0940911C095091D6
:10B1D0001D090F940FBE7B018C0160933E09709393
:10B1E0003F09809340099093410972E4C72E79E0AA
:10B1F000D72EA3019201C501B4010F9498111091AB
:10B200002209CC2389F02091120930911309409131
:10B2100014095091150960912202709123028091C6
:10B2200024029091250210C020911609309117092F
:10B2300040911809509119096091260270912702D6
:10B2400080912802909129020F940FBE24E0129F52
:10B25000F0011124EE5BFD4F208131814281538149
:10B260000F94EFBE9B01AC016091420970914309BC
:10B2700080914409909145090F940EBE6093420954
:10B2800070934309809344099093450982E499E0BF
:10B290000F940D13C0900E02D0900F02E090100298
:10B2A000F090110220E030E040E752E460911A0291
:10B2B00070911B0280911C0290911D020F94BDC1E0
:10B2C00060930E0270930F0280931002909311020C
:10B2D000E0912209F0E0E25EF64F10823ADDC09282
:10B2E0000E02D0920F02E0921002F0921102CF9162
:10B2F0001F910F91FF90EF90DF90CF90BF90AF9094
:10B300009F908F907F906F905F904F900895AF9235
:10B31000BF92CF92DF92EF92FF920F931F93CF9342
:10B32000DF93D82F2091F9083091FA084091FB085B
:10B330005091FC086091F5087091F6088091F7082B
:10B340009091F8080F94F8C0C62F172F082FF92EE8
:10B350006091580270915902882777FD8095982F47
:10B360000F948ABF20910E0230910F02409110027B
:10B37000509111020F94BDC120E030E040E752E44B
:10B380000F94EFBE20E030E048EC52E40F94EFBEA3
:10B39000209122092F93DF93FF920F931F93CF9356
:10B3A0005B016C01B2E0EB2E01E020E045EF58E0DC
:10B3B00061E079E086E399E00E9466FC80910109F2
:10B3C00090910209A0910309B09104098093360974
:10B3D00090933709A0933809B093390980910509F2
:10B3E00090910609A0910709B091080980933A0944
:10B3F00090933B09A0933C09B0933D0980910909C2
:10B4000090910A09A0910B09B0910C0980933E0913
:10B4100090933F09A0934009B093410980910D0991
:10B4200090910E09A0910F09B091100980934209E3
:10B4300090934309A0934409B09345090F9411B622
:10B440006093E8087093E9088093EA089093EB080A
:10B450000F900F900F900F900F900F90DF91CF9162
:10B460001F910F91FF90EF90DF90CF90BF90AF9022
:10B470000895CF93DF931F92CDB7DEB77C01E1EE45
:10B48000F9E084918F01882349F069830E94F94291
:10B490000F5F1F4FF80184916981F5CF70E04AE09A
:10B4A00050E084ED97E00E944841F8940F944126C3
:10B4B000179A10922709169A10922809149AEAE509
:10B4C000FEE084918F01882339F00E94F9420F5FDA
:10B4D0001F4FF8018491F7CFE2EBFAE40591149144
:10B4E000F8018491882329F00E94F9420F5F1F4FD1
:10B4F000F7CF8AE00E94F942E114F10499F0F701D4
:10B5000084918701882339F00E94F9420F5F1F4F11
:10B51000F8018491F7CF8AE00E94F942C7010E94A6
:10B52000E04606C0E6E1FAE4859194910F94C249A1
:10B53000789406E010E00150110951F068EC70E0D9
:10B5400080E090E00F9440B680E00F94FF84F3CF4A
:10B55000F894A895FECFCF93DF930F944126809166
:10B56000D608811136C081E08093D6088091F20E12
:10B570009091F30EA091F40EB091F50E8093EE0E23
:10B580009093EF0EA093F00EB093F10EEAE5FEE07B
:10B590008491EF01882331F00E94F9422196FE0147
:10B5A0008491F8CFE8EAFAE4C591D491FE01849140
:10B5B000882321F00E94F9422196F8CF8AE00E9468
:10B5C000F942EAE2F8E485919491DF91CF910D94EC
:10B5D0009649DF91CF9108958091D6080895FF9202
:10B5E0000F931F93CF93DF93EC01809122098093F7
:10B5F000D70884E50E94C242811102C080E06AC07F
:10B600000E94F0420F945CBFF62E6093D708662329
:10B61000A9F3E4E5FEE084918F01882339F00E94CC
:10B62000F9420F5F1F4FF8018491F7CFCD36D10556
:10B6300059F164F4C836D105A9F0C936D10509F02D
:10B640003DC0E6EFF9E4C591D49118C0CA3DD105DB
:10B6500029F1CD3DD10509F031C0E6EEF9E4C591FF
:10B66000D49126C0E8EFF9E4C591D491FE0184910C
:10B67000882321F10E94F9422196F8CF89918823ED
:10B68000E9F00E94F942FACFE4EFF9E4C591D491D0
:10B690008991882399F00E94F942FACFE8EEF9E403
:10B6A000C591D4918991882349F00E94F942FACF3B
:10B6B0008991882319F00E94F942FACF6F2D70E02A
:10B6C0004AE050E084ED97E00E942C418AE00E941D
:10B6D000F94281E0DF91CF911F910F91FF90089582
:10B6E0004F925F926F927F928F929F92AF92BF9292
:10B6F000CF92DF92EF92FF92CF93DF9300D01F9211
:10B70000CDB7DEB72B013C0129833A834B835C83A1
:10B710008DEE9FE00F9423CB8F3F01F58EEE9FE0DF
:10B720000F9423CB8F3FD1F48FEE9FE00F9423CB68
:10B730008F3FA1F480EF9FE00F9423CB8F3F71F4F4
:10B7400040E050E0BA018DEE9FE00F9447CB40E01F
:10B7500050E0BA0181EF9FE00F9447CB81EF9FE06B
:10B760000F942BCB4B015C018DEE9FE00F942BCB04
:10B770006B017C0169817A818B819C812CE330E0B3
:10B7800040E050E00F94BFC3C20ED31EE41EF51E6E
:10B79000B701A6018DEE9FE00F9447CBC301B20124
:10B7A00028EE33E040E050E00F94BFC3BA01A90196
:10B7B000480D591D6A1D7B1D81EF9FE00F9447CBFB
:10B7C00010927F09109280091092810910928209CB
:10B7D0000F900F900F900F90DF91CF91FF90EF900F
:10B7E000DF90CF90BF90AF909F908F907F906F90A1
:10B7F0005F904F900895CF92DF92EF92FF92209149
:10B8000046092223F1F020E030E040E05FE30F94AE
:10B81000BDC16B017C0120E030E0A9010F94E8BEBE
:10B82000882379F0A7019601C701B6010F94BDC125
:10B830002BED3FE049E450E40F94BDC19B01AC0106
:10B8400004C020E030E040E85FE360E070E080E8C2
:10B850009FE30F94EFBEFF90EF90DF90CF9008959D
:10B86000609146027091470280914802909149028E
:10B87000C2DF60934202709343028093440290932C
:10B8800045020895CF93DF93EC010F941B2981E0CB
:10B890005FD180E00F94FF84209799F0C233D105E7
:10B8A00040F062E370E080E090E00F9440B6E297F1
:10B8B000ECCFBE0180E090E00F9440B6C0E0D0E055
:10B8C000E4CFDF91CF9108958F929F92AF92BF9274
:10B8D000CF92DF92EF92FF920F931F93CF93DF935C
:10B8E000159881E080937A0982E090E0909378093E
:10B8F00080937709E0918609F0E0EE0FFF1FEE5F7D
:10B90000F54B859194910F94964920E030E04CE8F6
:10B9100052E46091420970914309809144099091E9
:10B9200045090F940FBE60934209709343098093B9
:10B93000440990934509E0903E09F0903F09009139
:10B9400040091091410920913A0930913B094091F9
:10B950003C0950913D0960913609709137098091F9
:10B96000380990913909C2E2D9E0DF93CF93812C55
:10B97000912CE0ECAE2EE0E4BE2EF2E4CF2EF9E006
:10B98000DF2E0F94280620E030E048EC51E460916F
:10B9900042097091430980914409909145090F949F
:10B9A0000FBE6093420970934309809344099093BA
:10B9B0004509E0903E09F0903F090091400910913F
:10B9C000410920913A0930913B0940913C0950913D
:10B9D0003D0960913609709137098091380990913D
:10B9E0003909DF93CF93812C912CA0E8AA2EAFE3E5
:10B9F000BA2E0F9428060F94891C20E030E0A9018C
:10BA000064EF71E084E50F9469BA82E390E03ADF75
:10BA100084E50F948DBD0F900F900F900F90809143
:10BA2000CB19882331F181E00F94CD8782E00F9408
:10BA3000FF84E0918609F0E0EE0FFF1FE658F84B17
:10BA4000859194910F9496491092790910927A09F0
:10BA50001092780910927709DF91CF911F910F9181
:10BA6000FF90EF90DF90CF90BF90AF909F908F901E
:10BA70000895809179098823B1F2E0918609F0E078
:10BA8000EE0FFF1FE257F54B8591949141E060E086
:10BA90000F94DA8A91E0811101C090E0C2E2D9E00E
:10BAA0009111C1CF81E00F94CD8782E00F94FF8484
:10BAB00020E030E048EC51E4609142097091430984
:10BAC00080914409909145090F940FBE60934209FB
:10BAD000709343098093440990934509E0903E098F
:10BAE000F0903F09009140091091410920913A09D5
:10BAF00030913B0940913C0950913D0960913609D4
:10BB0000709137098091380990913909DF93CF936B
:10BB1000812C912CE0E8AE2EEFE3BE2EF2E4CF2E86
:10BB2000F9E0DF2E0F9428060F94891CE091860916
:10BB3000F0E0EE0FFF1FE257F54B8591949141E045
:10BB400060E00F94DA8A0F900F9081116CCFAACF2A
:10BB5000CF92DF92EF92FF920F931F93CF93C82F54
:10BB600080916A02209104118823F1F080910602ED
:10BB70008823D1F080910811811116C080911E1286
:10BB800090911D12891B8F7079F48091C2098111E7
:10BB90000BC08091B509811107C08091CF19909198
:10BBA000D019089709F067C021110E949DCB8091A0
:10BBB000080F9091090F039714F40E94D5C50F94B4
:10BBC00011B60091E4081091E5082091E608309143
:10BBD000E708C090E808D090E908E090EA08F09003
:10BBE000EB086C197D098E099F09061717072807AE
:10BBF000390740F4012B022B032B21F064E087E48A
:10BC000095E037DC40910A0250910B0260910C02E2
:10BC100070910D02452B462B472B21F10F9411B645
:10BC20000091E8081091E9082091EA083091EB08AA
:10BC3000601B710B820B930B00910A0210910B0297
:10BC400020910C0230910D020617170728073907BB
:10BC500048F490911E1280911D12981303C0CC23BA
:10BC600009F470C0CF911F910F91FF90EF90DF907A
:10BC7000CF900D945604222309F461C00E94A4CBF6
:10BC8000882309F494CF20E030E04EE353E4609140
:10BC9000B4187091B5188091B6189091B7180F9498
:10BCA000EBC01816CCF40E949DCB20E030E0A90137
:10BCB00068EE73E084E50F9469BA82E390E0E2DD18
:10BCC00084E50F948DBD81E08093790961E088EE71
:10BCD00099E00E942DC56BCF80E00F94CD870F9423
:10BCE0003D4840E060E08AE499E10E945A3CE091DE
:10BCF0008609F0E0EE0FFF1FE854F54B8591949113
:10BD00000F946D5B42E060E08AE499E10E945A3C46
:10BD1000E0918609F0E0EE0FFF1FE45AF64B8591A3
:10BD200094910F946D5B60ED77E080E090E00F946C
:10BD300040B60F943D4881E00F94CD8738CF0E94E4
:10BD40007FCB35CF179A10922709169A109228099F
:10BD5000149A88CF2F923F924F925F926F927F9268
:10BD60008F929F92AF92BF92CF92DF92EF92FF920B
:10BD70000F931F93CF93DF934B015C01CC24CA94A4
:10BD8000DC2C76015AED252E59E0352E06ED19E012
:10BD900068EE462E63E0562E612C712C80911109BD
:10BDA000811112C12FEFC216D206E206F20651F03F
:10BDB000F7FC0AC10F9411B66C197D09683B7B40F2
:10BDC00008F002C10F9411B6681979098A099B0914
:10BDD000693E73408105910508F470C08091CB19CC
:10BDE000811168C0EEEDF9E08491EF01882331F014
:10BDF0000E94F9422196FE018491F8CFE091D70884
:10BE000024E0E29FF0011124EC54F74E408151816F
:10BE10006281738121E030E084ED97E00E94FD4172
:10BE2000F1018491CAEDD9E0882331F00E94F942F2
:10BE30002196FE018491F8CF6091D70870E04AE026
:10BE400050E084ED97E00E942C41F8018491C6ED0A
:10BE5000D9E0882331F00E94F9422196FE018491B5
:10BE6000F8CFF7FE03C0CDE1D7E01BC00F9411B6A9
:10BE70004B015C01C701B6016854744F8F4F9F4F4F
:10BE8000681979098A099B09A30192010F94BFC31C
:10BE9000BA01A9012AE030E084ED97E00E941A413E
:10BEA00006C08991882319F00E94F942FACF8AE0EE
:10BEB0000E94F9420F9411B64B015C010F941B29AB
:10BEC00080E046DE80E00F94FF84FFEFCF16DF06B0
:10BED000EF06FF0609F042C08091D508E091D7082F
:10BEE000F0E0EF01CC0FDD1FCC0FDD1FCC54D74E9F
:10BEF000EE0FFF1FE454F74E608171818823B9F083
:10BF0000882777FD8095982F0F948ABF20E030E036
:10BF100040E85FE30F940EBE9B01AC01688179811C
:10BF20008A819B810F94EBC087FF49C037CF882758
:10BF300077FD8095982F0F948ABF20E030E040E88D
:10BF40005FE30F940FBE9B01AC01688179818A8108
:10BF50009B810F94E8BE181694F520CFF7FC1ECFF6
:10BF6000E091D708F0E0EF01CC0FDD1FCC0FDD1F13
:10BF7000CC54D74EEE0FFF1FE454F74E6081718111
:10BF8000882777FD8095982F0F948ABF9B01AC017D
:10BF9000688179818A819B810F940EBE0F9457BF6F
:10BFA00097FF07C090958095709561957F4F8F4F53
:10BFB0009F4F66307105810591050CF4EFCE0F940B
:10BFC00011B66B017C01EACEDF91CF911F910F91E9
:10BFD000FF90EF90DF90CF90BF90AF909F908F90A9
:10BFE0007F906F905F904F903F902F9008950F93A8
:10BFF0001F93CF93DF931F921F92CDB7DEB7BE0181
:10C000006F5F7F4F88EF9FE00F948C4889819A8102
:10C010008156904F803A9F4000F11A821982EDEAD2
:10C02000F9E084918F01882339F00E94F9420F5F73
:10C030001F4FF8018491F7CF8AE00E94F942BE01B8
:10C040006F5F7F4F88EF9FE00F947B4880E799E018
:10C050000F949C9581E00F94CD870F900F90DF9106
:10C06000CF911F910F9108952F923F924F925F921F
:10C070006F927F928F929F92AF92BF92CF92DF92F8
:10C08000EF92FF920F931F93CF93DF93CDB7DEB75D
:10C09000CA58D2400FB6F894DEBF0FBECDBFC95804
:10C0A000DD4F688379838A839B83C757D240FE0123
:10C0B000E75FFD4F88E2DF011D928A95E9F7E850BE
:10C0C000F24080E991E0DF019C011D922150304057
:10C0D000E1F7C75ADD4F19821882C955D240CE0107
:10C0E000875A9D4F5C014E019FE6891A9EEF990A7F
:10C0F000DE01AF51BE4F3D0190EBC92E9FE0D92E1E
:10C1000023E2E22EF12C00E010E0C359DD4F8882DB
:10C11000CD56D240CD58DD4F9882C357D240B7019B
:10C12000882777FD8095982F0F948ABFD3016D9350
:10C130007D938D939D933D01F501619171915F0117
:10C14000882777FD8095982F0F948ABFD4016D932F
:10C150007D938D939D934D010F5F1F4F0630110509
:10C1600059F0B501C6010F948C48B5E0EB0EF11CF7
:10C17000E2E0CE0ED11CD3CFCF51DE4F28813981E2
:10C180004A815B81C15ED140C958DD4F68817981A8
:10C190008A819B81C757D2400F94E8BE87FD2BC38D
:10C1A000FE01EF51FE4F7F016E01FFE2CF1AFEEF5D
:10C1B000DF0A3E012BEB621A2DEF720AC359DD4FE5
:10C1C0000881CD56D240CD58DD4F1881C357D2409B
:10C1D00085E090E0CF58DD4F99838883C157D240E6
:10C1E000CF58DD4FA881B981C157D2401197CF58A0
:10C1F000DD4FB983A883C157D240F7012089318927
:10C200004289538964897589868997890F940EBEFE
:10C210004B015C01D80150962D913D914D915C915F
:10C22000539754966D917D918D919C9157970F9452
:10C230000EBEA50194010F94EFBEF6019293829376
:10C24000729362936F01D301BE92AE929E928E92D0
:10C250003D0104501109B4E0EB1AF108CF58DD4F4D
:10C26000E881F981C157D240EF2B09F0B9CF6E01B7
:10C27000FFECCF1AFDEFDF0A3E0127E4621A2EEF32
:10C28000720A2E013DE3430E511CCE0101967C0142
:10C2900001E010E0D6018D909D90AD90BC90139779
:10C2A00014962D913D914D915C911797C501B40164
:10C2B0000F940FBE9B01AC010F940FBEF70164A752
:10C2C00075A786A797A70130110541F080A691A612
:10C2D000A2A6B3A684829582A682B7820F5F1F4F63
:10C2E000D30114962D913D914D915C91179718961D
:10C2F0006D917D918D919C911B970F940EBE20E0C6
:10C3000030E040EC50E40F94BDC1F20160837183D2
:10C3100082839383F4E0CF0ED11C2CE2E20EF11C59
:10C3200034E0630E711C88E2480E511C0530110583
:10C3300009F0B0CF8E010B5A1F4F6E0191E5C90E67
:10C34000D11C22242394312C2C0E3D1EA8ED2A0E44
:10C35000311CF801B8972081318142815381F80165
:10C3600060817181828193810F94EFBE4B015C01EA
:10C37000E12CF12C3601F8E26F1A710826014E0CFF
:10C380005F1CF301EE0DFF1D24813581468157812D
:10C39000C501B4010F94BDC19B01AC01D20114963B
:10C3A0006D917D918D919C9117970F940EBEF20126
:10C3B0006483758386839783F4E0EF0EF11C24E198
:10C3C000E216F104D9F6045D1F4F38E2C30ED11C0A
:10C3D0000215130509F0BDCF1E0185EB280E311C97
:10C3E0006E0191EBC90ED11C3E01A7EE6A1AADEFAA
:10C3F0007A0A14E0E12EF12C270100E010E0812CF4
:10C40000912CA12CB12CF601E00FF11FD301A00F4C
:10C41000B11F2D913D914D915C916081718182811F
:10C4200093810F94BDC19B01AC01B401C5010F9470
:10C430000FBE4B015C01BFEF4B1A5B0A0C5F1F4F35
:10C44000E5E04E165104F9F69B01AC01D1016D9166
:10C450007D918D919C910F940EBEF60120813181CA
:10C46000428153810F94EFBED3016D937D938D93E1
:10C470009C931397B1E0EB1AF108E8E22E1A310809
:10C48000FCE2CF1AD10824E0621A7108E114F10429
:10C4900009F0B2CFCB50DE4F88819981AA81BB8150
:10C4A000C55FD140C957DD4F88839983AA83BB8379
:10C4B000C758D2408E01075F1D4FDE01AF5CBD4FF4
:10C4C000C558DD4FB983A883CB57D240C359DD4F40
:10C4D0002880CD56D240CD58DD4F3880C357D2404A
:10C4E000FE01EF51FE4FC358DD4FF983E883CD576E
:10C4F000D240C358DD4FA881B981CD57D240CD90ED
:10C50000DD90ED90FD90C358DD4FB983A883CD57E2
:10C51000D240C958DD4F288139814A815B81C75794
:10C52000D240C701B6010F94E8BE1816B4F0C35844
:10C53000DD4FE881F981CD57D240208131814281A0
:10C540005381C958DD4F688179818A819B81C757A2
:10C55000D2400F94E8BE1816FCF4CF58DD4F288166
:10C560003981C157D2402430310509F01FC1C95764
:10C57000DD4F288139814A815B81C758D240C95833
:10C58000DD4F688179818A819B81C757D2400F94A2
:10C59000EBC018160CF00AC1D80114968D919D912C
:10C5A0000D90BC91A02DC158DD4F88839983AA833B
:10C5B000BB83CF57D240F8014080518062807380A6
:10C5C000C558DD4FA881B981CB57D2408D919D913F
:10C5D0000D90BC91A02DC359DD4F88839983AA8308
:10C5E000BB83CD56D240D1018D919D910D90BC91D0
:10C5F000A02DCD57DD4F88839983AA83BB83C35871
:10C60000D240A7019601C958DD4F688179818A819E
:10C610009B81C757D2400F940EBECD58DD4F688323
:10C6200079838A839B83C357D24020E030E040E483
:10C6300050E40F9420C26B017C01A3019201C15808
:10C64000DD4F688179818A819B81CF57D2400F94D9
:10C650000EBE4B015C0120E030E040EC50E4C359D9
:10C66000DD4F688179818A819B81CD56D2400F94BC
:10C67000BDC19B01AC01C501B4010F94EFBEA70180
:10C6800096010F94BDC16B017C0120E030E040E0D9
:10C690005FE3C301B2010F94BDC14B015C01CD58F2
:10C6A000DD4F288139814A815B81C357D240CA015D
:10C6B000B9010F94BDC19B01AC01C501B4010F9438
:10C6C000BDC19B01AC01C701B6010F940FBE6B0148
:10C6D0007C01CD57DD4F288139814A815B81C35868
:10C6E000D240F10164817581868197810F940EBEDD
:10C6F000C359DD4F288139814A815B81CD56D240B3
:10C700000F94EFBE4B015C01C359DD4F2881398185
:10C710004A815B81CD56D240CA01B9010F940FBE48
:10C72000A30192010F94BDC12B013C01C359DD4F00
:10C73000288139814A815B81CD56D240C158DD4F75
:10C74000688179818A819B81CF57D2400F94BDC186
:10C750009B01AC01C301B2010F940FBE20E030E099
:10C7600040EC50E40F94EFBE9B01AC01C501B40155
:10C770000F940EBECD58DD4F288139814A815B81EF
:10C78000C357D2400F94BDC19B01AC01C701B60194
:10C790000F940FBECD57DD4F288139814A815B81CF
:10C7A000C358D2400F940FBE4B015C01CF58DD4FF0
:10C7B00028813981C157D2402F5F3F4FCF58DD4F7D
:10C7C00039832883C157D2400C5F1F4FC558DD4FB6
:10C7D00088819981CB57D2400496C558DD4F998303
:10C7E0008883CB57D24094E0290E311C2530310587
:10C7F00009F07FCE04C0812C912CA12CB12CB40166
:10C80000C501C657DD4F0FB6F894DEBF0FBECDBFD2
:10C81000DF91CF911F910F91FF90EF90DF90CF901C
:10C82000BF90AF909F908F907F906F905F904F9050
:10C830003F902F900895CF92DF92EF92FF926B017D
:10C840007C018091B3098823A1F086EA9FE00F94D0
:10C8500023CB882371F0C701B60106DC2091B21703
:10C860003091B3174091B4175091B5170F94EFBEA4
:10C8700003C060E070E0CB01FF90EF90DF90CF90BD
:10C8800008954F925F926F927F928F929F92AF9294
:10C89000BF92CF92DF92EF92FF920F931F93CF93AD
:10C8A000DF93CDB7DEB728970FB6F894DEBF0FBE83
:10C8B000CDBF0F94891C809158029091590290939A
:10C8C000B7098093B609E0912209F0E0EE0FFF1F4F
:10C8D000E454F74E60817181882777FD8095982F09
:10C8E0000F948ABF6093A7097093A8098093A90940
:10C8F0009093AA0980912009909121099093A6090B
:10C900008093A5090F9411B660938D0970938E09D9
:10C9100080938F09909390098091360990913709FF
:10C92000A0913809B091390989839A83AB83BC837C
:10C930008093950990939609A0939709B0939809CD
:10C9400040903A0950903B0960903C0970903D0935
:10C950004092990950929A0960929B0970929C09A1
:10C9600080913E0990913F09A0914009B091410901
:10C970008D839E83AF83B88780939D0990939E0992
:10C98000A0939F09B093A009609142097091430957
:10C9900080914409909145096093A1097093A2097F
:10C9A0008093A3099093A40920E030E040E85FE37E
:10C9B0000F940EBE6093420970934309809344091B
:10C9C0009093450982E299E09F938F93812C912C5B
:10C9D000B8ECAB2EB3E4BB2E12E4C12E19E0D12E7D
:10C9E000ED80FE800F811885A301920169817A8113
:10C9F0008B819C810F94280620E030E040EA51E4CE
:10CA000060913E0970913F098091400990914109E0
:10CA10000F940FBE2B013C010F900F9020E030E0EF
:10CA200042E553E40F94EBC018164CF040923E09D7
:10CA300050923F0960924009709241090CC080E019
:10CA400090E0A2E5B3E480933E0990933F09A09360
:10CA50004009B0934109E0903E09F0903F090091F0
:10CA600040091091410920913A0930913B094091C8
:10CA70003C0950913D0960913609709137098091C8
:10CA8000380990913909A2E26A2EA9E07A2E7F92A4
:10CA90006F92812C912CB0E7AB2EB1E4BB2EE2E477
:10CAA000CE2EE9E0DE2E0F9428061092BD181092CB
:10CAB000BC181092BF181092BE181092C118109294
:10CAC000C01880E090E0A8E4B2E480933609909327
:10CAD0003709A0933809B093390980E090E0AEE3BC
:10CAE000B3E480933A0990933B09A0933C09B09337
:10CAF0003D09E0903E09F0903F09009140091091F6
:10CB000041097F926F92812C912CF8E4AF2EF2E4D0
:10CB1000BF2E9C01AD01C501B4010F9428061092EF
:10CB20002109109220090F900F900F900F902896D6
:10CB30000FB6F894DEBF0FBECDBFDF91CF911F912E
:10CB40000F91FF90EF90DF90CF90BF90AF909F90AC
:10CB50008F907F906F905F904F900D94891C0F93F2
:10CB60001F93CF93DF9300D01F92CDB7DEB7E09134
:10CB7000220984E0E89FF0011124EC54F74E408133
:10CB8000518162817381EDE6F9E084918F01882300
:10CB900079F049835A836B837C830E94F9420F5F4B
:10CBA0001F4FF80184917C816B815A814981EFCFBD
:10CBB00022E030E084ED97E00E94FD41E9E6F9E0F3
:10CBC00084918F01882339F00E94F9420F5F1F4F33
:10CBD000F8018491F7CF6091220970E04AE050E0BB
:10CBE00084ED97E00E942C41E5E6F9E084918F0105
:10CBF000882339F00E94F9420F5F1F4FF80184919A
:10CC0000F7CF40919E1850919F186091A018709195
:10CC1000A11821E030E084ED97E00E94FD418AE018
:10CC20000F900F900F900F90DF91CF911F910F9168
:10CC30000C94F942CF93DF93CDB7DEB761970FB66F
:10CC4000F894DEBF0FBECDBF0F9411B66D877E87FF
:10CC50008F87988B2091C209298B179A10922709E8
:10CC6000169A10922809149A64E182E00F944A37C8
:10CC700064E182E00F947B3764E183E00F944A37EC
:10CC800064E183E00F947B3783E40F941A3A98872A
:10CC90008F834090EA0E5090EB0E6090EC0E7090F7
:10CCA000ED0E0F949B13481A590A610871080E94EF
:10CCB00084CA481A590A6108710877FE03C0412CDA
:10CCC000512C320190911E1280911D12981799F0EB
:10CCD000E0911D1282E5E89FF0011124E15EFD4E16
:10CCE00020E030E040E752E462A173A184A195A165
:10CCF0000F94BDC108C060910E0270910F02809127
:10CD00001002909111020F9457BF7E836D830F9490
:10CD1000AD0483E00F94F81CAB01BC018EE69FE0EC
:10CD20000F9447CB6091BB0981E0682782E79FE0C1
:10CD30000F9435CB0E94F3C31092C209789420E07F
:10CD400030E040E85FE360914209709143098091CF
:10CD50004409909145090F940EBE69837A838B83B1
:10CD60009C83E0903E09F0903F09009140091091AA
:10CD7000410920913A0930913B0940913C09509179
:10CD80003D09609136097091370980913809909179
:10CD90003909E2E22E2EE9E03E2E3F922F92812CBD
:10CDA000912CFEEBAF2EF2E4BF2EDE0111966D0149
:10CDB0000F9428060F94891C149A20E030E040E874
:10CDC0005FE3609142097091430980914409909119
:10CDD00045090F940EBE69837A838B839C8367E039
:10CDE00074E0EF81F8856E1B7F0BA4E07695679564
:10CDF000AA95E1F780E090E00F9488BF69877A8771
:10CE00008B879C872AE037ED43E25FE360913E0920
:10CE100070913F0980914009909141090F940FBE94
:10CE20006B017C012091B2173091B3174091B41778
:10CE30005091B51769857A858B859C850F94EFBED7
:10CE40009B01AC01C701B6010F940FBE7B018C01A1
:10CE500020913A0930913B0940913C0950913D099C
:10CE6000609136097091370980913809909139099C
:10CE70003F922F92812C912CB0E2AB2EB2E4BB2ECC
:10CE8000DE0111966D010F9428060F94891C149AE7
:10CE900020E030E040E85FE360914209709143098F
:10CEA00080914409909145090F940EBE69837A835D
:10CEB0008B839C832AE037ED43E25FE360913E0978
:10CEC00070913F0980914009909141090F940FBEE4
:10CED0006B017C012091B2173091B3174091B417C8
:10CEE0005091B51769857A858B859C850F94EFBE27
:10CEF0009B01AC01C701B6010F940FBE7B018C01F1
:10CF000020913A0930913B0940913C0950913D09EB
:10CF100060913609709137098091380990913909EB
:10CF20003F922F92FE0131966F010F9428060F94C5
:10CF3000891C149AB301A20181E99FE00F9447CBA9
:10CF40000F900F900F900F900F900F9005E71FE03C
:10CF5000F12C83E0E82E8F2D6E2D0F948BC3209142
:10CF60004B11222321F125E18202F001112483E0FB
:10CF70009802E00DF11D1124EE0FFF1FEE0FFF1FB1
:10CF8000E55BFE4E20E030E04AE754E461817281C7
:10CF9000838194810F94BDC120E030E040E05FE3E5
:10CFA0000F940FBE0F94C5BF0F9457BF02C060E02F
:10CFB00070E0C8010F944FCBF3940E5F1F4F99E0C0
:10CFC000F912C9CF6F81788583E79FE00F944FCB2B
:10CFD00040913609509137096091380970913909AB
:10CFE0008DE99FE00F9447CB40913A0950913B095E
:10CFF00060913C0970913D0981EA9FE00F9447CB15
:10D0000040913E0950913F0960914009709141095A
:10D010008DE89FE00F9447CBBE016B5F7F4F89E89F
:10D020009FE00F947B48E0912209F0E0EE0FFF1F94
:10D03000E454F74E60818CE89FE00F9435CB60910B
:10D04000BA188BE89FE00F9435CB6091200988E8EF
:10D050009FE00F9435CBA989AA2329F061E085EAE6
:10D060009FE00F9435CB0F94891CE0E6F9E08491A2
:10D070008F01882339F00E94F9420F5F1F4FF8019A
:10D080008491F7CF83E40F941A3A4AE050E0BC0150
:10D0900084ED97E00E94634184E69FE00F9423CBE8
:10D0A00061E0680F84E69FE00F9435CB8FEF9EE040
:10D0B0000F9430CBBC016F5F7F4F8FEF9EE00F94DA
:10D0C0004FCBE5E5F9E084918F01882339F00E9488
:10D0D000F9420F5F1F4FF8018491F7CF8AE00E9459
:10D0E000F9420F9411B6AB01BC018D859E85AF85C9
:10D0F000B889481B590B6A0B7B0B2AE030E084EDA2
:10D1000097E00E946F41F8941A8219828091010180
:10D110008460809301019FB7F8948091020184603C
:10D12000809302019FBF1A82198289819A81803D72
:10D13000974038F4000089819A8101969A83898307
:10D14000F4CF9FB7F894809102018B7F8093020106
:10D150009FBF9FB7F894809102018B7F809302015B
:10D160009FBF1A82198289819A8180349F4188F7F2
:10D17000000089819A8101969A838983F4CF6F9800
:10D180007798EAE6F0E080818F7B808380818068F9
:10D190008083EF9A08951F920F920FB60F92112479
:10D1A0002F933F934F935F936F937F938F939F93AF
:10D1B000AF93BF9320912009309121092B34310581
:10D1C0000CF449C080916A0086FF11C08091F81963
:10D1D0009091F919A091FA19B091FB1980938909DE
:10D1E00090938A09A0938B09B0938C092EC08091EB
:10D1F000F8199091F919A091FA19B091FB19409181
:10D20000890950918A0960918B0970918C09841B5E
:10D21000950BA60BB70B253631052CF043E050E0FB
:10D2200060E070E004C044E050E060E070E084172B
:10D230009507A607B70748F080916809909169099A
:10D240000296909369098093680980916A0090E43E
:10D25000892780936A00BF91AF919F918F917F91B1
:10D260006F915F914F913F912F910F900FBE0F9053
:10D270001F9018956C987498EAE6F0E080818160C0
:10D28000808380818D7F8083EC9A08951F920F9216
:10D290000FB60F9211240BB60F922F933F934F931B
:10D2A0005F936F937F938F939F93AF93BF93CF932E
:10D2B000DF93EF93FF93EC98E0E5F9E08491EF01C1
:10D2C000882331F00E94F9422196FE018491F8CF23
:10D2D0008AE00E94F9428091C2098111ABDCFF9182
:10D2E000EF91DF91CF91BF91AF919F918F917F91FE
:10D2F0006F915F914F913F912F910F900BBE0F90C7
:10D300000FBE0F901F9018954F925F926F927F9271
:10D310008F929F92BF92CF92DF92EF92FF920F93E4
:10D320001F93CF93DF93CDB7DEB7EA970FB6F8948C
:10D33000DEBF0FBECDBF88E89FE00F9423CBB82E91
:10D34000BE01675C7F4F89E89FE00F948C48EBE05B
:10D35000F8E084918F01882339F00E94F9420F5F31
:10D360001F4FF8018491F7CF69AD7AAD4AE050E0E4
:10D3700084ED97E00E9448418AE59FE00F9423CB1B
:10D38000882E912C4AE050E0B40184ED97E00E9491
:10D3900048410AE01FE0E12CF12C3E01F4E36F0E5E
:10D3A000711CE814F9042CF5FE01BC962F016801EC
:10D3B000C6010F9423CBF20181932F01FFEFCF1A07
:10D3C000DF0A46145704A1F71CAABE01645D7F4F13
:10D3D00084ED97E00E943741BE01645D7F4F80EC91
:10D3E00099E00E94B3C18FEFE81AF80A085F1F4F57
:10D3F000D8CF8E01015E1F4F95E9E92E9FE0F92EEF
:10D40000D02EC12EC7010F9423CBF80181938F0139
:10D41000FFEFEF1AFF0A8DE9E8168FE0F80691F7A3
:10D420001FA20D2D1C2DF80181918F01882319F069
:10D430000E94F942F8CF66E078E08D2D9C2D0F9484
:10D440000AC7CF92DF928FEF97E09F938F938E0161
:10D450000F5F1F4F1F930F930F94F7C80F900F90FC
:10D460000F900F900F900F907E01F5E0EF0EF11CE2
:10D47000F7018081882349F0992787FD90950F94C3
:10D48000F9C6F70181937F01F3CF60E0C8010E94E4
:10D4900069C481E99FE00F942BCBF62EE72ED82E9E
:10D4A000C92EE4EEF7E084914F01882341F00E94F9
:10D4B000F942FFEF8F1A9F0AF4018491F6CF2AE018
:10D4C00030E04F2D5E2D6D2D7C2D84ED97E00E9478
:10D4D0006F4161E080EE97E00E9469C46BED77E0F8
:10D4E000C8010F9415C78DE99FE00F942BCB6DAB4E
:10D4F0007EAB8FAB98AFCE01C5960F94404EBC016A
:10D50000C8010F94A4C768ED77E0C8010F940AC75B
:10D5100081EA9FE00F942BCB6DAB7EAB8FAB98AFC6
:10D52000CE01C5960F94404EBC01C8010F94A4C70C
:10D5300061ED77E0C8010F940AC760E0C8010E945E
:10D5400069C46CEC77E0C8010F9415C78DE89FE0C3
:10D550000F942BCB6DAB7EAB8FAB98AFCE01C59646
:10D560000F94404EBC01C8010F94A4C760E0C801ED
:10D570000E9469C461E08FEB97E00E9469C48AADA4
:10D580008F9389AD8F9388EB97E09F938F931F9331
:10D590000F930F94F7C860E0C8010E9469C482E746
:10D5A0009FE00F9423CB0F900F900F900F900F9050
:10D5B0000F90882329F061E084EB97E00E9469C412
:10D5C0006DEA77E0C8010F9415C78B2D90E09EABF4
:10D5D0008DABCE01C5960F941551BC01C8010F94B7
:10D5E000A4C760E0C8010E9469C4CF92DF92EF92A5
:10D5F000FF9284EA97E09F938F931F930F930F946A
:10D60000F7C860E0C8010E9469C461E080EA97E061
:10D610000E9469C40FB6F894DEBF0FBECDBFEA9674
:10D620000FB6F894DEBF0FBECDBFDF91CF911F9133
:10D630000F91FF90EF90DF90CF90BF909F908F90D1
:10D640007F906F905F904F9008954F925F926F928E
:10D650007F92AF92BF92CF92DF92EF92FF920F93A1
:10D660001F93CF93DF93CDB7DEB7E0970FB6F89453
:10D67000DEBF0FBECDBF2B013C0169017A01809155
:10D6800075088111F0C0F8940F947B138091EA0E15
:10D690009091EB0EA091EC0EB091ED0E809371087D
:10D6A00090937208A0937308B09374080F949B131F
:10D6B00040917108509172086091730870917408DC
:10D6C000481B590B61097109409371085093720806
:10D6D00060937308709374080E9484CA4091710823
:10D6E000509172086091730870917408481B590B2F
:10D6F000610971094093710850937208609373082F
:10D700007093740890911E1280911D12981799F0D1
:10D71000E0911D1282E5E89FF0011124E15EFD4ECB
:10D7200020E030E040E752E462A173A184A195A11A
:10D730000F94BDC108C060910E0270910F028091DC
:10D7400010029091110260935D0870935E088093BF
:10D750005F08909360080F94AD0480E1E6E3F9E080
:10D76000A1E6B8E001900D928A95E1F78091220937
:10D7700080935C088091090280935B080E94F3C348
:10D780001092C20981E080937508B19A10928500C9
:10D790001092840080ED97E0909389008093880038
:10D7A000789420E030E0A901C301B2010F94E8BEF3
:10D7B00081110AC020E030E0A901C701B6010F9431
:10D7C000E8BE882309F44FC06BE977E0FE0131968B
:10D7D0005F01CF010F9415C7F50101900020E9F713
:10D7E0008F01015011092091690830916A08409118
:10D7F0006B0850916C08C301B2010F940FBE23E077
:10D8000048E00F9438C468E977E0C5010F940AC76F
:10D81000F50101900020E9F78F010150110923E083
:10D8200046E0C701B6010F9438C465E977E0C50149
:10D830000F940AC7F50101900020E9F78F0101500C
:10D84000110960916202709163028091640290916B
:10D85000650223E048E00F9438C460E0C5010E94EF
:10D8600069C40E94C8C5E0960FB6F894DEBF0FBE2B
:10D87000CDBFDF91CF911F910F91FF90EF90DF907F
:10D88000CF90BF90AF907F906F905F904F90089532
:10D8900020E030E0A90160E070E080E291E4D5CEC4
:10D8A0008F929F92AF92BF92CF92DF92EF92FF92B0
:10D8B0000F931F93CF93DF9300D01F92CDB7DEB7A6
:10D8C0009B01AC0180917508882309F49FC0809169
:10D8D0005C088093220980915D0890915E08A09178
:10D8E0005F08B091600880930E0290930F02A0939E
:10D8F0001002B093110260916D0870916E088091D2
:10D900006F08909170080F940EBE69837A838B83A1
:10D910009C83CE0101960F940D1320E030E040E58A
:10D9200051E460916202709163028091640290916F
:10D9300065020F94EFBE4B015C01E0906908F09026
:10D940006A0800916B0810916C082091650830916D
:10D95000660840916708509168086091610870916D
:10D9600062088091630890916408E2E2F9E0FF9315
:10D97000EF93EDE6CE2EE8E0DE2E0F9428060F940E
:10D98000891C80E1E1E6F8E0A6E3B9E001900D92A0
:10D990008A95E1F780E1E6E3F9E0A1E0B9E00190E2
:10D9A0000D928A95E1F7409171085091720860914B
:10D9B0007308709174084093D10C5093D20C60930B
:10D9C000D30C7093D40C8CE19CE00E94C2A980918E
:10D9D000710890917208A0917308B09174088093B7
:10D9E000EA0E9093EB0EA093EC0EB093ED0E81E057
:10D9F0008093C2091092750881E997E09F938F93F5
:10DA00000F944AC80F900F900F900F900F900F90A7
:10DA10000F900F90DF91CF911F910F91FF90EF909A
:10DA2000DF90CF90BF90AF909F908F90089560E06F
:10DA300070E0CB0135CFFBDF81E08093AE0208952B
:10DA40002F923F924F925F926F927F928F929F920E
:10DA5000AF92BF92CF92DF92EF92FF920F931F93FC
:10DA6000CF93DF93CDB7DEB7C755D1090FB6F89482
:10DA7000DEBF0FBECDBF82E090E09093180280938E
:10DA8000170281E993E00E945A428823B1F0809105
:10DA9000020F9091030F6AE270E005960F94AFC7F2
:10DAA000009711F0DC011C928091020F9091030FFE
:10DAB00005960F9489490C94C59486E993E00E94D9
:10DAC0005A42882381F08BE797E00E945A42182F30
:10DAD00086E597E00E945A4281111260812F0E94D0
:10DAE0005D470C94C59485EA93E00E945A428823CE
:10DAF00019F0A1DF0C94C59483EB93E00E945A4285
:10DB0000882321F00E94B3470C94C59480EC93E0E5
:10DB10000E945A42882309F4A2C186EC93E00E9435
:10DB20005A42882391F08091CB19882311F40C94E8
:10DB3000C5940F9411B66093BC097093BD0980938E
:10DB4000BE099093BF090C94C5948BEC93E00E949E
:10DB50005A42882361F060918309709184094AE0F8
:10DB600050E084ED97E00E9463410C94C5948FECE3
:10DB700093E00E945A42882309F442C003ED13E067
:10DB8000F80181918F01882319F00E94F942F8CFA2
:10DB900080916209909163092CE3289FB001299F2D
:10DBA000700D11244AE050E084ED97E00E942C4172
:10DBB00067ED73E084ED97E00E9437410CED13E0D0
:10DBC000D8018D918D01882319F00E94F942F8CF78
:10DBD00080916409909165092CE3289FB001299FE9
:10DBE000700D11244AE050E084ED97E00E942C4132
:10DBF00067ED73E084ED97E00E9437410C94C59483
:10DC000082EE93E00E945A428823C1F08091CB19A2
:10DC1000882361F06091C9197091CA194AE050E0F7
:10DC200084ED97E00E9448410C94C59465EE73E042
:10DC300084ED97E00E9437410C94C59487EF93E000
:10DC40000E945A42882369F16091020F7091030F7C
:10DC50006D5F7F4F21E041E080EC99E00E9406B9C2
:10DC60008091240C9091250CA091260CB091270C4A
:10DC70008093D10C9093D20CA093D30CB093D40C7E
:10DC80008CE19CE00E94F9A88C010E94F9420A30C4
:10DC9000110531F760E080EC99E00E94A5B80C9482
:10DCA000C5948AEF93E00E945A42882399F00E941B
:10DCB000335081E0809385096091020F7091030FCA
:10DCC0006C5F7F4F21E040E080EC99E00E9406B954
:10DCD0000C94C5948EEF93E00E945A428823D9F1A8
:10DCE0008091CB19882309F4A1CF1092590801E043
:10DCF00014E0F80181918F01882319F00E94F94204
:10DD0000F8CF00E010E0FF24F39480915508909143
:10DD100056082091570830915808821B930B8F7733
:10DD20009927892B69F084ED97E00E943F40F0929B
:10DD300059080E94F9420F5F1F4F10925908E5CF12
:10DD40000331110514F381E0809359088AE00E94A1
:10DD5000F9420C94C59484E094E00E945A428823CE
:10DD600079F008E014E0D8018D918D01882319F035
:10DD70000E94F942F8CF8AE00E94F9420C94C594BF
:10DD800082E194E00E945A42882351F006E114E0B7
:10DD9000F80181918F01882371F30E94F942F8CF35
:10DDA00085E394E00E945A42882321F00F9427498A
:10DDB0000C94C5948AE394E00E945A42882341F06F
:10DDC00060E070E088EF9FE00F947B480C94C5946E
:10DDD0008DE394E00E945A42882359F06DE374E089
:10DDE00084ED97E00E94374140E052EC61E070E042
:10DDF00010C088E494E00E945A42882381F068E4CD
:10DE000074E084ED97E00E94374140E054E961E11D
:10DE100070E084ED97E00E94C43F0C944D9A84E535
:10DE200094E00E945A42882361F00F9411B66093E7
:10DE3000AF097093B0098093B1099093B2090C9423
:10DE4000C59489E594E00E945A42882311F40C9409
:10DE5000C59461E080E00E94D2470C94C5948EE5A1
:10DE60000E94C24281110C94C59487E40E94C24270
:10DE7000882311F40C94157E0E94F0420F9457BF32
:10DE80006C34710509F414C47CF56430710509F42F
:10DE900008C154F46230710509F4EBC00CF0F5C010
:10DEA00077FF77C00C94017E6C31710509F450C185
:10DEB0007CF46A30710509F445C16B30710511F0CD
:10DEC0000C94017E60E080E00E94AC570C94C594F5
:10DED0006E31710509F434C36B34710511F00C9483
:10DEE000017E08E210E0D1C36835710511F40C948D
:10DEF000C5940CF56135710511F40C94D17C64F472
:10DF00006F34710511F40C94EC776035710511F4E0
:10DF10000C9427780C94017E6635710511F40C94ED
:10DF2000817D6735710511F00C94017E81E00E94BE
:10DF3000EE460C94C5946C35710511F40C948A7DF1
:10DF40007CF46A35710511F40C94867D6B3571058E
:10DF500011F00C94017E81E08093EC080C94C59440
:10DF60006236710511F40C94EC7D6336710511F085
:10DF70000C94017E1092CB190F942C496091CB190F
:10DF800084EC9FE00F9435CB82E00F94FF840C94D7
:10DF9000C5948091D60881110C94C5940E94E153D8
:10DFA00060917F0970918009809181099091820927
:10DFB0000F9488BF6B017C01409042095090430947
:10DFC000609044097090450980900D0990900E0969
:10DFD000A0900F09B0901009A5019401C301B201EE
:10DFE0000F940EBE20E030E048EC52E40F94BDC127
:10DFF0009B01AC01C701B6010F94EBC01816E4F405
:10E00000A3019201C501B4010F940EBE20E030E0DF
:10E0100048EC52E40F94BDC19B01AC01C701B601AD
:10E020000F940FBE0F945CBF60937F0970938009BB
:10E03000809381099093820980911F098823A9F018
:10E0400088E50E94C242811110C089E50E94C24247
:10E0500081110BC08AE50E94C242811106C085E48D
:10E060000E94C24281110C94CE940E94A9560C9435
:10E07000C5948091D60881110C94C5940E94645473
:10E0800081E00E9487590C94C5948091D608811133
:10E090000C94C5940E94645480E00E9487590C94AB
:10E0A000C59480E50E94C242882339F00E94F04264
:10E0B0000F945CBF6B017C0103C0C12CD12C760195
:10E0C00083E50E94C242882361F00E94F04220E072
:10E0D00030E04AE754E40F94BDC10F945CBF6B017C
:10E0E0007C01C114D104E104F10431F0E4ECFAE460
:10E0F000859194910F9496490F94891C0F9411B6B1
:10E100004B015C018C0C9D1CAE1CBF1C0F9411B606
:10E110006093E8087093E9088093EA089093EB080D
:10E120000F9411B6681579058A059B0510F00C94BB
:10E13000C5940F941B2980E00E94A85D80E00F9495
:10E14000FF84EECF60E081E00E94AC570C94C59450
:10E150000F94891C81E08093B40988E50E94C24233
:10E16000182F89E50E94C242082F8AE50E94C24208
:10E17000782E101308C0181305C07724739401E09B
:10E1800011E001C0012F0E94B0DC60904B11109291
:10E190004B1182E00F94F81C60933E0970933F0985
:10E1A000809340099093410971100E94B7F9409102
:10E1B0000E0250910F026091100270911102409373
:10E1C000ED085093EE086093EF087093F00880918B
:10E1D0005802909159029093B7098093B60984E64A
:10E1E00090E090935902809358020F9411B6609377
:10E1F000E8087093E9088093EA089093EB0881E0BF
:10E200000F94CD1480E1E6E3F9E0A1E0B9E00190DC
:10E210000D928A95E1F710920E0210920F02109261
:10E22000100210921102112321F080E090E00E9470
:10E23000D34B002321F081E090E00E94D34B88E58E
:10E240000E94C242882341F00E94E542672B682B5E
:10E25000692B11F00C94FD9489E50E94C242882339
:10E2600041F00E94E542672B682B692B11F00C945A
:10E270001395772009F4F1C080912709882321F0B4
:10E2800080912809811108C080E090E00E94D34B62
:10E2900081E090E00E94D34B0E9405DDEBE4FCE4BA
:10E2A00085919591A591B49189839A83AB83BC8321
:10E2B000E7E4FCE485919591A591B4918F8F98A3A3
:10E2C000A9A3BAA325E039E041E059E0BE016F5FA0
:10E2D0007F4FCE014F960E940F450E9477DC20E0D1
:10E2E00030E040E850EC609105097091060980919A
:10E2F0000709909108090F94E8BE87FF0CC080E0E1
:10E3000090E0A0E8B0EC8093050990930609A093F3
:10E310000709B093080980E090E0A0EAB0E4809398
:10E32000090990930A09A0930B09B0930C0920E006
:10E3300030E040E251E460916202709163028091AA
:10E340006402909165020F94EFBE60930E02709389
:10E350000F02809310029093110210923E091092C6
:10E360003F09109240091092410980E00F94CD14AA
:10E37000E0903E09F0903F09009140091091410959
:10E3800020913A0930913B0940913C0950913D0957
:10E390006091360970913709809138099091390957
:10E3A000F2E4CF2EF9E0DF2E0F94981180900E0248
:10E3B00090900F02A0901002B0901102E090090915
:10E3C000F0900A0900910B0910910C0920910509A0
:10E3D000309106094091070950910809609101099F
:10E3E000709102098091030990910409E2E2F9E039
:10E3F000FF93EF93ADE0CA2EA9E0DA2E0F94280622
:10E400000F94891C8091010990910209A091030940
:10E41000B09104098093360990933709A093380985
:10E42000B09339098091050990910609A0910709D7
:10E43000B091080980933A0990933B09A0933C0955
:10E44000B0933D0981E00F94CD140F94B51482E090
:10E4500090E00E94D34B0F900F908AE50E94C24239
:10E46000882341F00E94E542672B682B692B11F04D
:10E470000C942995E0903E09F0903F0900914009E5
:10E480001091410920913A0930913B0940913C0992
:10E4900050913D0960913609709137098091380992
:10E4A00090913909E2E4CE2EE9E0DE2E0F94981126
:10E4B00080E00F94CD148091ED089091EE08A0912A
:10E4C000EF08B091F00880930E0290930F02A09392
:10E4D0001002B09311028091B6099091B709909300
:10E4E0005902809358020F9411B66093E808709314
:10E4F000E9088093EA089093EB080F94B5140E9402
:10E5000005DD0E9457DE88E50E94C24281110C940D
:10E51000919489E50E94C24281110C94919487E5FF
:10E520000E94C24281110C9491948AE50E94C242D9
:10E5300081110C9491940F94891C1092B40987C591
:10E540000F94891C81E00E946E428091620290913A
:10E550006302A0916402B091650280930E029093D1
:10E560000F02A0931002B093110220E030E043E0CC
:10E5700060E070E080E291EC0E94E6DEE2E7FBE41E
:10E5800005911491F8018491882329F00E94F942A1
:10E590000F5F1F4FF7CFEEE4FCE084918F018823DB
:10E5A00039F00E94F9420F5F1F4FF8018491F7CFB5
:10E5B00040913609509137096091380970913909B5
:10E5C00025E030E084ED97E00E94FD41E9E4FCE0C5
:10E5D00084918F01882339F00E94F9420F5F1F4F09
:10E5E000F8018491F7CF40913A0950913B0960912D
:10E5F0003C0970913D0925E030E084ED97E00E94F0
:10E60000FD41E4E4FCE084918F01882339F00E940D
:10E61000F9420F5F1F4FF8018491F7CF40913E09F7
:10E6200050913F09609140097091410925E030E027
:10E6300084ED97E00E94FD41E2E4FCE084918F01CB
:10E64000882339F00E94F9420F5F1F4FF80184912F
:10E65000F7CF0E949C420C94C594B801882777FD9F
:10E660008095982F0F948ABF0E943460AB01BC0143
:10E6700022E030E084ED97E00E94FE410F5F1F4FE3
:10E680000F36110511F40C94C5944AE050E0B8011E
:10E6900084ED97E00E942C4151E1E52E57E0F52EE4
:10E6A000D7018D917D018823C1F20E94F942F8CFF4
:10E6B000ECE0F8E4859194910F949C95E0918609A3
:10E6C000F0E0EE0FFF1FE25DF74B8591949140E083
:10E6D00060E00F94DA8A882359F0E0918609F0E02F
:10E6E000EE0FFF1FE65DF64B859194910F949C957C
:10E6F00080912709882341F080912809882321F0FF
:10E7000080912909811109C00E94C8C561E08BE38D
:10E710009CE00E942DC50C94C59481E090E09093FC
:10E72000180280931702EDE1FCE084918F018823A9
:10E7300039F00E94F9420F5F1F4FF8018491F7CF23
:10E740008AE00E94F9421A821982C090AE18D090D5
:10E75000AF18E090B018F090B11820E030E040EA37
:10E7600050E4C701B6010F94EFBE0F9457BF45E0C8
:10E77000469F9001479F300D1124B901882777FDEE
:10E780008095982F0F948ABF2B013C0120E030E048
:10E790004CE052E40F94E8BE87FF06C0412C512C98
:10E7A0002CE0622E22E4722EA7019601C301B20171
:10E7B0000F94E8BE87FF0AC020E030E040EA50E452
:10E7C000C301B2010F940FBE2B013C01E9E0FCE054
:10E7D00084918F01882339F00E94F9420F5F1F4F07
:10E7E000F8018491F7CF22E030E0B301A20184ED7B
:10E7F00097E00E94FE4120E030E040EF51E4C30189
:10E80000B2010F940EBE20E030E04CE852E40F94C9
:10E810000FBE0F9457BF7093BB186093BA1884E073
:10E8200090E0909378098093770981E090E090934D
:10E83000760980937509E0918609F0E0EE0FFF1FDD
:10E84000E65EF74B8591949121E0892B09F420E055
:10E8500020937A0980E090E0A0EAB1E48093360941
:10E8600090933709A0933809B093390980E090E07C
:10E87000A0E7B2E480933A0990933B09A0933C0946
:10E88000B0933D098AE999E9A9E1BEE380933E0985
:10E8900090933F09A0934009B093410982E299E027
:10E8A0009F938F93812C912C18E4A12E12E4B12E0A
:10E8B00002E4C02E09E0D02E1AE9E12E19E9F12E6A
:10E8C00009E11EE320E030E040E752E460E070E060
:10E8D00080EA91E40F9428060F94891C0F900F9002
:10E8E000A30192016091AE187091AF188091B01899
:10E8F0009091B1180F94E8BE87FF07C088EE93E0AF
:10E900000E94425C0E94AF65EBCF60E086EA9FE028
:10E910000F9435CB80E090E0A0EAB0E480933E090C
:10E9200090933F09A0934009B093410920913A097F
:10E9300030913B0940913C0950913D096091360965
:10E94000709137098091380990913909E2E2F9E034
:10E95000FF93EF93812C912CE8E4AE2EE2E4BE2EDF
:10E96000F2E4CF2EF9E0DF2EE12CF12C00EA10E4E6
:10E970000F942806E7E4FCE485919591A591B49164
:10E980008093360990933709A0933809B0933909D9
:10E99000EBE4FCE4259135914591549120933A099B
:10E9A00030933B0940933C0950933D09E0903E0968
:10E9B000F0903F090091400910914109609136099A
:10E9C000709137098091380990913909E2E2F9E0B4
:10E9D000FF93EF93812C912CB8E4AB2EB2E4BB2EC5
:10E9E0000F9428060F94891C20E030E043E060E09B
:10E9F00070E080E89FEB0E94E6DE80913E099091F6
:10EA00003F09A0914009B09141098AAF9BAFACAFDB
:10EA1000BDAFE8E0FCE084910F900F900F900F9055
:10EA20008F01882339F00E94F9420F5F1F4FF801D0
:10EA30008491F7CF8AE00E94F942E1E0FCE0849102
:10EA40008F01882339F00E94F9420F5F1F4FF801B0
:10EA50008491F7CF40913E0950913F096091400960
:10EA60007091410922E030E084ED97E00E94FD4181
:10EA7000E0E0FCE084918F01882339F00E94F942A4
:10EA80000F5F1F4FF8018491F7CF8AE00E94F9428F
:10EA90002EEA222E2FE0322E33E2E32EF12C0FEF5E
:10EAA0001FEFB701882777FD8095982F0F948ABFB5
:10EAB0004B015C01E9EFFBE084916F01882341F099
:10EAC0000E94F942FFEFCF1ADF0AF6018491F6CFD8
:10EAD0004AE050E0B8016E5F7F4F84ED97E00E94FE
:10EAE0002C41ECEEFBE084916F01882341F00E9401
:10EAF000F942FFEFCF1ADF0AF6018491F6CF8AE0E0
:10EB00000E94F942E8EDFBE084916F01882341F017
:10EB10000E94F942FFEFCF1ADF0AF6018491F6CF87
:10EB20004AE050E0B70184ED97E00E942C41E9EC07
:10EB3000FBE084916F01882341F00E94F942FFEFCE
:10EB4000CF1ADF0AF6018491F6CF4AE050E060E088
:10EB500070E084ED97E00E942C41E8ECFBE08491AA
:10EB60006F01882341F00E94F942FFEFCF1ADF0ABC
:10EB7000F6018491F6CF8AE00E94F9420F3FFFEF41
:10EB80001F0731F0BE016F5F7F4FC1010F947B48BB
:10EB9000A5019401C301B2010F94E8BE181664F4F4
:10EBA0000F5F1F4F25E0E20EF11C32E0230E311CF7
:10EBB0000530110509F075CF380147E2641A48EFB6
:10EBC000740A660C771C280163E0460E511C85E030
:10EBD000809FD001819FB00D1124212C312C9D9656
:10EBE000B9AFA8AFC201029705970CF0BCC168ADE0
:10EBF00079AD620D731D882777FD8095982F0F944E
:10EC00008ABF22966CAF7DAF8EAF9FAF2297E1ECAB
:10EC1000FBE084918F01882339F00E94F9420F5F55
:10EC20001F4FF8018491F7CF4AE050E0B20184ED24
:10EC300097E00E942C41EEEBFBE084918F0188234A
:10EC400039F00E94F9420F5F1F4FF8018491F7CF0E
:10EC50008AE00E94F942509276094092750920E0BC
:10EC600030E040EF51E422966CAD7DAD8EAD9FADAE
:10EC700022970F940EBE20E030E040E251E40F9462
:10EC8000BDC120E030E040EA50E40F94EFBE20E048
:10EC900030E048E452E40F940FBE0F9457BF7093D6
:10ECA000BB186093BA1880E090E0A0EAB1E48093CA
:10ECB000360990933709A0933809B093390980E059
:10ECC00090E0A0E7B2E480933A0990933B09A093C7
:10ECD0003C09B0933D098AE999E9A9E1BEE3809333
:10ECE0003E0990933F09A0934009B0934109A2E2E5
:10ECF000B9E0BF93AF93812C912CB8E4AB2EB2E472
:10ED0000BB2E12E4C12E19E0D12E1AE9E12E19E929
:10ED1000F12E09E11EE320E030E040E752E460E03C
:10ED200070E080EA91E40F9428060F94891C0F90FC
:10ED30000F9022962CAD3DAD4EAD5FAD2297609108
:10ED4000AE187091AF188091B0189091B1180F94CF
:10ED5000E8BE87FF07C088EE93E00E94425C0E94F5
:10ED6000AF65E7CF80E090E0A0EAB0E480933E0991
:10ED700090933F09A0934009B093410920913A092B
:10ED800030913B0940913C0950913D096091360911
:10ED9000709137098091380990913909A2E2B9E060
:10EDA000BF93AF93812C912C08E4A02E02E4B02EE7
:10EDB000E2E4CE2EE9E0DE2EE12CF12C00EA10E4B4
:10EDC0000F942806E7E4FCE485919591A591B49110
:10EDD0008093360990933709A0933809B093390985
:10EDE000EBE4FCE4259135914591549120933A0947
:10EDF00030933B0940933C0950933D09E0903E0914
:10EE0000F0903F0900914009109141096091360945
:10EE1000709137098091380990913909A2E2B9E0DF
:10EE2000BF93AF93812C912CA8E4AA2EA2E4BA2E12
:10EE30000F9428060F94891C20E030E043E060E046
:10EE400070E080E89FEB0E94E6DE2AAD3BAD4CAD62
:10EE50005DAD60913E0970913F09809140099091AC
:10EE600041090F940EBE2091B2173091B317409113
:10EE7000B4175091B5170F94BDC10F9457BF7A8343
:10EE80006983EDEBFBE084910F900F900F900F9052
:10EE90008F01882339F00E94F9420F5F1F4FF8015C
:10EEA0008491F7CF8AE00E94F942E9EAFBE084917D
:10EEB0008F01882339F00E94F9420F5F1F4FF8013C
:10EEC0008491F7CF4091AE185091AF186091B0186F
:10EED0007091B11822E030E084ED97E00E94FD418E
:10EEE000EAE9FBE084918F01882339F00E94F9421E
:10EEF0000F5F1F4FF8018491F7CF2AAD3BAD4CADAA
:10EF00005DAD60913E0970913F09809140099091FB
:10EF100041090F940EBEAB01BC0122E030E084ED4C
:10EF200097E00E94FD41E9E9FBE084918F0188238D
:10EF300039F00E94F9420F5F1F4FF8018491F7CF1B
:10EF40008AE00E94F942BE016F5F7F4FC3010F94B8
:10EF50007B48F2E06F0E711C2FEF421A520A35E027
:10EF6000230E311C3FCE109278091092770910922F
:10EF70007A0961E086EA9FE00F9435CBEAE5FBE091
:10EF800084918F01882339F00E94F9420F5F1F4F4F
:10EF9000F8018491F7CF8AE00E94F942179A109203
:10EFA0002709169A10922809149A1092BB181092E9
:10EFB000BA18E0918609F0E0EE0FFF1FEA5EF74B0A
:10EFC000859194910F949C9581E00F94CD8782E078
:10EFD0000F94FF840C94C5940FEF10E0B7E5CB2E8F
:10EFE000BBE0DB2E1093210900932009A4E6EA2E52
:10EFF000F12C84E690E00E94425CF1E0EF1AF10807
:10F00000C1F74AE050E0B80184ED97E00E942C413E
:10F01000F6018491F7E5EF2EFBE0FF2E882341F007
:10F020000E94F942FFEFEF1AFF0AF7018491F6CF31
:10F0300060916409709165094AE050E084ED97E0C1
:10F040000E9448410550110969F60C94C59481E06D
:10F050008093880986E50E94C242882359F0E09196
:10F06000020FF091030F8181893021F08F7D11F023
:10F070000E94D842209127098091CF199091D019F0
:10F08000222341F020912809222321F020912909EF
:10F0900021110FC0029749F00E94C8C561E080E5C8
:10F0A0009BE00E942DC50C94C594109288090C9485
:10F0B000C59410925A08029721F4109288090C9472
:10F0C000C594F0917A092896FFAF28972091770987
:10F0D000309178092A963FAF2EAF2A978091750913
:10F0E000909176092C969FAF8EAF2C9781E08093FC
:10F0F0007A0981E090E0909378098093770983E121
:10F1000090E0909376098093750981E00F94FF84D5
:10F110008BE491E10E9481FA0E94B7F980E090E0CF
:10F12000A0EAB0E480933E0990933F09A093400980
:10F13000B093410920E030E040E752E46091620280
:10F140007091630280916402909165020F94EFBE0A
:10F150004B015C0120913A0930913B0940913C09F7
:10F1600050913D09609136097091370980913809B5
:10F1700090913909E2E2F9E0FF93EF9312E4C12E96
:10F1800019E0D12EE12CF12C00EA10E40F942806AE
:10F19000E7E4FCE485919591A591B49180933609BB
:10F1A00090933709A0933809B0933909EBE4FCE454
:10F1B00085919591A591B49180933A0990933B09DB
:10F1C000A0933C09B0933D096AE379E086E399E0B6
:10F1D0000E94C94520E030E040EF51E460915A02BE
:10F1E00070915B0280915C0290915D020F94EFBE82
:10F1F0004B015C01E0903E09F0903F09009140090D
:10F200001091410920913A0930913B0940913C0904
:10F2100050913D0960913609709137098091380904
:10F2200090913909E2E2F9E0FF93EF930F942806F9
:10F230000F94891C20E030E040EA51E460915A02CA
:10F2400070915B0280915C0290915D020F94EFBE21
:10F250000F9457BF8B0120E030E040E252E4609110
:10F2600062027091630280916402909165020F9432
:10F27000EFBE0F9457BF7B010E9463DC23968FAFD4
:10F28000239780E00E946E420F900F900F900F9096
:10F29000A7E4BCE4BBAFAAAF212C312CC701AA273D
:10F2A00097FDA095BA2F60968CAF9DAFAEAFBFAF64
:10F2B0006097C801AA2797FDA095BA2F64968CAFD6
:10F2C0009DAFAEAFBFAF6497C10163E070E00F9434
:10F2D000ACC37FAF6EAF99AF88AF60FF06C0A2E04E
:10F2E000B0E0A81BB90BB9AFA8AF2396BFAD239769
:10F2F000BB2379F12114310461F18EAD9FAD880FEC
:10F30000991FEEADFFAD8E0F9F1F28AD39AD820F57
:10F31000931F880F991F8D53904F0F9430CBBC01D2
:10F32000882777FD8095982F0F948ABF2AE037EDC4
:10F3300043E25CE30F94BDC120914C1130914D111B
:10F3400040914E1150914F110F940FBE2B013C0173
:10F3500003C0412C512C320180E090E0A0EAB0E4DF
:10F3600080933E0990933F09A0934009B0934109CF
:10F3700060966CAD7DAD8EAD9FAD60970F948ABFEA
:10F3800027966CAF7DAF8EAF9FAF279720913A093C
:10F3900030913B0940913C0950913D0960913609FB
:10F3A000709137098091380990913909A2E2B9E04A
:10F3B000BF93AF9327968CAC9DACAEACBFAC2797F8
:10F3C000E2E4CE2EE9E0DE2EE12CF12C00EA10E49E
:10F3D0000F9428060F94891CEAADFBAD8591959199
:10F3E000A591B4918093360990933709A093380979
:10F3F000B0933909EAADFBAD349685919591A5910D
:10F40000B49180933A0990933B09A0933C09B0933F
:10F410003D096AE379E086E399E00E94C945649674
:10F420006CAD7DAD8EAD9FAD64970F948ABF4B01DF
:10F430005C01E0903E09F0903F0900914009109175
:10F44000410920913A0930913B0940913C09509182
:10F450003D09609136097091370980913809909182
:10F460003909A2E2B9E0BF93AF930F9428060F9435
:10F47000891C0F900F900F900F902396FFAD23974C
:10F48000FF2361F02114310449F020E030E040E82E
:10F490005FE3C301B2010F940EBE04C060E070E0F0
:10F4A00080E291EC20E030E043E00E94E6DE811152
:10F4B00008C0E0918609F0E0EE0FFF1FE45BF44B1B
:10F4C0001FC0C0903E09D0903F09E0904009F090E5
:10F4D0004109A701960160E070E080EA90E40F9492
:10F4E0000EBE2DEC3CEC4CEC5DE30F94E8BE87FFC8
:10F4F0000AC0E0918609F0E0EE0FFF1FE85BF44BD5
:10F500006590749066C023962FAD23972223B9F09F
:10F51000A7019601C301B2010F940EBE9F7720E0B0
:10F5200030E040E85FE30F94EBC0181644F4E0913C
:10F530008609F0E0EE0FFF1FE05BF44BE1CF609136
:10F54000AE187091AF188091B0189091B1180E94C8
:10F550001B649B01AC01A7E08EAD9FADA89F80010D
:10F56000A99F100D1124E8ADF9AD0E0F1F1F000F5C
:10F57000111F000F111F055B1E4E60913E09709117
:10F580003F0980914009909141090F940EBED80126
:10F5900011966D937D938D939C931497809175092B
:10F5A0009091760901979093760980937509BFEF42
:10F5B0002B1A3B0A81E00F94FF84EAADFBAD38962D
:10F5C000FBAFEAAFF9E02F16310409F07DCE612CD4
:10F5D000712C80E090E0A0EAB0E480933E09909323
:10F5E0003F09A0934009B093410920913A09309115
:10F5F0003B0940913C0950913D0960913609709159
:10F6000037098091380990913909E2E2F9E0FF93D6
:10F61000EF9327968CAC9DACAEACBFAC2797E2E4E1
:10F62000CE2EE9E0DE2EE12CF12C00EA10E40F945E
:10F6300028060F94891C0F900F9029E022163104A0
:10F6400021F060E0C3010C9422840E949C420E943D
:10F650009FF980EC9FE00F9423CBA82ECE0101965A
:10F660003C01B12C52E5952E66E4862E9CE49983EC
:10F670009A828B8282E48C83D3018D913D010E941A
:10F68000C242882319F00E94E5421DC0B1E0AB12CE
:10F6900031C1BB1528F0B11009C08FEB9FE00BC042
:10F6A000E2E0BE1206C08DEB9FE005C08EEB9FE04E
:10F6B00002C08CEB9FE00F9423CB682F772767FD68
:10F6C0007095872F972F611571058105910509F4B4
:10F6D00011C10F948ABF2FE632E143E85AE30F9439
:10F6E000BDC16B017C019F7727E139ED4EEC5DE3F5
:10F6F0000F94EBC018160CF033C0EAE5FEE08491DD
:10F700008F01882339F00E94F9420F5F1F4FF801E3
:10F710008491F7CFECE2FBE084918F01882339F0EC
:10F720000E94F9420F5F1F4FF8018491F7CF22E04A
:10F7300030E0B701A60184ED97E00E94FD41E3E2CD
:10F74000FBE084918F01882339F00E94F9420F5F1A
:10F750001F4FF8018491F7CF8AE00E94F942CAC096
:10F76000F2E0BF1609F469C023E0B21609F494C0B0
:10F7700031E0B31689F120E030E040E05FE3C701FB
:10F78000B6010F94BDC11B012C010CE411E1A201D3
:10F790009101D80114966D917D918D919C9117974F
:10F7A0000F940FBEF8016483758386839783A70146
:10F7B000960160817181828193810F940FBED8017F
:10F7C0006D937D938D939C931397045E1F4FB1E1CE
:10F7D000003A1B07E1F68EC020E030E040E05FE336
:10F7E000C701B6010F94BDC11B012C0100E511E159
:10F7F000A2019101F80160817181828193810F944E
:10F800000FBED8016D937D938D939C931397A701A1
:10F81000960114966D917D918D919C9117970F94FF
:10F820000FBEF8016483758386839783045E1F4F40
:10F83000F1E1043A1F07E1F65DC020E030E040E06E
:10F840005FE3C701B6010F94BDC11B012C010CE49D
:10F8500011E1A2019101D8015C966D917D918D918C
:10F860009C915F970F940FBEF801648F758F868F00
:10F87000978FA701960160817181828193810F9496
:10F880000FBED8016D937D938D939D938D01B1E152
:10F8900008351B07F1F62EC020E030E040E05FE3C2
:10F8A000C701B6010F94BDC11B012C0108E611E18F
:10F8B000A2019101F80160817181828193810F948D
:10F8C0000FBED8016D937D938D939D938D01A701FC
:10F8D000960158966D917D918D919C915B970F94B7
:10F8E0000FBEF801608F718F828F938FF1E1043723
:10F8F0001F07F1F6B39424E0B212B8CE8BE491E185
:10F900000E949CFA81E080934B110E94C9F2E09121
:10F91000220934E0E39FF0011124EC54F74E20E07B
:10F9200030E04EE353E460817181828193810F94D2
:10F93000EBC0181694F48091B309882371F086EA1D
:10F940009FE00F9423CB882341F08091BA189091C7
:10F95000BB18C29714F00C943F9581E090E090930F
:10F9600018028093170228964FAD289740937A0982
:10F970002A968EAD9FAD2A97909378098093770948
:10F980002C96AEADBFAD2C97B0937609A0937509B8
:10F99000109288091092870982E00F94FF840C94DA
:10F9A000C59480914B11882309F49CC0E9E1FBE0E8
:10F9B00084918F01882339F00E94F9420F5F1F4F15
:10F9C000F8018491F7CF4AE050E067E070E084ED01
:10F9D00097E00E942C41E7E1FBE084918F018823AE
:10F9E00039F00E94F9420F5F1F4FF8018491F7CF61
:10F9F0004AE050E067E070E084ED97E00E942C411F
:10FA0000E4E0FBE084918F01882339F00E94F94201
:10FA10000F5F1F4FF8018491F7CF4AE050E065E097
:10FA200070E084ED97E00E942C41E2EFFAE08491CF
:10FA30008F01882339F00E94F9420F5F1F4FF801B0
:10FA40008491F7CF8AE00E94F94200E010E03FEE97
:10FA5000A32E3AE0B32E4DEE842E4AE0942EE12CF4
:10FA6000F12C98012D503E4E6901F50184912FEE45
:10FA7000622E2AE0722E882341F00E94F942FFEFA5
:10FA80006F1A7F0AF3018491F6CFF601EE0DFF1D88
:10FA9000418152816381748125E030E084ED97E0FB
:10FAA0000E94FD41F4E0EF0EF11C2CE1E216F1049E
:10FAB000E1F6F40184919DEEE92E9AE0F92E882377
:10FAC00041F00E94F942FFEFEF1AFF0AF70184911B
:10FAD000F6CF0C5111090C33FFEF1F0709F0BFCF10
:10FAE0000C94C594EFECFAE084918F01882311F413
:10FAF0000C94BB6E0E94F9420F5F1F4FF801849176
:10FB0000F5CF86EE0E94EE460C94C5941092EC0858
:10FB10000C94C59485E40E94C242811102C00F94E6
:10FB2000891CFFEE6F2EF4E07F2EAAE28A2EA9E058
:10FB30009A2EB6E3AB2EB9E0BB2E512CD3018D919A
:10FB40003D010E94C2428823D9F1B3E05B120CC090
:10FB50000E94F042F501608371838283938382E483
:10FB600099E00F940D132CC00E94F042D4012D9106
:10FB70003D914D915C910F940FBEF50160837183AF
:10FB800082839383E0903E09F0903F090091400901
:10FB90001091410920913A0930913B0940913C096B
:10FBA00050913D096091360970913709809138096B
:10FBB00090913909E2E4CE2EE9E0DE2E0F949811FF
:10FBC0005394F4E08F0E911C24E0A20EB11C34E09B
:10FBD0005312B4CF0C94C59481E08093CB190F9449
:10FBE00011B66093BC097093BD098093BE099093D0
:10FBF000BF096091CB1984EC9FE00F9435CB0C9436
:10FC0000C59480910C0F90910D0F8F5E904F9F9334
:10FC10008F938AEB9AE09F938F930F944AC80F902B
:10FC20000F900F900F900C94C5948DE40E94C242E7
:10FC3000882311F40C949B93E091020FF091030F31
:10FC4000319681918032E9F38930D9F380538A303B
:10FC5000A0F080910C0F90910D0F8F5E904F9F93AD
:10FC60008F9385EA9AE09F938F930F944AC80F90E1
:10FC70000F900F900F900C94C5940E94F0420F9437
:10FC800057BF9B01693C710511F40C94BE8B0CF0BD
:10FC9000E6C06135710511F40C94AE870CF064C0B8
:10FCA0006931710509F42AC43CF56431710509F420
:10FCB000C5C394F46131710509F4B4C334F46230FE
:10FCC000710508F4F1C20C9488936231710511F446
:10FCD0000C94DD870C9488936631710509F4D7C3C1
:10FCE0000CF4CFC36731710509F4D7C368317105CE
:10FCF00009F4EEC30C9488936E31710509F447C47E
:10FD00008CF46B31710509F40DC40CF4FDC36C3136
:10FD1000710509F40DC46D31710511F40C94C5948D
:10FD20000C9488936C32710509F458C554F46F3102
:10FD3000710509F4FAC46032710509F460C40C94C9
:10FD400088936D32710509F458C56F32710511F051
:10FD50000C94889384E090E09093180280931702AB
:10FD60000F94DD5F0C94C5946E36710511F40C94FC
:10FD7000B588ACF56C35710511F40C943188A4F498
:10FD80006335710511F40C94D88714F40C94D4875E
:10FD90006435710511F40C94DD876535710511F436
:10FDA0000C9416880C9488936A36710511F40C949F
:10FDB000788754F46836710509F426C569367105EB
:10FDC00009F453C50C9488936B36710511F40C94A7
:10FDD000A8876D36710509F48DC60C948893673732
:10FDE000710511F40C94278ADCF46137710511F464
:10FDF0000C94C8884CF46037710511F00C9488930A
:10FE000063E087E495E01EC56237710511F40C9438
:10FE100022896337710511F40C94EE880C94889351
:10FE20006C38710509F410C57CF46837710511F45C
:10FE30000C94228A6937710511F00C94889381E043
:10FE40000F94CD140C94C5946E3B710509F4FCC657
:10FE5000683C710511F40C94498B0C948893663FAF
:10FE600041E0740711F40C94958F0CF08BC0603F47
:10FE7000710511F40C94C5940CF03FC06F3C7105F2
:10FE800011F40C94DF8C2CF56C3C710511F40C947E
:10FE9000F88B6CF46B3C710511F00C9488930FEEA9
:10FEA00014E03AEBE32E37E1F32E0C94E98B6D3C32
:10FEB000710511F40C941A8C6E3C710511F00C94C0
:10FEC00088930FEE14E02AE2E22E29E0F22E0C9441
:10FED000D08C613D710511F40C943A8D14F40C949E
:10FEE000148D6C3D710511F40C948C8D6D3D710574
:10FEF00011F40C949B8D0C9488936033B1E07B07D4
:10FF000011F40C94B28EDCF46D32F1E07F0711F441
:10FF10000C94F78D3CF42C32314011F40C94C18DCB
:10FF20000C9488932E3281E0380711F40C94468F9C
:10FF30002F32314011F40C94548F0C948893603913
:10FF4000A1E07A0711F40C948C8F4CF46E5571403B
:10FF50006230710510F40C94C5940C948893643F3E
:10FF6000E1E07E0711F40C948F8F653FF1E07F078D
:10FF700011F00C94889360E084E190E00E94583A7C
:10FF80000C94C5946E3843E0740711F40C942592D8
:10FF90002F3863E036070CF030C12A3582E038078D
:10FFA00011F40C94F191F4F42D3FA1E03A0711F40F
:10FFB0000C94988F54F4273F314011F00C9488939F
:10FFC00080E00E9402350C94C5942835F2E03F078A
:10FFD00011F40C9487902935324011F40C94E3917C
:10FFE0000C948893233563E0360711F40C94B58F95
:10FFF0000CF0F6C02D3B92E0390711F40C946E938F
:020000021000EC
:100000002E3B324011F00C94889350906A0210926B
:100010006A0281E080937A0982E090E09093780907
:1000200080937709E0918609F0E0EE0FFF1FE25020
:10003000F84B859194910F94964920E030E044E389
:1000400052E4609142097091430980914409909172
:1000500045090F940EBE6093420970934309809343
:10006000440990934509E0903E09F0903F090091C2
:1000700040091091410920913A0930913B09409182
:100080003C0950913D096091360970913709809182
:10009000380990913909E2E26E2EE9E07E2E7F92D6
:1000A0006F92812C912CFCEAAF2EF2E4BF2EA2E4D9
:1000B000CA2EA9E0DA2E0F9428060F94891C20E09E
:1000C00030E040E751E4609142097091430980912A
:1000D0004409909145090F940EBE609342097093B4
:1000E00043098093440990934509E0903E09F090BC
:1000F0003F09009140091091410920913A0930913E
:100100003B0940913C0950913D096091360970913D
:10011000370980913809909139097F926F92812C2B
:10012000912CB0E8AB2EB1E4BB2E0F9428060F94AF
:10013000891C20E030E040EA51E46091420970916E
:10014000430980914409909145090F940EBE609334
:100150004209709343098093440990934509E090C4
:100160003E09F0903F09009140091091410920910A
:100170003A0930913B0940913C0950913D09609109
:1001800036097091370980913809909139097F9229
:100190006F920F9428060F94891CE0918609F0E075
:1001A000EE0FFF1FEA5CF64B859194910E94E046AA
:1001B000149A64E670E080E090E00F9440B69FB738
:1001C000F894809102018460809302019FBF0F9098
:1001D0000F900F900F900F900F9010E00C9483935E
:1001E0002B38B3E03B0711F40C94FF912C383340CB
:1001F00011F40C94C5940C9488932339F3E03F07D1
:1002000011F40C948F92D4F4203963E0360711F482
:100210000C945A9214F40C942892213993E03907E3
:1002200011F40C948C922239334011F00C94889381
:10023000109218190F94AC370C94C5942639B3E07A
:100240003B0711F40C943C936CF42439F3E03F0722
:1002500011F40C9495922539334011F40C940A93BF
:100260000C948893203A63E0360709F431C2273EA4
:10027000334011F00C9488931092D6080F94C7491C
:100280008091EE0E9091EF0EA091F00EB091F10ED4
:100290008093F20E9093F30EA093F40EB093F50EAC
:1002A0000E9476530C94C5940091020F1091030F95
:1002B0000E5F1F4F80E50E94C242882379F00E94A2
:1002C000F0420F945CBF6B017C01BB24B3946115B9
:1002D00071058105910531F4B12C04C0B12CC12CFC
:1002E000D12C760183E50E94C242882399F00E94B6
:1002F000F04220E030E04AE754E40F94BDC10F948F
:100300005CBF6B017C01AA24A39461157105810572
:10031000910509F4A12C6AE270E0C8010F94AFC7FF
:10032000009711F0DC011C92F801CF0121912032DD
:10033000E1F3B11007C0A11005C0222319F00F94FA
:10034000894906C0E0EFF7E4859194910F949649AE
:1003500081E00F9469490F94891C0F9411B6609342
:10036000E8087093E9088093EA089093EB08C114B9
:10037000D104E104F104F1F00F9411B64B015C01DA
:100380008C0C9D1CAE1CBF1C84E090E09093180266
:10039000809317020F9411B6681579058A059B059D
:1003A00010F00C9481950F94244B81110C9481953D
:1003B0000C948C950F94224B882311F40C94C594C3
:1003C00084E090E090931802809317020F94244BDE
:1003D000811109C00F941B2981E00E94A85D80E073
:1003E0000F94FF84F3CF82E090E090931802809303
:1003F00017028091C209E0918609F0E0EE0FFF1F1D
:10040000882341F0E05EF64B859194910F949649D4
:100410000C94C594E658F84B859194910F949649A5
:100420000C94C594E4E9F9E4859194910F9496496C
:1004300017981698159814980C94C594E2E2FBE46A
:1004400005911491F8018491882329F00E94F942C2
:100450000F5F1F4FF7CF8AE00E94F94280EC99E0CE
:100460000E946BB6ECEBFAE405911491F8018491CB
:10047000882311F40C94BB6E0E94F9420F5F1F4F4A
:10048000F5CF80EC99E00E94D8BE0C94C59480EC26
:1004900099E00E94B2B60C94C5948091020F90919D
:1004A000030F6AE270E004960F94AFC7009711F053
:1004B000DC011C926091020F7091030F6C5F7F4F03
:1004C00021E041E080EC99E00E9406B90C94C594CB
:1004D0008091C409811102C00E94BE4780EC99E05E
:1004E0000E94B6B60F9411B66093E0087093E108CD
:1004F0008093E2089093E3080C94C59480EC99E013
:100500000E94BEB60C94C5948091C309882311F44F
:100510000C94C59483E50E94C24281110C94969577
:100520000C94C59480EC99E00E9433B70C94C59468
:100530008091020F9091030F6AE270E004960F948D
:10054000AFC78C010097A9F080910C0F90910D0F0F
:100550006EE470E08F5E904F0F94AFC760E270E082
:100560000F94AFC701969093030F8093020FF80189
:1005700010826091020F7091030F6C5F7F4F21E03A
:1005800040E080EC99E00E9406B90C94C5948091FB
:10059000C309882311F40C94C59460E080EC99E0C1
:1005A0000E94A5B88091020F9091030F6AE270E05B
:1005B00004960F94AFC78C010097A9F080910C0F9F
:1005C00090910D0F6EE470E08F5E904F0F94AFC767
:1005D00060E270E00F94AFC701969093030F809391
:1005E000020FD8011C926091020F7091030F6C5F93
:1005F0007F4F80EC99E00E948CC00C94C594809150
:10060000C20981110F94891C0091020F1091030FF0
:100610000C5F1F4F6AE270E0C8010F94AFC77C0106
:1006200061E270E0C8010F94AFC7009719F08C0128
:100630000F5F1F4FE114F10411F0F701108280E504
:100640000E94C242F82E2091020F3091030F021730
:10065000130708F4F12C8091C309882311F40C943A
:10066000C59421E02F2541E0B80180EC99E00E947B
:1006700006B983E50E94C2428823B9F02091020F97
:100680003091030F2017310780F40E94E542AB013F
:10069000BC014093D10C5093D20C6093D30C709357
:1006A000D40C8CE19CE00E94C2A980EC99E00E94ED
:1006B000B6B6F1100C94C5940F9411B66093E0088F
:1006C0007093E1088093E2089093E3080C94C5943A
:1006D0008091020F9091030F6AE270E005960F94EB
:1006E000AFC78C010097A9F080910C0F90910D0F6E
:1006F0006EE470E08F5E904F0F94AFC760E270E0E1
:100700000F94AFC701969093030F8093020FD80107
:100710001C926091020F7091030F6B5F7F4F80EC12
:1007200099E00E94D6BB0C94C5940F9411B66093C7
:10073000DC087093DD088093DE089093DF08009159
:10074000E0081091E1082091E2083091E308601B75
:10075000710B820B930B28EE33E040E050E00F94D6
:10076000BFC3CA01B9012CE330E040E050E00F9470
:10077000BFC37F936F933F932F9386E99AE09F9334
:100780008F93CE0101969F938F930F94F7C8E4E562
:10079000FEE084910FB6F894DEBF0FBECDBF04E536
:1007A0001EE0882339F00E94F9420F5F1F4FF801C5
:1007B0008491F7CF8E010F5F1F4FD8018D918D016E
:1007C000882319F00E94F942F8CF8AE00E94F9428A
:1007D000CE0101960F9489490C94C5948FEF0E9425
:1007E000EE4660E070E088EF9FE00F944FCB0E94F0
:1007F0001DDC0E94B0DC0C94C5948AE50E94C242C4
:100800000E9406510C94C59488E690E00E94EF5A2D
:1008100081110C94C59483E50E94C242882371F033
:100820000091D7080E94F04210E0000F111F0454FD
:10083000174E0F9457BFF801718360830F944026C1
:100840000C94C5940E94395A83E50E94C2428823C1
:1008500011F40C94C5940E94F0420F9457BF70930A
:10086000BB186093BA180C94C59489E690E00E9476
:10087000EF5A81110C94C594E0E9FAE084918F015C
:10088000882339F00E94F9420F5F1F4FF8018491CD
:10089000F7CFE091D70824E0E29FF0011124EC5457
:1008A000F74E408151816281738121E030E084ED17
:1008B00097E00E94FD41EDE8FAE084918F018823E2
:1008C00039F00E94F9420F5F1F4FF8018491F7CF72
:1008D000E091D708F0E0EE0FFF1FE454F74E60817F
:1008E0007181882777FD8095982F0F948ABFAB017F
:1008F000BC0121E030E084ED97E00E94FD41E9E891
:10090000FAE084918F01882339F00E94F9420F5F49
:100910001F4FF8018491F7CF40919E1850919F1876
:100920006091A0187091A11821E030E084ED97E06B
:100930000E94FD41E6E8FAE084918F01882339F0B6
:100940000E94F9420F5F1F4FF8018491F7CF609129
:10095000BA187091BB18882777FD8095982F0F944F
:100960008ABFAB01BC0121E030E084ED97E00E943A
:10097000FD41E3E8FAE084918F01882339F00E9479
:10098000F9420F5F1F4FF8018491F7CF4AE050E022
:1009900060E070E084ED97E00E942C41E1E8FAE02D
:1009A00084918F01882339F00E94F9420F5F1F4F15
:1009B000F8018491F7CF4091B4185091B518609127
:1009C000B6187091B71821E030E084ED97E00E94EE
:1009D000FD41EEE7FAE084918F01882339F00E940F
:1009E000F9420F5F1F4FF8018491F7CF6091BC1857
:1009F0007091BD18882777FD8095982F0F948ABF36
:100A0000AB01BC0121E030E084ED97E00E94FD41A4
:100A1000EAE7FAE084918F01882339F00E94F942D5
:100A20000F5F1F4FF8018491F7CF8091D70890E0B6
:100A30000F94E5234AE050E0BC0184ED97E00E946A
:100A40002C41E5E7FAE084918F01882339F00E9478
:100A5000F9420F5F1F4FF8018491F7CF8FEF9FEF9F
:100A60000F94E5234AE050E0BC0184ED97E00E943A
:100A70002C41E1E7FAE084918F01882339F00E944C
:100A8000F9420F5F1F4FF8018491F7CF4091AE18E4
:100A90005091AF186091B0187091B11821E030E01A
:100AA00084ED97E00E94FD41EDE6FAE084918F012C
:100AB000882339F00E94F9420F5F1F4FF80184919B
:100AC000F7CF4091A8185091A9186091AA18709179
:100AD000AB1821E030E084ED97E00E94FD418AE010
:100AE0000E94F94281E090E09093180280931702EF
:100AF0000C944D9A8DE690E00E94EF5A81110C946F
:100B0000C594E0918609F0E0EE0FFF1FE05CF54B25
:100B1000859194910F94964981E090E090937E099D
:100B200080937D098091CB19882321F081E090E0AA
:100B30000F94BF5583E50E94C242882391F0009133
:100B4000D7080E94F04210E0000F111F0454174E06
:100B50000F9457BFD8016D937C9381E08093080276
:100B600015C082E50E94C242882381F00091D70817
:100B70000E94F04210E0000F111F0454174E0F9412
:100B800057BFF80171836083109208020F944026CA
:100B90000F9411B66B017C010091D70810E0F801A9
:100BA000EE0FFF1FE454F74E60817181882777FDB7
:100BB0008095982F0F948ABFF801EE0FFF1FEE0F5C
:100BC000FF1FEC54F74E11E02081318142815381A7
:100BD0000F94EBC018160CF010E01093D50881E0CC
:100BE00090E0909318028093170210921109C701A8
:100BF000B6010E94AA5EE0918609F0E0EE0FFF1FA9
:100C0000E45CF54B859194910F94964982E090E0D5
:100C1000909318028093170290937E0980937D0928
:100C20008091CB19882321F082E090E00F94BF558A
:100C30000F9411B66093E8087093E9088093EA086E
:100C40009093EB080C94C594E0918609F0E0EE0FC8
:100C5000FF1FEC5AF44B859194910F94964983E0D1
:100C600090E090937E0980937D098091CB19882331
:100C700021F081E090E00F94BF5583E50E94C242CD
:100C8000882361F00E94F0420F9457BF7093BB1805
:100C90006093BA1881E0809308020FC082E50E9439
:100CA000C242882351F00E94F0420F9457BF7093C4
:100CB000BB186093BA18109208020F9411B64B013A
:100CC0005C01109211096091BA187091BB188827C5
:100CD00077FD8095982F0F948ABF11E020919E1880
:100CE00030919F184091A0185091A1180F94EBC01B
:100CF00018160CF010E01093D50881E090E0909366
:100D00001802809317020AE61AE036E6E32E3AE06C
:100D1000F32E42E6C42E4AE0D42E8091D50860918D
:100D2000BA187091BB18882309F4A8C080911109E2
:100D30008111A4C0882777FD8095982F0F948ABFD2
:100D400020919E1830919F184091A0185091A118A1
:100D50000F94EBC018160CF0A8C00F9411B66819C8
:100D600079098A099B09693E73408105910508F458
:100D70007CC08091CB19811174C0E091220924E0DC
:100D8000E29FF0011124EC54F74E408151816281C1
:100D90007381F80184912AE6A22E2AE0B22E8823DC
:100DA00001F165964FAF659766965FAF6697679658
:100DB0006FAF679768967FAF68970E94F942FFEF21
:100DC000AF1ABF0AF501849168967FAD6897679660
:100DD0006FAD679766965FAD669765964FAD659701
:100DE000DECF22E030E084ED97E00E94FD41F70184
:100DF000849196E6A92E9AE0B92E882341F00E94AC
:100E0000F942FFEFAF1ABF0AF5018491F6CF609166
:100E1000220970E04AE050E084ED97E00E942C4106
:100E2000F6018491B2E6AB2EBAE0BB2E882341F0E6
:100E30000E94F942FFEFAF1ABF0AF5018491F6CF85
:100E400040919E1850919F186091A0187091A11820
:100E500021E030E084ED97E00E94FD418AE00E94AD
:100E6000F9420F9411B64B015C010F941B2980E0ED
:100E70000E94A85D80E00F94FF844FCF882777FD04
:100E80008095982F0F948ABF20919E1830919F18BB
:100E90004091A0185091A1180F94E8BE87FF05C09B
:100EA00080910802882309F458CFE0918609F0E088
:100EB000EE0FFF1FE85AF44B859194910F949649D9
:100EC00082E090E0909318028093170284E090E013
:100ED00090937E0980937D090F9411B66093E80882
:100EE0007093E9088093EA089093EB080C94C594FA
:100EF00083E50E94C242882319F10E94F04220E05B
:100F000030E0A9010F94E8BE87FD0FC00E94F042B7
:100F100020E030E04FE753E40F94EBC0181644F0A4
:100F20000E94F0420F9457BF05C060E070E002C01D
:100F30006FEF70E070932109609320090C94C594C1
:100F40008FEF90E090932109809320090C94C59431
:100F500010922109109220090C94C5940F944126F7
:100F60000F94891C149A0F940B1D10922109109252
:100F7000200968EE73E080E090E00F9440B6109294
:100F80001902E2E9F9E44591549120E63AE06EE570
:100F90007AE08CE594E00E9432CD0F94964980E08F
:100FA0000F94FF840C94C5941092BB090C94C594C3
:100FB00081E08093BB090C94C59483E50E94C242F2
:100FC000882399F00E94F04220E030E04AE754E4A0
:100FD0000F94BDC10F945CBF60930A0270930B0223
:100FE00080930C0290930D021DC088E50E94C242BE
:100FF00081110C94A79589E50E94C24281110C943D
:10100000A7958AE50E94C24281110C94A79585E4B8
:101010000E94C24281110C94A7950F94891C149AC6
:101020000F940B1D109274090C94C59483E50E94D3
:10103000C242882311F40C94C5940E94F04220E02F
:1010400030E04AE754E40F94BDC10F945CBF609355
:10105000E4087093E5088093E6089093E7080C9401
:10106000C5942FEE34E039AF28AF0AEA17E16AEBF6
:10107000C62E67E1D62E7AE6E72E77E1F72E312CE1
:10108000A8ADB9AD8D91B9AFA8AF0E94C242882377
:1010900009F45CC0B3E03B1252C00E94F0422B0145
:1010A0003C0120E030E040EA51E40F94E8BE87FFC5
:1010B0003FC0A3019201F801608171818281938117
:1010C0000F94EFBE4B015C019B01AC0160918A174C
:1010D00070918B1780918C1790918D170F94BDC1D3
:1010E00060938A1770938B1780938C1790938D174A
:1010F000A5019401D6016D917D918D919C910F94E4
:10110000BDC1F6016083718382839383D7016D91A2
:101110007D918D919C910F9488BFA50194010F94AE
:10112000BDC10F945CBFF701608371838283938399
:10113000D8014D925D926D927C92139707C00E94E8
:10114000F042F801608371838283938333940C5F50
:101150001F4FF4E0CF0ED11C24E0E20EF11C34E06E
:10116000331611F40C94C5948BCF8EE40E94C242C6
:10117000882311F40C94C5940E94E5426093F20E0A
:101180007093F30E8093F40E9093F50E0C94C59427
:1011900083E50E94C242882331F00E94D8428093A6
:1011A00012020C94C594E4E5FEE084918F0188233B
:1011B00039F00E94F9420F5F1F4FF8018491F7CF79
:1011C0004091120250E060E070E087E59AE00E94F2
:1011D0001C478AE00E94F9420C94C59486E50E945F
:1011E000C242882371F00F9454B28C01F8018491AB
:1011F000882311F40C94BB6E0E94F9420F5F1F4FBD
:10120000F5CF85E50E94C242882369F08091020FE4
:101210009091030F01969093030F8093020F0F9408
:10122000C5B40C94C594E2EFF9E405911491F8016A
:101230008491882311F40C94C5940E94F9420F5FA5
:101240001F4FF5CFE4E5FAE084918F01882339F050
:101250000E94F9420F5F1F4FF8018491F7CF409130
:10126000360950913709609138097091390922E0A7
:1012700030E084ED97E00E94FD41E0E5FAE08491E2
:101280008F01882339F00E94F9420F5F1F4FF80148
:101290008491F7CF40913A0950913B0960913C0904
:1012A00070913D0922E030E084ED97E00E94FD411D
:1012B000ECE4FAE084918F01882339F00E94F9422E
:1012C0000F5F1F4FF8018491F7CF40913E09509175
:1012D0003F09609140097091410922E030E084EDBE
:1012E00097E00E94FD41E8E4FAE084918F018823B1
:1012F00039F00E94F9420F5F1F4FF8018491F7CF38
:101300004091420950914309609144097091450907
:1013100022E030E084ED97E00E94FD41ECEEFAE43B
:1013200005911491F8018491882329F00E94F942D3
:101330000F5F1F4FF7CF0F94EA1C0F948ABF2091C5
:10134000AA173091AB174091AC175091AD170F947D
:10135000EFBEAB01BC0122E030E084ED97E00E94DB
:10136000FD41E4E4FAE084918F01882339F00E9482
:10137000F9420F5F1F4FF8018491F7CF81E00F947E
:10138000EA1C0F948ABF2091AE173091AF1740919D
:10139000B0175091B1170F94EFBEAB01BC0122E022
:1013A00030E084ED97E00E94FD41E0E4FAE08491B2
:1013B0008F01882339F00E94F9420F5F1F4FF80117
:1013C0008491F7CF82E00F94EA1C0F948ABF20919A
:1013D000B2173091B3174091B4175091B5170F94CD
:1013E000EFBEAB01BC0122E030E084ED97E00E944B
:1013F000FD41ECE3FAE084918F01882339F00E94EB
:10140000F9420F5F1F4FF8018491F7CF83E00F94EB
:10141000EA1C0F948ABF2091B6173091B7174091FC
:10142000B8175091B9170F94EFBEAB01BC0122E081
:1014300030E084ED97E00E94FD418AE00E94F9428D
:101440000C94C59480E00F94CD140C94C594ECEEEC
:10145000F9E405911491F8018491882329F00E9400
:10146000F9420F5F1F4FF7CF8AE00E94F942E0E98F
:10147000F7E405911491F8018491882329F00E94E2
:10148000F9420F5F1F4FF7CF1E9B15C0E0ECFAE447
:1014900005911491F8018491882329F00E94F94262
:1014A0000F5F1F4FF7CF8AE00E94F942E2E9F7E4AD
:1014B000059114910DC0EEEBFAE405911491F80139
:1014C0008491882381F30E94F9420F5F1F4FF7CF69
:1014D000F8018491882329F00E94F9420F5F1F4F81
:1014E000F7CF8091060182FF15C0E0ECFAE4059188
:1014F0001491F8018491882329F00E94F9420F5F2A
:101500001F4FF7CF8AE00E94F942E4E8F7E4059123
:1015100014910DC0EEEBFAE405911491F801849159
:10152000882381F30E94F9420F5F1F4FF7CFF80124
:101530008491882329F00E94F9420F5F1F4FF7CF53
:101540001D9B15C0E0ECFAE405911491F80184911B
:10155000882329F00E94F9420F5F1F4FF7CF8AE0DE
:101560000E94F942E6E8F7E4059114910DC0EEEB14
:10157000FAE405911491F8018491882381F30E9483
:10158000F9420F5F1F4FF7CFF8018491882329F0AC
:101590000E94F9420F5F1F4FF7CF8091060187FF2E
:1015A00015C0E0ECFAE405911491F80184918823C8
:1015B00029F00E94F9420F5F1F4FF7CF8AE00E9487
:1015C000F942EEE7F7E4059114910DC0EEEBFAE471
:1015D00005911491F8018491882381F30E94F942C6
:1015E0000F5F1F4FF7CFF8018491882329F00E94E5
:1015F000F9420F5F1F4FF7CF1C9B15C0E0ECFAE4D8
:1016000005911491F8018491882329F00E94F942F0
:101610000F5F1F4FF7CF8AE00E94F942E0E8F7E43E
:10162000059114910DC0EEEBFAE405911491F801C7
:101630008491882381F30E94F9420F5F1F4FF7CFF7
:10164000F8018491882329F00E94F9420F5F1F4F0F
:10165000F7CF01990FC0E0ECFAE405911491F8017D
:101660008491882311F40C94BB6E0E94F9420F5FA1
:101670001F4FF5CFEEEBFAE405911491F801849138
:10168000882311F40C94BB6E0E94F9420F5F1F4F28
:10169000F5CF809122098093D70884E50E94C24249
:1016A000882319F10E94F0420F945CBF6093D70821
:1016B0006623D9F0E4E5FEE084918F01882339F0B8
:1016C0000E94F9420F5F1F4FF8018491F7CFEAEEB5
:1016D000F9E405911491D8018D918D01882311F4BD
:1016E0000C94C5940E94F942F6CF84E40E94C24251
:1016F000882311F40C94C5940E94F04220E030E05D
:10170000A9010F94E8BE811103C01092460932C0AE
:101710000091D70810E00E94F042F801EE0FFF1F81
:10172000EE0FFF1FEA5BFD4F60837183828393831B
:10173000E0904602F0904702009148021091490261
:1017400020E030E0A901B701C8010F94E8BE811183
:1017500004C0E12CF12C00E410E4C701D80180930F
:10176000460290934702A0934802B093490281E059
:10177000809346090E94305C0C94C5940FEE14E0EF
:101780004AE9E42E47E1F42EF80181918F010E948D
:10179000C242882351F00E94F0420F945CBFD701EF
:1017A0006D937D938D939C931397B4E0EB0EF11C96
:1017B000E4E0033F1E0741F70F9433130C94C594E4
:1017C000F4E0EF0EF11C24E0033F120711F40C9437
:1017D000C594D8018D918D010E94C242882381F366
:1017E0000E94F042F7016083718382839383E8CF84
:1017F00083E50E94C242882351F00E94F042609328
:10180000921770939317809394179093951784E58C
:101810000E94C242882311F40C94C5940E94F042A5
:1018200060938E1770938F178093901790939117F2
:101830000C94C59483E50E94C242882351F00E9413
:10184000F042609396177093971780939817909330
:10185000991784E50E94C242882351F00E94F04209
:1018600060937A1770937B1780937C1790937D1702
:1018700082E40E94C242882361F00E94F0420F94E9
:101880005CBF6093CA177093CB178093CC1790936B
:10189000CD1788E50E94C242882391F00E94F04251
:1018A00060938217709383178093841790938517A2
:1018B00060937E1770937F178093801790938117A2
:1018C00089E50E94C242882351F00E94F042609351
:1018D00082177093831780938417909385178AE5F6
:1018E0000E94C242882351F00E94F0426093861702
:1018F00070938717809388179093891785E40E94C7
:10190000C242882351F00E94F04260938A1770937C
:101910008B1780938C1790938D1720E030E040E276
:1019200051E460917E1770917F178091801790919C
:1019300081170F94EBC0181664F480E090E0A0E2E9
:10194000B1E480937E1790937F17A0938017B09394
:10195000811720E030E040E251E4609182177091FD
:10196000831780918417909185170F94EBC01816F8
:1019700014F00C94C59480E090E0A0E2B1E4809370
:10198000821790938317A0938417B0938517FDC790
:10199000F4E0EF0EF11C24E0023F120709F4F5C752
:1019A000D8018D918D010E94C242882389F30E9443
:1019B000F042F7016083718382839383E9CF83E5EB
:1019C0000E94C242882351F00E94F0426093260296
:1019D00070932702809328029093290286E40E9444
:1019E000C242882381F00E94F04220E030E040E7CC
:1019F00052E40F94EFBE60931E0270931F02809317
:101A00002002909321028AE50E94C242882309F4B1
:101A1000BCC70E94F04260931A0970931B0980931F
:101A20001C0990931D09B1C783E50E94C242882317
:101A300051F00E94F0426093160970931709809349
:101A400018099093190986E40E94C242882309F478
:101A50009CC70E94F04220E030E040E752E40F943F
:101A6000EFBE60931A0270931B0280931C02909346
:101A70001D028BC783E50E94C242882309F485C7F3
:101A80000E94F0420F9457BF6115710549F0613013
:101A9000710559F481E080931F0910921E0975C7E2
:101AA00010921F0910921E0970C7E4E5FEE08491B0
:101AB0008F01882339F00E94F9420F5F1F4FF80110
:101AC0008491F7CFE2E0F8E405911491F801849154
:101AD000882329F00E94F9420F5F1F4FF7CF009132
:101AE0000C0F10910D0F0F5E104FD8018D918D01CD
:101AF000882319F00E94F942F8CFE7E3FAE08491D5
:101B00008F01882311F40C94BB6E0E94F9420F5F81
:101B10001F4FF8018491F5CF83E50E94C2428823CC
:101B200009F433C70E94F0420F9457BF70935902D3
:101B3000609358022AC783E50E94C242882309F4B1
:101B400024C70E94F0420F9457BF6B017C0184E5CB
:101B50000E94C242882381F08DED90E00E94EF5AEE
:101B6000811113C7E091D708F0E0EE0FFF1FEC5A88
:101B7000FD4FD182C08209C7D0925702C09256024F
:101B800004C783E50E94C242882331F00E94F042DC
:101B90000F9457BF8B0102C00EE610E080E50E9453
:101BA000C242882331F00E94F0420F9457BFCB010C
:101BB00002C088EE93E06C01EE24D7FCE094FE2C8A
:101BC000101611067CF420E030E0A901B80184E58C
:101BD0000F9469BAC701B6010F9440B684E50F941B
:101BE0008DBDD3C6C701B6010F9440B6CEC680E501
:101BF0000E94C242882351F00E94F0426093AA02E0
:101C00007093AB028093AC029093AD0289E40E9482
